S31508001800001D0020DD180008EB180008ED18000878
S3150800181000000000000000000000000000000000BA
S315080018200000000000000000000000000519000884
S31508001830000000000000000007190008594D0008C4
S31508001840F95600080B1900080B1900080B190008AF
S315080018500B190008912C0008B52C0008D92C000893
S315080018600B1900080D2A0008452A0008812A0008D5
S31508001870C12200080B1900080B190008B94F000807
S315080018807950000800000000000000000B1900084D
S31508001890000000000B1900080B1900080B190008B6
S315080018A0000000000B1900080B1900086153000816
S315080018B00B1900080B1900080B1900080000000096
S315080018C0EE11AA550448854600F0ACFC00480047CE
S315080018D02D760008C046C046001D00200B4880F340
S315080018E008880B4880470B480047FEE704207146E6
S315080018F0084202D0EFF3098001E0EFF30880714651
S3150800190005F030FCFEE7FEE7FEE7FEE7001D0020D7
S315080019101D4F0008C518000830B50B4601460020C3
S315080019202022012409E00D46D5409D4205D31D46D7
S315080019309540491B2546954040191546521E002DCF
S31508001940F1DC30BD70B500242546002801DA0124F3
S315080019504042002901DA01254942FFF7DDFFAC4282
S3150800196000D04042002C00D0494270BD03460B43CC
S315080019709B0703D009E008C9121F08C0042AFAD237
S3150800198003E00B780370401C491C521EF9D27047BD
S31508001990D2B201E00270401C491EFBD270470022F9
S315080019A0F6E710B513460A4604461946FFF7F0FF50
S315080019B0204610BDF8B502464A40D40F42004B00F7
S315080019C052085B089A4202D20246084611464A0065
S315080019D023D0C30D4A00DDB2120EAD1A202D35DA1A
S315080019E049020126490AF6058A19002C00D05242F6
S315080019F020214F1B1146B9402A411018C20D9A42A0
S31508001A0021D0002C17D0012D08DCDA05801AD20F58
S31508001A108019D207DBB200F022FBF8BDDA05801A7E
S31508001A20012340001B06C01880185A428018CA0FA6
S31508001A301043490007E04908C2071143DA05801A2E
S31508001A4080194008801800F002FBF8BD61000122E9
S31508001A50511A001BF7E70122D2075140AAE70122D3
S31508001A60D2075040A6E7024670B54A40D30FDB07B7
S31508001A7040002DD04A002AD0010E140E0002120290
S31508001A800919400A520A8418E50104465443000A13
S31508001A90120A2E045043A4194219200CC543AA1849
S31508001AA0120C0125AD03521C521912047F39240465
S31508001AB000D0521C104301D44000491EC2B20C0685
S31508001AC0C0092018401C4008802A02D003E00020E4
S31508001AD070BD40084000002900DA0020184370BD98
S31508001AE070B502464A40D50F40004A00ED07400847
S31508001AF05208002814D0002A12D0C40DD30D410272
S31508001B000120C0055202490A520AE41A0918121895
S31508001B107D34914201D3641C00E04900002C01DAAF
S31508001B20002070BD0023914201D3891A034340085F
S31508001B3049000028F7D100290AD0914202D1012193
S31508001B40C90705E0914201D2012101E00121C943FB
S31508001B50E005C018401900F07AFA70BDF0B50746DE
S31508001B600846584087B0C00F049048000E465900F2
S31508001B7040084908BC1A884105D2384631461E46EF
S31508001B8017460B4602465800400810434DD0300D04
S31508001B90039040055900400D490D0590401A0290E2
S31508001BA0402873DA18030121000B09050843019040
S31508001BB004980092002806D01146019A494200204E
S31508001BC0904100910190029840210A1A01990098C3
S31508001BD000F01AFA05460C466B4607CB00F024FAC5
S31508001BE0C0197141039A0E0D0023D71756401A469D
S31508001BF07A40164344D0049A002A2DD0029A012A24
S31508001C00039A15DC1205C01A914101263605001CF7
S31508001C107141D20F059ED2070093019202962A4679
S31508001C20234600F062FA07B0F0BD38463146FAE7B7
S31508001C301605234A0F46B218C01AB74101210905ED
S31508001C40001C4F4100187F41114618187941E20FD0
S31508001C5010436D19644113E0E2076D0815436408E3
S31508001C60C2071443039A01261205C01A9141360584
S31508001C70001C7141CE07400830434908C01851413D
S31508001C802A46234600F024FACDE7FFE70498012206
S31508001C904000C117121A00238B4104983146C41715
S31508001CA0381AA141EEE730B40124E407634030BC9A
S31508001CB054E730B40124E407614030BC4EE7000025
S31508001CC00000E0FFF0B51FB488B00B99099800240E
S31508001CD048400999C00F490049080991C0070B995E
S31508001CE00090490049080B9109990898A6460843A7
S31508001CF01CD00B990A98084318D00998012440006B
S31508001D00420D4800410D099824050003000B2043A5
S31508001D1009900B980003000B20430B9050181C49A0
S31508001D204018002201901446104605E0002001469E
S31508001D300DB0F0BD032801DA034600E003239C46F4
S31508001D40C11A0AAE0AE05F0008ADED5B4F00F75B0B
S31508001D507D430027AA187C41491C5B1E6145F2DDBC
S31508001D60410004AB5A522104120C0A43240C401CAD
S31508001D700828DFDB019802900099704601910090CF
S31508001D80059B049A0799069800F0AFF9D0E700007A
S31508001D900DFCFFFFF0B50C465C4085B0E40FE40788
S31508001DA003944C00002664085900944649080246E4
S31508001DB00296224321D062460A431ED06200570D7E
S31508001DC04A000E032303550D012402462C49240517
S31508001DD0781B1B0B360B401823432643614600909D
S31508001DE01C46501AB44103D30098401C009002E0E8
S31508001DF0921800985B41002803DA0020014605B0D6
S31508001E00F0BD0020012109050746864611E0644613
S31508001E101D46141BB54106D36546521BB34174468D
S31508001E2007430C43A646CD0740084908284392189D
S31508001E305B4105460D43EAD11046184313D0604668
S31508001E40194650407140084306D06046101AB341FF
S31508001E5006D20122002306E000220123DB0702E066
S31508001E600122D2435310009874460105381C61417B
S31508001E70029C039D0019694100F02AF9BFE700009A
S31508001E80FD030000C217C10F504010B54018CA071D
S31508001E909623002100F0E3F810BD10B50022962322
S31508001EA0114600F0DCF810BD410040020122400A4C
S31508001EB0D205090E80187F2901DA00207047962975
S31508001EC003DC9622511AC8407047963988407047F5
S31508001ED0C20FD207400040080BD0C10D0723DB0113
S31508001EE0C91840020905400A1143C20840071143B0
S31508001EF0704700200146704710B5002904DB01240D
S31508001F00E40740428C412146002B04DB1C46012392
S31508001F10DB075242A3418B4200D1824210BD00002A
S31508001F2010B5002904DB0124E40740428C41214610
S31508001F30002B04DB1C460123DB075242A3419942CE
S31508001F4000D1904210BD0000CB0FDB07490010B549
S31508001F50490802460A4307D00A0D07240903E40183
S31508001F60090B121B002A01DC002010BDC900440F12
S31508001F700C43C100E018D205801800F068F810BDBF
S31508001F800122D207002800DB101A002900DB511AAB
S31508001F90814270470122D207002800DB101A002967
S31508001FA000DB511A88427047F0B51FB40646002078
S31508001FB082B005464024019100901BE00199224613
S31508001FC00F46304600F040F9049A059B801A99415D
S31508001FD010D310461946224600F016F8361A8F41D5
S31508001FE00197224601200021009F00F00DF83818BD
S31508001FF04D4100902046641E0028DFDC019B0098B6
S315080020002946324607B0F0BD10B5202A04DB014642
S31508002010203A9140002010BD914020239C1A034687
S31508002020E3401943904010BD10B5202A06DBCB17B4
S315080020300846203A1041C1170B4306E00B461341E8
S31508002040D0402024A21A91400843194610BD002901
S3150800205004DA401C490001D140084000704770B4BA
S315080020600024050C05D11024000402D1002921D032
S315080020701124050E01D100020834050F01D1000113
S31508002080241D850F01D18000A41C002801DB400017
S31508002090641C002908D020252E1B0D46F540A140BA
S315080020A000D001212943084301061B1B000ADB1D3A
S315080020B002D5002070BC7047DB0518188018002967
S315080020C0F8DA401C4900F5D170BC4008400070475A
S315080020D010B5002B08DA0024401C614192185B41B8
S315080020E01A4301D14008400010BDF0B51FB482B0B4
S315080020F005460C0003D0084603F040FB02E003F057
S315080021003DFB20300246009021462846FFF77CFF1B
S31508002110049B059A04460F4618431143084314D0F6
S31508002120184610431BD0009840210A1A18460599EC
S3150800213000F08AF805460E46009A05990498FFF7B6
S3150800214063FF084305D0012004E02046394607B05E
S31508002150F0BD0020C11705430E432C4337430099B1
S315080021600E986305401A7905E40A00220C43FD0A15
S315080021700A3002D500200146E9E701051019694130
S315080021800C9C0D9D00196941FFF7A2FFDFE770B5AA
S315080021904B005B0803430BD04B005C0D002633460F
S315080021A06542B341D417AD1AA34102DB00200146AC
S315080021B070BD12053018514170BD00000EB5C2172A
S315080021C0C10F5040CA0740180021054B02930192DF
S315080021D000910A460B46FFF788FF03B000BD0000D2
S315080021E0330400004A0009030123090B1B051943A0
S315080021F00A4B10B5520D9A4202DA0020014610BD6C
S31508002200064B34339A4203DC9A1A00F01DF810BDC7
S31508002210034BD218FFF7F8FE10BD0000FF030000BD
S31508002220CDFBFFFF064C0125064E05E0E36807CC0B
S315080022302B430C3C98471034B442F7D3FFF746FBC0
S31508002240B8DF0008D8DF000810B5202A04DB0846E6
S31508002250203AD040002110BD0B46D340D040202460
S31508002260A21A91400843194610BD70B58C18057816
S31508002270401C6B075B0F01D10378401C2A1106D15D
S315080022800278401C03E006780E70401C491C5B1E51
S31508002290F9D12B0705D40023521E0DD40B70491C07
S315080022A0FAE70378401CCB1A921C03E01D780D70E0
S315080022B0491C5B1C521EF9D5A142D8D3002070BD1B
S315080022C010B50121064800F042F9002806D0012081
S315080022D0044908600121024800F08AF810BD000090
S315080022E0002401400802002070B587B00020049041
S315080022F005900690009001900290039001242EE02C
S31508002300002520E0A800281886B20CE0F00016493F
S3150800231040186100405AA9006918711A490004AAB0
S315080023205052701C86B2681C81004018B042EDDC21
S3150800233004A800F0A7FAA1006A4651584018A1005F
S315080023405050681C85B2042DDCDBA000694608588D
S315080023508003000C6100054A5052601C84B2042CAC
S31508002360CEDB07B070BD0000501600201202002018
S3150800237030B50907090F08290CDAC36D8D000F243B
S31508002380AC40A343C365C36D8D001446AC402343DC
S31508002390C3650FE0036E0C46083CA5000F24AC404D
S315080023A0A3430366036E0C46083CA5001446AC40DE
S315080023B02343036630BD002904D0826E01231A43E5
S315080023C0826603E0826E52085200826670470F29C1
S315080023D000DD0F2141667047012904D142690123B6
S315080023E01A43426103E0426902231A434261704775
S315080023F0012904D1426901231A43426103E0426973
S3150800240002231A4342617047002904D04268012317
S315080024101A43426003E0426852085200426070471D
S3150800242000B589B00121480201F046FB03A800F077
S3150800243021F90020039070200490012040020590A5
S3150800244000216846017600200790089003A93448C1
S3150800245000F0A4F8072300221146314800F0BAF824
S315080024600723002201212E4800F0B4F80723002292
S315080024700C212B4800F0AEF802212948FFF7A7FFE8
S31508002480002211462648FFF773FF01221146244809
S31508002490FFF76EFF0C2202212148FFF769FF012191
S315080024A01F48FFF788FF01211D48FFF795FF012206
S315080024B011461B4800F056F80121480401F0DCFAE1
S315080024C00121880401F0D8FA02A801F004F80321D2
S315080024D068460181012181720021C17202A9092081
S315080024E0C00600F081FF02A800F0F5FF80216846CB
S315080024F00181012181720021C17202A9094800F0F7
S3150800250073FF0C216846017101214171817101A88F
S3150800251001F0F4F801210248FFF776FF09B000BD83
S315080025200024014000040048002904D082680823DA
S315080025301A43826003E0826808239A4382607047E0
S3150800254002468B0010461830C05880B270470246C3
S31508002550012902D150690840704750690223184082
S315080025604008F9E710B501290BD1002A04D0836881
S315080025700124234383600FE083685B085B00836064
S315080025800AE0002A04D0836802242343836003E018
S3150800259083680224A343836010BD000042680B4B86
S315080025A01A4042600B684A681A4343681A434260F5
S315080025B08268074B1A4082600B694A691A438B681E
S315080025C01A4383681A438260704700000FBCFFFFF6
S315080025D08FF1F9FFF0B504460D4616461F463F072C
S315080025E03F0F2B46082B0FD91B071B0F083B606FA5
S315080025F09A000F21914088436067606F99003A46B8
S315080026008A40104360670BE0206F9A000F219140C3
S3150800261088432067206F99003A468A40104320670E
S31508002620E0680121A9408843E060E0680121A940EB
S315080026300843E060012080032840002803D00120D9
S3150800264000F020F807E00120C0032840002802D047
S31508002650012000F017F8F0BD002905D08268FF2395
S3150800266001331A43826004E08268FF2301339A43E8
S3150800267082607047002101604160816001730161D9
S3150800268041617047002806D0064949680C22114363
S31508002690044A516005E0034949680C229143014AFE
S315080026A0516070470024014000B503461846FFF7FD
S315080026B0E9FF00BD10B503F0E7FD064800780028DD
S315080026C006D0FFF711FE00200249087000F00CFF43
S315080026D010BD000010020020FFB583B00C4602941E
S315080026E000200190002726E000261CE0721C0399B2
S315080026F051430846791CFFF70FF90546A54201D94B
S31508002700281B00E0601B05460298A84204D90295DA
S3150800271005980670069807700298002802D10120CD
S31508002720019002E0761C402EE0D300BF01980028F5
S3150800273000D002E07F1C042FD6D300BF029807B052
S31508002740F0BD000000BF00BF00BF00BF00BFBFF361
S315080027504F8F00BF00BF00BF06480749C86000BFCB
S3150800276000BF00BFBFF34F8F00BF00BF00BF00BF51
S3150800277000BFFDE70400FA0500ED00E010B500F023
S3150800278001F810BD10B523480078002817D1224853
S3150800279001F01AFA01283CD11F480078002838DDD4
S315080027A01D480078402834DC02F0AEFD1B4908605D
S315080027B001201849087000201949087029E0164AAE
S315080027C017490978491C501801F0FEF9012816D155
S315080027D013480078401C124908700F480078097899
S315080027E0884216D100200B4908700B484078FF280C
S315080027F00FD10B48007802280BD1FFF7A3FF02F090
S3150800280083FD064909686431884202D900200149D6
S31508002810087010BD3D0100202C0400204001002056
S315080028203C01002078B50246002327E0002020E07E
S315080028308400155B441CA400145BA54218DD8400C3
S31508002840A5182E886C4626806D8865808400A51894
S31508002850441CA400A41826882E8064886C80441C16
S31508002860A400A5186C4624882C806C4664886C8065
S31508002870401C4C1EE41A8442DADC5B1C4C1E9C424B
S31508002880D4DC78BD30B5014600231AE0002212E0F8
S3150800289050000D5A501C4000085A854209DD500068
S315080028A00C5A501C4000085A55004853501C40000A
S315080028B00C52501C82B20420C01A9042E8DC581C04
S315080028C083B2032BE2DB888830BD000010B586B0E2
S315080028D004460121880301F0EFF80121880401F07C
S315080028E0CBF803221146224800F0CBFD032204212F
S315080028F01F4800F0C6FD01A802F0D7FD019430215B
S315080029006846018100214181818101821821C181A6
S3150800291001A9184802F086FD0121164802F05FFD5C
S3150800292005A800F0D8FD0821684681820121817535
S315080029301821C17505A90E4800F056FD10216846F4
S3150800294081824821C17505A9094800F04DFD1B2162
S3150800295068460170032141700121817000F0CEFEA6
S3150800296001220221034802F052FD06B010BD000004
S31508002970000400480038014070B502460B46FF25A2
S31508002980FF2408E01178521C69400748405C604003
S3150800299005460648445C18465E1EB3B20028F1D1C7
S315080029A02802204370BD0000AADC0008AADD000842
S315080029B001B504490098086000BF0248006800286D
S315080029C0FBD108BD48010020014600220E4B1A61C2
S315080029D0CA005A6100229A6105221A6100BF0A4A92
S315080029E01069C207D20F002A04D00122120402403D
S315080029F0002AF4D0044A126952085200024B1A619E
S31508002A0000229A617047000000E000E010B500213E
S31508002A100948FFF721FE022000F056F80021064873
S31508002A20FFF782FD01200549087003F0E3FB00214A
S31508002A300348C17110BD0000002401407801002040
S31508002A402004002010B5202000F066F8002805D0E4
S31508002A50012009490860202000F036F801204002CC
S31508002A6000F05AF8002805D0012004490860400201
S31508002A7000F02AF810BD0000DC010020E00100206B
S31508002A8010B50120400300F047F8002805D00120C2
S31508002A9008490860400300F017F80120400400F0D8
S31508002AA03BF8002805D0012003490860400400F0DF
S31508002AB00BF810BDE4010020E80100200149486038
S31508002AC07047000000000240014948607047000056
S31508002AD0000002400268520852000A43026070472A
S31508002AE010B5044620684008400020600020206099
S31508002AF06060A060E060E1B2084608380521FEF78C
S31508002B000BFF01460F2088400249496808430149DE
S31508002B10486010BD000002400146044800680840AD
S31508002B20002801D0012070470020FCE70000024081
S31508002B30002A03D003680B43036002E003688B4353
S31508002B400360704710B50A7A8B7D1A430B7C1A43CB
S31508002B504B7C1A434B8A1A438B8A1A430B8B1A43AC
S31508002B604B8B1A430368094C23401A4302600268D8
S31508002B700123DB039A438B8B1A430260CA684260BF
S31508002B800A6882604A68C26010BD00000F80FFFFB5
S31508002B900021016041600172C16001744174418283
S31508002BA081828175018341838183704770B50646AA
S31508002BB00C4621460A4800F01FFA0546002D01D1A9
S31508002BC0401E70BD0648854202D10648051B00E036
S31508002BD02D1B224629463046FEF7C8FE2046F0E75A
S31508002BE000F4000800FC000870B506460C462146AD
S31508002BF00A4800F001FA0546002D01D1401E70BDB5
S31508002C000648854202D10648051B00E02D1B2246D0
S31508002C1029463046FEF7AAFE2046F0E700F00008EF
S31508002C2000F8000870B506460C4621460A4800F02A
S31508002C30E3F90546002D01D1401E70BD06488542C0
S31508002C4002D10648051B00E02D1B224629463046C0
S31508002C50FEF78CFE2046F0E700F8000800000108A1
S31508002C6070B505460C4622460249284600F085F905
S31508002C70204670BD00F4000870B505460C4622468D
S31508002C800249284600F079F9204670BD00F0000890
S31508002C9010B5012000F038F8002805D0034804498B
S31508002CA00880012000F02AF810BD000088130000F3
S31508002CB0D400002010B5082000F026F8002805D01A
S31508002CC0034804490880082000F018F810BD0000E1
S31508002CD088130000D400002010B5202000F014F856
S31508002CE0002805D0034804490880202000F006F88B
S31508002CF010BD000088130000D40000200149486177
S31508002D007047000000040140014607484069084032
S31508002D10002806D0044800680840002801D0012091
S31508002D2070470020FCE70000000401408179002973
S31508002D3048D02D490968026891432B4A116011460B
S31508002D40496802689143284A51600179002906D1E9
S31508002D501146096802681143234A116005E02249B1
S31508002D60496802681143204A51601F498968026808
S31508002D7091431D4A91601146C968026891431A4AEF
S31508002D80D160417910290CD111468968026811432E
S31508002D90154A91601146C96802681143124AD16002
S31508002DA020E04179082906D10F498968026811434C
S31508002DB00D4A916016E00C49C968026811430A4A2F
S31508002DC0D1600FE00179002906D107490968026830
S31508002DD09143054A116005E0034949680268914331
S31508002DE0014A5160704700000004014010B50D4AC1
S31508002DF08B109B00D3588A07140F0F22A2409343C7
S31508002E00084A8C10A40013518B109B00D2588B07CC
S31508002E101C0F0346A3401A43024B8C10A4001A51F8
S31508002E2010BD0000080001400021016001710C215D
S31508002E30417100218171704710B504460848006940
S31508002E400221084306490861084644610069402191
S31508002E50084303490861034800F00EF910BD000055
S31508002E6000200240FF0F00000C48C068C007C00FD2
S31508002E70002801D0012070470848C068042108408E
S31508002E80002801D00220F6E70448C068102108404F
S31508002E90002801D00320EEE70420ECE700200240DA
S31508002EA0034800698021084301490861704700000A
S31508002EB00020024030B504460D4605480069012148
S31508002EC008430349086125800F2000F0D5F830BD76
S31508002ED00020024010B57E2002F01AFC064800F0D9
S31508002EE00FF87E2002F014FC044800F009F87E2052
S31508002EF002F00EFC10BD000000F4000800F0000807
S31508002F0010B5044600F0ACF82046FFF795FFFFF72A
S31508002F10C7FF10BD70B503460125002208E0500022
S31508002F201C5A0748844201D0002506E0501C82B28C
S31508002F30CE0F761876109642F1DC00BF284670BD93
S31508002F40FFFF0000F8B505460E46144600F088F85F
S31508002F507E2002F0DDFB002707E029883046FFF7D0
S31508002F60A9FFB61CAD1C781C87B2E10F09194910D8
S31508002F70B942F2DCFFF794FFF8BDF8B507460C46F0
S31508002F8015462946204600F037F80646002E0DD18C
S31508002F902046FFF7B5FF012080022018FFF7B0FF93
S31508002FA02A4621463846FFF7CDFF24E00120800255
S31508002FB02018401BB0420AD1012080022018FFF7D2
S31508002FC09FFF2A4631463846FFF7BCFF13E001202B
S31508002FD0C0022018401BB04208D12046FFF790FFD8
S31508002FE02A4631463846FFF7ADFF04E02A46314601
S31508002FF03846FFF7A7FFF8BDF8B505460E462F4633
S31508003000E807C00F002801D000BFFEE731460120BF
S31508003010C002FEF797FC002901D000BFFEE7002496
S315080030200BE020467043471931463846FFF772FFD2
S31508003030012800D108E0601C84B231460120C00294
S31508003040FEF780FCA042ECDC00BF31460120C0023E
S31508003050FEF778FCA04200D100273846F8BD0000EC
S31508003060024803494860034848607047230167459A
S3150800307000200240AB89EFCD10B5024600BFFFF72E
S31508003080F3FE0346521EFF2400E0641E002CFCD10A
S31508003090012B01D1002AF2D106480069772188431D
S315080030A0044908613420C860002A01D1052010BDF2
S315080030B01846FCE7002002401FB50121880400F0ED
S315080030C0DBFC0121480400F0D7FC01A800F003FA54
S315080030D001216846818081710421C17101A95E4878
S315080030E000F082F901A800F0F6F90221684681800D
S315080030F0012181711021C17101A9574800F074F9A5
S3150800310001A800F0E8F9042168468180012181714F
S315080031100421C17101A9504800F066F901A800F020
S31508003120DAF9202168468180012181710421C17163
S3150800313001A9494800F058F901A800F0CCF908217E
S3150800314068468180012181710421C17101A9092084
S31508003150C00600F049F901A800F0BDF901214902AD
S3150800316068468180012181712821C17101A9092040
S31508003170C00600F039F901A800F0ADF9FF210131C8
S3150800318068468180012181711021C17101A9092038
S31508003190C00600F029F901A800F09DF9402168460B
S315080031A08180012181711021C17101A92A4800F08D
S315080031B01BF900210120FFF719FE05210120FFF761
S315080031C015FE03210020FFF711FE02A8FFF72CFECB
S315080031D001200290002168460173102141730121E4
S315080031E0817302A8FFF7A2FD02A8FFF71DFE2020A3
S315080031F002900021684601730821417301218173F9
S3150800320002A8FFF793FD02A8FFF70EFE082002901A
S31508003210002168460173102141730121817302A8B8
S31508003220FFF784FD05216846017001214170817010
S3150800323000F064FA06216846017001214170817028
S3150800324000F05CFA0721684601700121417081701F
S3150800325000F054FA1FBD00000004004810B502F043
S3150800326031F904463A480068002803D0042C01DBEB
S31508003270201FC4B2374844800121374800F015F9A9
S31508003280002825D13548364908800221324800F001
S3150800329015F9002806D002212F4800F018F90A204F
S315080032A03049087004212C4800F0FFF800280BD09C
S315080032B02C480078002807D1264840880F2803DACA
S315080032C00220294908700EE00120274908700AE003
S315080032D023480088002803DD01202349087002E0FE
S315080032E000202149087008210920C00600F0DDF8F1
S315080032F0002829D019481A4908801B48007802284E
S3150800330011D1002019490870FF2101310920C00692
S3150800331000F0D4F800281AD1FF2101310920C0068F
S3150800332000F0D7F813E001201049087001020920BF
S31508003330C00600F0C3F8002809D0FF210131092092
S31508003340C00600F0C4F802E000200849087010BD65
S31508003350DC000020880300200004004888130000D1
S31508003360D4000020D700002013010020CD00002043
S3150800337008B50121480400F07FFB0121880400F00C
S315080033807BFB0121C80400F077FB0121080500F04A
S3150800339073FB684600F09FF80F49684601800021D4
S315080033A0C17069460920C00600F01EF8684600F09C
S315080033B092F80021C943684601800021C170694618
S315080033C0064800F011F86946054800F00DF8694608
S315080033D0044800F009F808BDFF9F000000080048EF
S315080033E000040048000C0048F8B50246CD782F07BF
S315080033F03F0FCD7810263540002D01D08D782F430C
S315080034001446002011E085062B0E0D8801268640FD
S315080034103540002D07D025680F269E40B5433E4609
S315080034209E4035432560451CE8B20828EBDB141D91
S315080034300D882D120095002011E085062B0E01251A
S315080034408540009E3540002D07D025680F269E40F2
S31508003450B5433E469E4035432560451CE8B20828DC
S31508003460EBDBCD78282D04D155690E883543556197
S3150800347006E0CD78482D03D115690E8835431561C8
S31508003480F8BD70B54D07EB0E082902DA054620355A
S3150800349001E0054624352C460F269E402568B5438F
S315080034A016469E403543256070BD02469068084022
S315080034B0002801D0012070470020FCE70246D068AA
S315080034C00840002801D0012070470020FCE7416130
S315080034D07047016170470021C9430180022181704C
S315080034E00421C17070470000F0B593B0002601258D
S315080034F01CE069005C4A505AFEF7CFFC0746FEF707
S31508003500E7FC0022594B0D910C90FEF743FC002274
S31508003510574B0F910E90FEF7D5FB11911090FEF7C1
S3150800352013FDA900534A5050681C85B2042DE0DBF0
S3150800353050498868504901F083FE504908600024C4
S315080035401BE0A1004E4A5058FEF7C2FC119110909C
S3150800355048494868FEF7BCFC00224A4B0D910C907E
S31508003560FEF7B0FB0F910E90119B109AFEF7C4FC64
S3150800357001D2264603E0601C84B2332CE1DB00BF8F
S31508003580701EFEF77FFC40490B90FEF76CFA074663
S31508003590FEF79EFC721E9200394B0F910E909958B9
S315080035A0B2009858FEF757FA0746FEF791FC0991BC
S315080035B00890711E8900324A5058FEF789FC059119
S315080035C004902C494868FEF783FC00222D4B019194
S315080035D00090FEF777FB03910290059B049AFEF78D
S315080035E062FB07910690099B089AFEF7D3FB002217
S315080035F0244B0B910A90FEF765FB0D910C900F9BDF
S315080036000E9AFEF7ABFA11911090FEF79DFC1F4932
S3150800361008601849C8681849FEF762FA07461C493F
S31508003620FEF721FA1B490860144801681748006824
S31508003630FEF7C0F91849086008460068FEF748FC16
S3150800364002460B461191109014A002F087F8114813
S315080036500068FEF73DFC02460B461191109014A037
S3150800366002F07CF813B0F0BD1202002000FEAF4055
S3150800367000000840F016002000004040200200200C
S31508003680ACDE000800002440000020411C02002097
S315080036900000A040280200202402002074656D70F6
S315080036A05F616C6C203D20252E326620200A0000C2
S315080036B04241545F56203D20252E3266200A0000DE
S315080036C001480068704700004C0100200348006864
S315080036D00349097840180149086070474C010020E1
S315080036E05401002010B501F04FFCFF216831024853
S315080036F001F06EFC10BD0000E70300008178002988
S3150800370025D01749032212028918027892109200CE
S31508003710895802789207D30EFF229A40914342783D
S315080037209207120E03789B07DB0E9A4011430C4A48
S3150800373003231B02D21803789B109B00D1500178F3
S31508003740CA06D20E01219140054A116007E00178A8
S31508003750CA06D20E01219140014A80321160704793
S3150800376000E100E00EB500210120FFF73FFB012034
S31508003770019000216846017210214172012181726F
S3150800378001A8FFF7D3FA03210020FFF72FFB082033
S31508003790019000216846017210214172012181724F
S315080037A001A8FFF7C3FA05210120FFF71FFB202018
S315080037B0019000216846017210214172012181722F
S315080037C001A8FFF7B3FA0521684601700121417087
S315080037D08170FFF793FF0621684601700121417049
S315080037E08170FFF78BFF0721684601700121417040
S315080037F08170FFF783FF0EBD0D4A1268920892008A
S3150800380002430B4B1A600B4A126904231A43094BED
S315080038101A61012901D130BF02E040BF20BF20BF95
S31508003820044A126904239A43024B1A61704700003E
S315080038300070004000ED00E008B502214448FFF79B
S3150800384046FE40214348FFF742FE02214148FFF762
S3150800385040FEFF2101310920C006FFF738FE01218D
S3150800386009030920C006FFF732FEFFF781FDFFF7BF
S3150800387023FC0121480400F0FFF80121880400F028
S31508003880FBF80121080500F0F7F86846FFF723FE64
S315080038900121C90268460180032181701021C17087
S315080038A069460920C006FFF79FFD6846FFF713FE25
S315080038B0022168460180032181701021C170694682
S315080038C00920C006FFF790FD6846FFF704FE0121B0
S315080038D0090368460180032181701021C170694679
S315080038E00920C006FFF780FD6846FFF7F4FD0421AE
S315080038F0684601801021C17003218170694609203C
S31508003900C006FFF771FD04210920C006FFF7DFFD99
S315080039100121C9020920C006FFF7D9FD02210C487A
S31508003920FFF7D5FD40210B48FFF7D1FD02210948D5
S31508003930FFF7CFFDFF2101310920C006FFF7C7FDBC
S31508003940012109030920C006FFF7C1FD08BD0000D3
S31508003950000C00480004004810B527A001F0FEFE40
S315080039600020FEF7A1FE00212748FEF74DFD0021A5
S315080039702648FFF7AFF8002124481430FFF7AAF8C5
S31508003980002122482830FFF7A5F800211F483C30BF
S31508003990FFF7A0F800211E4800F090FD00211D4801
S315080039A000F08CFD00210120800701F087FB002133
S315080039B0194801F014FD0121480200F07DF80021A4
S315080039C0012000F059F800210120800300F074F866
S315080039D000210120000300F06FF800210120800378
S315080039E000F05AF80021012000F056F8FFF724FFEE
S315080039F0FFF7B8FE10BD00006C6F77706F776572C1
S31508003A0020696E20210A0000002401401C000240A3
S31508003A1000300140003800400038014010B501F080
S31508003A207DFAE1204002FEF751FF01F071FC00210A
S31508003A300D48C171FFF740FB00F0DCF800F004FC0C
S31508003A4000F0D0F900F002FA00F0D2FEFFF74AFEC5
S31508003A50FEF7E6FC01210548FEF7FEFD0448054988
S31508003A600880FFF7FBFB10BD780200200024014008
S31508003A7088130000D4000020002905D0054A5269A1
S31508003A800243044B5A6104E0024A52698243014BDD
S31508003A905A61704700100240002905D0054AD269CC
S31508003AA00243044BDA6104E0024AD2698243014BBD
S31508003AB0DA61704700100240002905D0054A92696C
S31508003AC00243044B9A6104E0024A92698243014B1D
S31508003AD09A6170470010024010B500F031F80449A9
S31508003AE04968F02211400909024A515CC84010BDD4
S31508003AF0001002401701002010B5FFF7EDFF054939
S31508003B004968072212021140090A034A515CC84053
S31508003B1010BD0000001002401701002010B5FFF785
S31508003B20DBFF054949680722D2021140C90A034A40
S31508003B30515CC84010BD000000100240170100206B
S31508003B40F8B51E4840680C210840042802D0082809
S31508003B502ED101E01A4C2DE0184840300069C00704
S31508003B60C00F00280AD015484030006902210840D5
S31508003B70002801D0134802E0114800E01048074623
S31508003B800E4840300069FF2109040840000C451C16
S31508003B900A4840300069072109020840000A461C05
S31508003BA03946694308463146FDF7B6FE044601E044
S31508003BB0034C00BF00BF2046F8BD000000100240BD
S31508003BC000127A0000093D0070B50446002502215E
S31508003BD0074801F00AFC002808D0054801F05EFCF9
S31508003BE020700221024801F0F8FB0125284670BD25
S31508003BF00038014000B585B001210803FFF75CFFD6
S31508003C00684600F0BBFC042168460170002141802B
S31508003C100821017100214171012181710021018171
S31508003C2002214181002101736946324800F060FC97
S31508003C300021304800F016FC01212E4800F012FC45
S31508003C4001212C4803F0F0F82A48C06920210843CE
S31508003C502849C86101214804FFF70EFF0022042104
S31508003C600920C006FFF70DFC002205210920C00621
S31508003C70FFF707FC002206210920C006FFF701FC12
S31508003C80002207210920C006FFF7FBFB04A8FFF75F
S31508003C9022FC102168460182012181741821C17411
S31508003CA004A90920C006FFF79FFB04A8FFF713FC29
S31508003CB0A02168460182012181741821C17404A9D2
S31508003CC00920C006FFF790FB04A8FFF704FC402173
S31508003CD068460182012181744821C17404A909201A
S31508003CE0C006FFF781FB0121024800F0E7FB05B09B
S31508003CF000BD00000030014038B505460EA000683A
S31508003D0000902C042002010E684641702004010E22
S31508003D1068468170C47000F05DF90121074800F01B
S31508003D20C1FB0421684600F0CFF80021034800F0E3
S31508003D30B9FB00F0D3F838BDD800000000300140C8
S31508003D407CB504460D4616460EA103C9019100909E
S31508003D502002010E684641702004010E68468170F3
S31508003D60C4700121094800F09DFB0521684600F052
S31508003D70ABF8B1B2284600F09DF80021034800F0E0
S31508003D8091FB7CBD0B000000FF00000000300140E5
S31508003D90F8B504460D46164610A0006800902002A5
S31508003DA0010E684641702004010E68468170C47091
S31508003DB000F010F901210A4800F074FB0421684656
S31508003DC000F082F8B1B2284600F07EF800210448D7
S31508003DD000F068FB00F082F8F8BD00000200000061
S31508003DE0003001401CB50FA0006801900024012195
S31508003DF00D4800F057FB042101A800F065F80221E0
S31508003E00684600F057F80021074800F04BFB684663
S31508003E100478240240780443214604A001F09EFC5D
S31508003E201CBD000090000000003001400D0A5350F0
S31508003E304920466C61736820446576696365494420
S31508003E40203A203078253034780000001CB59F21B0
S31508003E500191002401210E4800F024FB012101A84C
S31508003E6000F032F80321684600F024F800210848DB
S31508003E7000F018FB684604782402407804432402BC
S31508003E80684680780443214602A001F067FC1CBD01
S31508003E90003001400D0A53504920466C6173682072
S31508003EA04A45444543204944203A2030782530364F
S31508003EB07800000070B505460C46002C03D0214654
S31508003EC0284600F099F870BD70B505460C46002CDA
S31508003ED003D02146284600F023F970BD1CB5002002
S31508003EE0019011A000680090002400BF01210F482E
S31508003EF000F0D8FA02216846FFF7E6FF012101A87B
S31508003F00FFF7D8FF0021094800F0CCFA2046641CC8
S31508003F100749884200D905E068460079C007C00FFE
S31508003F200028E3D100BF1CBD05FF0000003001409A
S31508003F30FFFF0000F7B5C0B00C464098FFF7DCFE5F
S31508003F40002616E0002507E0300241194298405C39
S31508003F5069464855681C85B2FF2DF5DD4099090468
S31508003F6032028818FF2201326946FFF711FF701CDA
S31508003F7086B2E117090E09190912B142E2DC204698
S31508003F80E117090E091809120902611A20D000253D
S31508003F9007E0300241194298405C69464855681C5A
S31508003FA085B22046E117090E091809120902611A95
S31508003FB0A942EEDC2746409909043302C818E117DE
S31508003FC0090EC91909120902621A6946FFF7E0FEC5
S31508003FD043B0F0BD08B5062000900121054800F061
S31508003FE061FA01216846FFF76FFF0021014800F0DA
S31508003FF059FA08BD0030014030B58BB005460C466D
S315080040000021019101210846FFF736FD4048FEF7D9
S3150800401067FD3F481430FEF763FD03A8FEF7B8FDB9
S315080040203C4803900495002168460175069401777B
S31508004030802141770021C183018408A8817003216A
S315080040400903684681840021C184018503A9304893
S31508004050FEF778FD2020FEF731FD012202212C48CB
S31508004060FEF766FD03A8FEF793FD2A48001F039096
S3150800407001A804901021684601750694002101776D
S315080040804177C183018408A8817003210903684622
S3150800409081840021C184018503A91D481430FEF7D7
S315080040A051FD0A216846017201214172817202A8F6
S315080040B0FFF724FB01211648FEF70CFD01211448E1
S315080040C01430FEF707FD00201349086013490860FD
S315080040D001211048001F00F0FDF900BF0E480068D6
S315080040E00028FBD000BF0D4800680028FBD000213F
S315080040F00848001F00F0EEF900210548FEF7EAFC23
S31508004100002103481430FEF7E5FC0BB030BD000073
S315080041101C00024004300140DC010020E0010020C0
S3150800412030B58BB005460C460021019101210846A1
S31508004130FFF7A2FC4048FEF7D3FC3F481430FEF7D1
S31508004140CFFC03A8FEF724FD3C48039001A8049081
S31508004150002168460175069401774177C183018479
S3150800416008A8817003210903684681840021C18457
S31508004170018503A93048FEF7E5FC2020FEF79EFCE2
S31508004180012202212C48FEF7D3FC03A8FEF700FD06
S315080041902A48001F03900495102168460175069465
S315080041A000210177802141770021C183018408A875
S315080041B0817003210903684681840021C184018531
S315080041C003A91D481430FEF7BDFC0A216846017292
S315080041D001214172817202A8FFF790FA012116485F
S315080041E0FEF778FC012114481430FEF773FC002012
S315080041F0134908601349086001211048001F00F0A0
S3150800420069F900BF0E4800680028FBD000BF0D48BA
S3150800421000680028FBD000210848001F00F05AF962
S3150800422000210548FEF756FC002103481430FEF726
S3150800423051FC0BB030BD00001C00024004300140A8
S31508004240DC010020E001002000B585B001218803CB
S31508004250FFF722FC684600F091F9042168460170D0
S3150800426000214180082101710021417101218171DC
S3150800427000210181042141810021017369462248F8
S3150800428000F036F90021204800F0ECF801211E481C
S3150800429000F0E8F801214804FFF7EEFB0121880445
S315080042A0FFF7EAFB07220A210920C006FFF7E9F80B
S315080042B004220B210920C006FFF7E3F804A8FFF73C
S315080042C00AF90321890268460182012181741821AD
S315080042D0C17404A90920C006FFF786F804A8FFF7E9
S315080042E0FAF8FF2101316846018201218174102103
S315080042F0C17404A90548FFF777F80121024800F0C0
S31508004300DDF805B000BD0000003800400004004894
S3150800431030B58BB005460C460021019101210846AF
S31508004320FFF7AAFB4048FEF7DBFB3F481430FEF7D1
S31508004330D7FB03A8FEF72CFC3C48039001A8049081
S31508004340002168460175069401774177C183018487
S3150800435008A8817003210903684681840021C18465
S31508004360018503A93048FEF7EDFB01204003FEF75F
S31508004370A5FB012202212C48FEF7DAFB03A8FEF76B
S3150800438007FC2A48001F039004951021684601750A
S31508004390069400210177802141770021C183018499
S315080043A008A8817003210903684681840021C18415
S315080043B0018503A91C481430FEF7C4FB0B21684687
S315080043C0017201214172817202A8FFF797F9012152
S315080043D01548FEF77FFB012113481430FEF77AFBD8
S315080043E00020134908601349086001210F48001F7F
S315080043F000F070F800BF0E4800680028FBD000BF28
S315080044000C4800680028FBD000210848001F00F06F
S3150800441061F800210448FEF75DFB002102481430CC
S31508004420FEF758FB0BB030BD44000240043800408C
S31508004430E4010020E801002070B505460C46002C72
S315080044400DD0FF2101310648FFF741F821462846DD
S31508004450FFF75EFFFF2101310148FFF73AF870BD0B
S3150800446000040048002906D0012909D002290CD0E9
S31508004470032914D10EE0826910231A4382610FE0E2
S31508004480826908231A4382610AE0826910239A43E3
S31508004490826105E0826908239A43826100E000BFD1
S315080044A000BF7047002904D0826A120A120282628B
S315080044B003E0826AFF231A4382627047002904D008
S315080044C0826901231A43826103E082695208520015
S315080044D082617047002905D0826901235B021A436D
S315080044E0826104E0826901235B029A438261704714
S315080044F04A880123DB029A4203D182691A43826100
S3150800450004E082690123DB029A43826182690123FE
S315080045109B029A430B891A438261826904239A4350
S315080045200B781A438261C26904239A430B7B1A43A8
S31508004530C261C26902239A434B791A43C261C269AE
S31508004540520852008B791A43C261C26908231A437A
S31508004550C261026A120C12044B891A4302620A7972
S31508004560202A04DBC26A52095201C26205E0C26A05
S31508004570520952010B791A43C26270470021017031
S3150800458041800821017100214171012181710021B9
S31508004590018102214181002101737047FFB585B071
S315080045A006460F460E9C2046E117090D0918091301
S315080045B00903611A89B20391E117090D091809015E
S315080045C0090C04910020029008983818401EC3B2BE
S315080045D007983018401EC2B2F9B2F0B2019000F046
S315080045E081FA2C2000F0AEFA00250FE00F99090495
S315080045F02A038818012212030E49FFF7A1FB01219D
S3150800460009030C4800F0AAFA681C85B2049885428A
S31508004610ECDB039800280BD00F9909042A038818A5
S315080046200449039AFFF78CFB0248039900F096FAAF
S3150800463009B0F0BD4E060020FFB583B00746154603
S31508004640680028180290029803F084F8064600BF0E
S31508004650002414E00C980002000E610061187054E2
S315080046600C980004010E60002018401C31540C9868
S31508004670C1B260002018801C3154601C84B2AC4260
S31508004680E8DB069904984018401EC3B27819401E04
S31508004690C2B20498C0B20190F8B20090019900F035
S315080046A021FA2C2000F04EFA002407E068002818AA
S315080046B081B2304600F052FA601C84B206988442F1
S315080046C0F4DB304602F062FC07B0F0BD70B5044674
S315080046D00D462E1DF3B2E2B2E9B2E0B200F002FADC
S315080046E02C2000F02FFA0F21014800F037FA70BD90
S315080046F0BD01002038B50446A023522200210846F1
S315080047000094FFF799FF38BDFFB585B007460F9DA2
S315080047102846E917090D091809130903691A89B200
S315080047200391E917090D09180901090C049108995B
S3150800473006984018401EC3B207983818401EC2B2E1
S315080047400698C0B20290F8B20190029900F0CAF930
S315080047502C2000F0F7F9002620E0002414E03103AD
S315080047600A190E99885CFDF798FB0190109880004D
S315080047701D4A11580198FDF776F90290FDF794FB4A
S315080047801A490855601C84B2012000038442E6DBFE
S315080047900146164800F0E2F9701C86B20498864273
S315080047A0DBDB039800281DD0002414E031030A1926
S315080047B00E99885CFDF771FB0190109880000A4AF3
S315080047C011580198FDF74FF90290FDF76DFB07495F
S315080047D00855601C84B203988442E7DB03480399B2
S315080047E000F0BCF909B0F0BD940100204E06002087
S315080047F008B501214804FFF73FF901218804FFF7AE
S315080048003BF901210805FFF737F96846FEF763FE0D
S31508004810022168460180012181701021C170694614
S31508004820A448FEF7E1FD6846FEF755FE0121C903D7
S3150800483068460180012181701021C17069460920EE
S31508004840C006FEF7D1FD6846FEF745FE012168461B
S31508004850018081701021C17069469648FEF7C4FD33
S315080048606846FEF738FE01210903684601800321E0
S3150800487081701021C17069460920C006FEF7B4FD93
S3150800488002218C48FEF725FE0121C9030920C0062E
S31508004890FEF71FFE01218748FEF71BFE00F00CF904
S315080048A0112000F04FF9212000F04CF9B12000F05A
S315080048B049F9012000F03AF92C2000F037F92D20AB
S315080048C000F034F9B22000F03DF9012000F02EF98D
S315080048D02C2000F02BF92D2000F028F9B32000F049
S315080048E031F9012000F022F92C2000F01FF92D20C3
S315080048F000F01CF9012000F019F92C2000F016F937
S315080049002D2000F013F9B42000F01CF9032000F064
S315080049100DF9C02000F016F9622000F007F9022010
S3150800492000F004F9042000F001F9C12000F00AF9AA
S31508004930C02000F0FBF8C22000F004F90D2000F0BA
S31508004940F5F8002000F0F2F8C32000F0FBF88D20FF
S3150800495000F0ECF86A2000F0E9F8C42000F0F2F85C
S315080049608D2000F0E3F8EE2000F0E0F8C52000F016
S31508004970E9F80E2000F0DAF82A2000F0E3F8002023
S3150800498000F0D4F8002000F0D1F8002000F0CEF8AE
S31508004990832000F0CBF82B2000F0D4F8002000F09C
S315080049A0C5F8002000F0C2F8002000F0BFF8A120EA
S315080049B000F0BCF8E02000F0C5F8102000F0B6F8CA
S315080049C00E2000F0B3F8022000F0B0F8032000F043
S315080049D0ADF80E2000F0AAF8072000F0A7F802208C
S315080049E000F0A4F8072000F0A1F80A2000F09EF8CD
S315080049F0122000F09BF8272000F098F8372000F0E6
S31508004A0095F8002000F092F80D2000F08FF80E209F
S31508004A1000F08CF8102000F089F8E12000F092F8F8
S31508004A20102000F083F80E2000F080F8032000F034
S31508004A307DF8032000F07AF80F2000F077F80620BA
S31508004A4000F074F8022000F071F8082000F06EF803
S31508004A500A2000F06BF8132000F068F8262000F012
S31508004A6065F8362000F062F8002000F05FF80D20A7
S31508004A7000F05CF80E2000F059F8102000F056F807
S31508004A803A2000F05FF8062000F050F8362000F0D3
S31508004A9059F8C82000F04AF8292000F053F86C208D
S31508004AA0FFF728FE012109030920C006FEF711FDBC
S31508004AB008BD0000000C004810B50120FDF778FF7E
S31508004AC001210748FEF703FD0120FDF771FF0121CB
S31508004AD00348FEF7FEFC7820FDF76AFF10BD0000CC
S31508004AE0000C0048F8B504460D4616461F462046F3
S31508004AF01830C4B2681CC5B230461830C6B2781C25
S31508004B00C7B22A2000F01EF80020009068464470BC
S31508004B10C670042100F022F82B2000F013F868462E
S31508004B204570C770042100F019F8F8BD01B50121D8
S31508004B30C9030920C006FEF7CCFC01216846FFF729
S31508004B407BFC08BD01B50121C9030920C006FEF793
S31508004B50BEFC01216846FFF76FFC08BD70B5044628
S31508004B600D460121C9030920C006FEF7B2FC2946F5
S31508004B702046FFF761FC70BD10B500F001F810BDC6
S31508004B8000B585B06248006801210843604908609D
S31508004B9000BF5F480068022108400028F9D05D4838
S31508004BA05D4908605D480068102108435B49086054
S31508004BB008460068C008C000086057490968481ECA
S31508004BC05749FCF7A9FE0490544800680499490718
S31508004BD0490F0843514908604D4840685149084003
S31508004BE04B49486008464068902108434849486050
S31508004BF0084640684860484800684649884207D9D8
S31508004C0043484068052109020843414948600BE0CA
S31508004C10414800684449884206D93D484068012110
S31508004C20890208433A4948606B4601AA3A4801682E
S31508004C303E48FDF751FD364840300069800880003F
S31508004C403349403108610846006940084000086158
S31508004C50684600784007400F02906846007940068B
S31508004C60400E03902A48C069890508432849C86147
S31508004C702748403000692E490840254940310861D7
S31508004C800398000402990902084321494031096939
S31508004C9008431F49403108611D480068012109067B
S31508004CA008431B49086000E000BF19480068012155
S31508004CB0490608400028F7D0154840688008800053
S31508004CC0134948600846406802210843104948606D
S31508004CD000E000BF0E4840680C2108400828F8D1BB
S31508004CE00120FDF771FE0A484068102188430849EB
S31508004CF048600120FDF768FE054840688021884322
S31508004D00034948600120FDF75FFE05B000BD0000BD
S31508004D100010024000A24A04280100200020024098
S31508004D2000366E010FC0FFFF0051250200127A00FF
S31508004D30FFF800FF042806D1064909690422114331
S31508004D40044A116105E00349096904229143014AAD
S31508004D501161704700E000E010B5FEF7B7FC614846
S31508004D60C068401C5F49C8605F480068002804D0D6
S31508004D705D480068401E5C4908605A483830007A29
S31508004D8001280ED157484069401C564948610846D3
S31508004D9040695649884207D900215248383001727D
S31508004DA002E000204F4948614E483830807A012891
S31508004DB005D14C48C06A401C4A49C86202E0002036
S31508004DC04849C8624A480068002804D0484800682C
S31508004DD0401E4749086043483830C07A012812D136
S31508004DE040214448FEF775FB3E4881688068401CB0
S31508004DF03C4A9060FF20F530814223D900211046B5
S31508004E003830C1721EE037483830C07A022812D1CD
S31508004E1040213848FEF75DFB324881688068401CAF
S31508004E20304A90607D20C00081420BD9002110468F
S31508004E303830C17206E000202A49886040212D4892
S31508004E40FEF745FB2C480088002804DD2A48008820
S31508004E50401E2949088029480078012808D1284891
S31508004E600068002804D026480068401E24490860C7
S31508004E70244800680F21C943884204D221480068A3
S31508004E80401C2049086020480078002804DD1E4898
S31508004E900078401E1C4908701C480078002804DD6C
S31508004EA01A480078401E19490870194800681949B7
S31508004EB088420CD211480078012803D00F480078A0
S31508004EC0022804D112480068401C1149086012489B
S31508004ED00068002804D010480068401E0E49086083
S31508004EE010BD000040020020480100208813000081
S31508004EF0F001002000040048D4000020160100201C
S31508004F00EC010020D0000020D7000020D8000020A7
S31508004F10F4010020C0270900DC00002010B516485F
S31508004F200068012108431449086008464068134987
S31508004F3008401149486008460068114908400E496A
S31508004F400860084600680121890488430A49086000
S31508004F5008464068C321090488430749486008464B
S31508004F60006808490840044908609F2000048860D2
S31508004F70FFF702FE10BD0000001002400CC0FFF84B
S31508004F80FFFFF6FEFFFF8F0008B501214804FEF774
S31508004F9073FD022211460920C006FEF772FA0421A3
S31508004FA0684601801821C17001218170694609206F
S31508004FB0C006FEF719FA08BD10B50821C80600F0A4
S31508004FC0A0F8002803D00821C80600F073F810BD21
S31508004FD030B589B004460D4601210846FEF75CFD4A
S31508004FE006A800F023F90794684605830021018482
S31508004FF008A881706846817606A90120800700F016
S31508005000DFF80F2168460171022141710121817182
S3150800501001A8FEF773FB0821C80600F047F801222D
S315080050200821C80600F07AF802A800F0B5F8602151
S3150800503068460172012141720020039000216846EA
S31508005040017402A90120800700F072F80821C80639
S3150800505000F09CF84021080600F04AF8012188076C
S3150800506000F018F80121880700F034F801218807B4
S3150800507000F024F809B030BD10B50121044800F04D
S3150800508040F8002803D00121014800F013F810BDAC
S3150800509000040040002904D0026880231A430260F5
S315080050A003E0026880239A430260704702698A43D4
S315080050B00261704702698A4302617047002904D079
S315080050C0026801231A43026003E00268520852008C
S315080050D002607047002905D0426C0123DB031A439E
S315080050E0426404E0426C0123DB039A43426470473E
S315080050F0C26970239A430A43C26170470146C86B66
S315080051007047024610690840002805D0D068084054
S31508005110002801D0012070470020FCE7002A03D0B0
S31508005120C3680B43C36002E0C3688B43C360704720
S3150800513010B5C26970239A430B781A43C2610A7A7A
S3150800514012024B781B021A43036A03242402A34360
S315080051501A4302624A68C2630B4A904213D14A7ADA
S3150800516012028B781B021A43036AA400A3431A434C
S3150800517002624A8912018B891B011A434368A400FB
S31508005180A3431A43426010BD002C0140C26908239C
S315080051909A430A43C26170470021017041708170C9
S315080051A041600172417241818181704701229207F3
S315080051B0904201D1C16301E08AB2C2637047000020
S315080051C0026803231B029A430B891A430260134A97
S315080051D0904206D001229207904202D0104A90428D
S315080051E005D1026870239A438B781A4302600B4AEA
S315080051F0904205D00B4A904202D00B4A904205D104
S31508005200026B120A12028B7A1A4302634A68C26256
S315080052100A8882620122426170470000002C014020
S315080052200004004000440140004801400021C943F1
S315080052304160002101800181817081727047000000
S31508005240F3B597B00020159014902A4813902A4871
S3150800525012902A4811902A48109018991798FCF726
S31508005260FEFB05462349FCF73BFC044621461798F6
S31508005270FCF736FC14901098FCF72AFE0D910C905A
S315080052801198FCF725FE0391029013991498FCF7E0
S3150800529027FC0190FCF71CFE044602F01DF80646A2
S315080052A0039B029AFCF776FD079106907F20C005BE
S315080052B01299FCF715FC0446FCF70AFE05910490C2
S315080052C0079B069AFCF74AFC02460B46099108908A
S315080052D000200C49FCF75EFD0B910A900D9B0C9A79
S315080052E0FCF7E1FC0F910E90FCF72EFE1590159831
S315080052F019B0F0BD0050C3473313954300D0844519
S31508005300339388430000F03F10B5FEF7D9F910BD76
S3150800531070B5FEF7E1FB05467D21C900FCF7FCFAEE
S315080053200446601E0C49884200D90CE0601E0B49F1
S3150800533048610321081F00F047FA002007498861E1
S315080053400720086100BF0420FFF7F4FC0021481E6F
S3150800535000F03AFA70BD0000FFFFFF0000E000E031
S3150800536010B502210A4800F049F800280ED008486E
S3150800537000F094F8C4B20748407A002802D12046C3
S3150800538001F02EFE0221024800F027F810BD0000A9
S31508005390003801407802002010B504462146054829
S315080053A000F080F800BF0121024800F01EF800282E
S315080053B0F9D010BD0038014070B504460D467E2070
S315080053C000F0A6F903E02078641CFFF7E5FF2846FD
S315080053D0691E8DB20028F6D170BD41617047826999
S315080053E0520852000A438261704702469068084094
S315080053F0002801D0012070470020FCE70246D0684B
S315080054000840002801D0012070470020FCE7002A48
S3150800541003D003690B43036102E003698B4303610D
S315080054207047000070B504460D460026E069302135
S31508005430884329790843E061E06944218843A979CA
S315080054400843E061E06980088000297A0843E06142
S31508005450A0691821884369890843A061A0690421C5
S315080054608843297B0843A0610B48844203D1FEF791
S3150800547055FB064602E0FEF73FFB0646304629681E
S31508005480FCF74AFA0009206230462968FCF744FA14
S315080054900007000F606270BD003801400146486889
S315080054A0C0B27047CAB2026070474B21C901016099
S315080054B03021017100218171017218214181002179
S315080054C00173704770B56F480068FCF701FD044624
S315080054D06D4A6E4BFCF724FD03D800206C49087012
S315080054E0CCE068480068FCF7F3FC0446694A6A4B56
S315080054F0FCF716FD03D8012065490870BEE061482F
S315080055000068FCF7E5FC0446624A5242634BFCF726
S3150800551007FD03D802205E490870AFE059480068C5
S31508005520FCF7D6FC0446584A52425D4BFCF7F8FC99
S3150800553003D8032056490870A0E052480068FCF7D3
S31508005540C7FC04460022574BFCF7EAFC03D80420A4
S315080055504F49087092E04B480068FCF7B9FC0446CE
S315080055604C4A514BFCF7DCFC03D805204849087027
S3150800557084E044480068FCF7ABFC0446424A5242C1
S315080055804A4BFCF7CDFC03D806204149087075E064
S315080055903C480068FCF79CFC04463B4A444BFCF735
S315080055A0BFFC03D807203A49087067E03548006809
S315080055B0FCF78EFC0446374A52423E4BFCF7B0FCD9
S315080055C003D808203249087058E02E480068FCF7CE
S315080055D07FFC04460022384BFCF7A2FC03D80920BE
S315080055E02B4908704AE027480068FCF771FC044616
S315080055F0284A324BFCF794FC03D80A202449087041
S315080056003CE020480068FCF763FC04461E4A524208
S315080056102B4BFCF785FC03D80B201D4908702DE0A1
S3150800562018480068FCF754FC0446174A254BFCF753
S3150800563077FC03D80C20164908701FE0114800684B
S31508005640FCF746FC0446134A52421F4BFCF768FC1B
S3150800565003D80D200E49087010E00A480068FCF7C8
S3150800566037FC04460022194BFCF75AFC03D80E20D7
S315080056700749087002E00F200549087004480078B9
S3150800568070BD000028020020CDCCCCCCCCCC10407C
S31508005690D60000209A999999999910406666104003
S315080056A0333310400000104099990F4033330F40B0
S315080056B0CCCC0E4066660E4000000E4099990D400F
S315080056C033330D40CCCC0C4066660C4000000C40D1
S315080056D00348806840084000014988607047000018
S315080056E0002C004003488068002801D0012070473C
S315080056F00020FCE7002C004010B5FFF7F3FF002858
S3150800570004D0FFF7E5FF662000F002F810BD0000A0
S315080057104106490E014A116070470000002C0040FE
S3150800572010B57E20FFF7F4FF0948FDF7E9FB0949A4
S31508005730094801810621083000F0EAFD06490831CA
S3150800574088814022024904480830FDF716FC10BD3E
S3150800575000F80008FBAA0000800300200FB410B56B
S3150800576003A9044B044A029800F0A6F910BC08BC29
S3150800577004B01847696F0008300200202021020C87
S3150800578001D010211046020A01D010460839020934
S3150800579001D01046091F820801D01046891E42080A
S315080057A001D0881E7047081A704730B47446641EC4
S315080057B02578641CAB4204D3635D5B00E31830BCF8
S315080057C018471D46F8E7000010B5002819DB1A4AE5
S315080057D003231B02D21883089B00D2588307DC0ECA
S315080057E0FF23A3409A438B071B0E8407E40EA340AE
S315080057F01A43114B032424021B198408A4001A51C6
S3150800580018E00E4A03071B0F083B9B089B00D2585B
S315080058108307DC0EFF23A3409A438B071B0E8407DE
S31508005820E40EA3401A43054B0407240F083CA408BA
S31508005830A4001A5110BD000000E100E01CED00E0D4
S31508005840F8B504464F1EC8000838211815461E46E6
S31508005850086849683A4606239A4310D02A463346CA
S31508005860FCF730FA3A46D200083AA3181A687F1E9F
S315080058705B68FCF773F906223B469343EED1022F89
S3150800588023D0042F11D0062F2FD12A463346FCF7F2
S3150800589019FAE36AA26AFCF761F92A463346FCF765
S315080058A011FA636A226AFCF759F92A463346FCF765
S315080058B009FAE369A269FCF751F92A463346FCF767
S315080058C001FA63692269FCF749F92A463346FCF767
S315080058D0F9F9E368A268FCF741F92A463346FCF76A
S315080058E0F1F963682268FCF739F9F8BD002210B5AA
S315080058F0134610460149FCF74DFA10BD0000F03F6B
S3150800590010B50122FCF743FC10BD002210B5134662
S3150800591010461146FCF73EFA10BD02E008C8121FF1
S3150800592008C1002AFAD170477047002001E001C17A
S31508005930121F002AFBD17047014908607047000012
S315080059403C020020F0B51FB486B00998089A030DEA
S315080059500021024314D05148514A181850430514DF
S315080059601198012810981AD0281A401C00264D4F65
S315080059704D49009601910490002812DA444211E03C
S315080059801198012449A3012801D11098C14306980A
S31508005990119A84600360C26041600BB0F0BD40425A
S315080059A0E4E70446210500203F4A001C51410391C3
S315080059B0029012E0E00707D032463B46019900986C
S315080059C0FCF780F90191009032463B46104619468D
S315080059D0FCF778F906460F466410002CEAD10498BD
S315080059E0039B0028029A0999089806DAFCF76AF9CF
S315080059F0019B009AFCF766F905E0FCF7CBF9019BD9
S31508005A00009AFCF7C7F904460E460022284BFCF715
S31508005A1087FA03D80020C043014607E00022254B39
S31508005A2020463146FCF79AF8FCF7DCFB102409E01F
S31508005A30002C0ADB0A220023FCF7B6FA079B303251
S31508005A401A55641E02460A43F2D11122641C079BAA
S31508005A50121B1C19119B012B03D0012308430ED1DD
S31508005A600AE0084304D0112010900020119077E72F
S31508005A701098151A6D1E0BE01098824202DD00235D
S31508005A806D1C03E0824201DA00236D1E002BEED066
S31508005A90069811998260C16030C07EE701FCFFFF5D
S31508005AA0104D0000000014400000F03F30000000D8
S31508005AB00000F0430000E03FFFB597B0064600251A
S31508005AC01BE2252876D100242746F749049400E0EE
S31508005AD00443761C32780120203A90400842F7D1D8
S31508005AE030782A280ED00222307801463039092922
S31508005AF016D804990A235943303940181443761C9A
S31508005B000490F1E7189802C804911890002904DA5D
S31508005B100120400304434842049002200443761CB3
S31508005B2030782E2814D1042004437078761C2A284D
S31508005B3009D11898761C80C8189009E00A214F43A5
S31508005B40303FC719761C3078014630390929F5D90E
S31508005B5030786C2810D006DC4C281AD068280ED06D
S31508005B606A2817D104E0742813D07A2812D110E0D5
S31508005B700120400504430CE00121090501E0032149
S31508005B8009050C437178814203D1012000052418C8
S31508005B90761C761C307866280BD013DC58287DD006
S31508005BA009DC00287BD04528F6D04628F4D04728BB
S31508005BB01AD1A9E118E0632835D0642870D0652881
S31508005BC012D1A1E170286CD008DC6728F1D06928C9
S31508005BD07DD06E280DD06F2806D1BCE073282ED054
S31508005BE0752873D0782859D01A9A199990476D1C38
S31508005BF082E16002400F022809D003280DD004284C
S31508005C00189801680DD00D60001D189074E1189859
S31508005C10EA1701680D604A60F6E7189801680D8072
S31508005C20F2E70D70F0E718986A4601781172001DC0
S31508005C3018900020507202A80090012005E01898DC
S31508005C4002C8189000200091C04361070ED50021B4
S31508005C5001E00199491C0191B94213DA8142F8DB46
S31508005C60019A0099895C0029F3D10BE0002101E033
S31508005C700199491C01918142FADB019A0099895CD4
S31508005C800029F5D1019904981A9B471A21463846E6
S31508005C90199A00F099FA4019019903E051E030E1A8
S31508005CA015E050E0451807E0009800990078491C6F
S31508005CB000911A9A199990470198401E0190401C24
S31508005CC0F2D1214638461A9B199A12E137E00A2082
S31508005CD00021009001916002410F022907D0189A0D
S31508005CE001CA1892C2179446032908D00AE01898E0
S31508005CF0C01DC108C90005C91891944607E000B23D
S31508005D00C2179446042902D140B2C1178C46002214
S31508005D106146944506DA0A460021404291418C467E
S31508005D202D2102E0210504D52B216A461173012194
S31508005D3003E0E10701D02021F7E7029156E00A20A7
S31508005D400AE0102008E010200090002104200443F7
S31508005D500191082703E008200021019100906002C4
S31508005D60410F022907D0189A01CA189200229446B0
S31508005D70032908D008E01898C01DC108C90005C93C
S31508005D801891944603E080B2042900D1C0B20021DC
S31508005D90029121072AD531780D91702906D0009AEB
S31508005DA01021019B4A401A4305D00EE040216A465D
S31508005DB01173012108E06146014306D030216A4685
S31508005DC011730D99517302210291009A0821019BC2
S31508005DD04A401A430AD16146014301D1610705D5F4
S31508005DE030216A46117301217F1E029131785829A4
S31508005DF004D02EA10E910DA90D910DE030A1F9E761
S31508005E006146019B009AFCF7CFF80E9B8C469B5C7B
S31508005E100D9A521E0D92137061460143F0D10D98EA
S31508005E2005A9081A20300190600703D5012000044F
S31508005E30844300E001270198874201DD381A00E013
S31508005E400020019900904118029809180498401AF0
S31508005E500490E00306D421461A9B199A049800F088
S31508005E60B3F94519002706E003A81A9AC05D1999DF
S31508005E7090476D1C7F1C02988742F5DBE0030CD522
S31508005E8021461A9B199A049800F09EF9451904E0D0
S31508005E901A9A3020199990476D1C0099481E00904F
S31508005EA00029F5DC1FE000000928010030313233F3
S31508005EB03435363738396162636465660000000038
S31508005EC03031323334353637383941424344454622
S31508005ED0000000000D980D990078491C0D911A9A3A
S31508005EE0199990476D1C0199481E01900029F1DC0B
S31508005EF04DE100F059F94519761C3078002800D094
S31508005F00DFE528461BB0F0BD600700D406271898C1
S31508005F10C01DC108C90048680A680831C30FDB07F5
S31508005F201891190001D09CA108E0210501D59BA173
S31508005F3004E0E10701D09AA100E09AA1430010917C
S31508005F4030785B0865280CD006DC452809D0462839
S31508005F501DD0472841D141E0662818D067283CD192
S31508005F603CE00021112F01DB112000E0781C019193
S31508005F70009008A911A8FFF7E5FC139905910021DF
S31508005F80119A15927F1C12980197009150E00120F2
S31508005F90C00703900120019008A9009711A8FFF7F0
S31508005FA0D1FC139A149905920022119B009212981B
S31508005FB01593059A0192002901D0104602E0791C32
S31508005FC040180190381A01D5019804E04042401E55
S31508005FD00090781C0190C01B029043E0012F00DA64
S31508005FE001270021112F01DD112000E0384601911B
S31508005FF0009008A911A8FFF7A5FC13990591119A15
S315080060000021129815920091019721070CD4059941
S31508006010B94201DB019900E00191012904DD159AD5
S31508006020491E515C302906D0B84201DA011D05DA4D
S315080060300121029115E00199491EEDE7002805DCCA
S315080060400099411800910199091A03E0019A411C27
S31508006050914200DD01910099401A401C02900120EE
S31508006060C0070390200706D402990198814202DBF3
S315080060700020C043029000206946C87707AF012177
S3150800608003980337C907884224D0022011902B2091
S315080060901290039800280CDA404203902D201290A3
S315080060A007E00A210398FBF737FC30317F1E03907F
S315080060B039701199481E11900029F2DC03980028BE
S315080060C0EFD1791E129808703078202108404530A3
S315080060D0BF1E387006A8C01BC01D03901098007814
S315080060E0002800D00120019941180298C017091804
S315080060F0039809180498401A401E0490E00306D431
S3150800610021461A9B199A049800F05EF845191098CA
S315080061100078002803D01A9A199990476D1CE00355
S3150800612024D521461A9B199A049800F04DF845196A
S315080061301CE00098002807DB00990598884203DDD3
S315080061401598405C199901E0199930201A9A9047D8
S3150800615000986D1C401C00900298401E0290002872
S3150800616004D11A9A2E20199990476D1C0199481E38
S3150800617001900029DDDC05E038781A9A7F1C199908
S3150800618090476D1C0399481E03900029F4DC2146AC
S315080061901A9B199A0498ACE62D0000002B00000003
S315080061A02000000000000000F8B5044600251E4641
S315080061B01746880404D405E039462020B0476D1CEC
S315080061C0641EF9D52846F8BDFFB50446002581B0FA
S315080061D01E46C80301D5302700E02027880404D5C9
S315080061E005E038460399B0476D1C641EF9D5284664
S315080061F005B0F0BD10B51D480078012835D100203E
S315080062001A4908701A49088012E01948008840009F
S315080062101849085A18490988C900184A8918144A91
S3150800622012885200885212480088401C104908807B
S315080062300F4800880428E8DB7E20FFF769FA012169
S315080062400F48FCF709FA01210D48FCF76DF90A48D1
S315080062500088401C0849088008460088142804DB82
S315080062600020088001200749087010BD7801002029
S315080062708E0100207004002090010020A804002050
S31508006280002401407001002010B51C480068002851
S3150800629032D000201949086000211948FCF750F946
S315080062A018490978C900184A8918488001211448EC
S315080062B0FCF746F913490978C900134A89188880F2
S315080062C00C210F48FCF73CF90E490978C9000E4A1B
S315080062D08918C8800B480078401C0A490870084687
S315080062E00078142804DB002008700120074908708C
S315080062F001210348FCF7B0F910BD00000802002090
S31508006300002401402C020020501600201002002014
S3150800631010B502460023002901D1002010BD03E074
S315080063201488921CE01883B208464C1EA1B20028B5
S31508006330F6D11846F2E7000070B50025B148807A14
S3150800634001280ED1AF483838C06A7D21C900884275
S3150800635007D90021AB4881720020AB490880AB49B8
S315080063600870A848407A012874D1A748007A0128FD
S3150800637011D003280ED1A648807E002806D1A14850
S31508006380007A002802D101219E48017200209D4909
S31508006390383948612FE19C48407A082870D007DCD4
S315080063A00300FFF702FA0816275A88859FA0B085CA
S315080063B0A5287AD006DC092878D00A2877D0A1281B
S315080063C076D105E1AA2874D0AB2873D0B128F7D1C5
S315080063D00DE100208B493839486101218948C1718E
S315080063E0002202218B48FFF712F800208549383928
S315080063F0C860FEE000208349383948618248807ABF
S31508006400012811D18048007B282825DA7E48007BA0
S315080064100A2821DD7C48017B7A4810304181012118
S3150800642010388173C17017E07748807A022812D134
S31508006430754A117BD07A00F089FE0546282D0BDABD
S315080064400A2D09DD6F481030458101211038817306
S31508006450C17001E0D3E070BDCBE00020694938394E
S3150800646048616948807A02281ED1674A117BD07A2A
S3150800647000F06CFE012804D103216548817613E0FB
S3150800648051E0614A117BD07A00F060FE00280BD1FA
S3150800649000215F4881765B48C07B012804D100F063
S315080064A027FD00215748C173A3E094E043E089E043
S315080064B09EE093E096E05448807A02280ED1524A2C
S315080064C0117BD07A00F042FE4E491031C880012176
S315080064D04C48C173002001F0EFF902E0012001F0F9
S315080064E0EBF986E085E00020464938394861464A96
S315080064F0117BD07A00F02AFE4249103148800120EB
S3150800650001F040FA75E000203E49383948613E4AB4
S31508006510117BD07A00F01AFE3A49103188800320A0
S3150800652001F030FA65E00020364938394861022022
S3150800653001F028FA5DE000203249383948613249CD
S31508006540887AC117890F091889108900411A33D129
S315080065502D49887AC117890F09188910294A1032D6
S315080065601181104600891C2826DA00241FE0A200A3
S31508006570921D254B9B1D995CA200521D985C00F04C
S31508006580E5FD0146A2001F481E308152A2000832CE
S315080065901D4B9B1D995CA200D21D985C00F0D6FD90
S315080065A00146A20017481E3010184180641C154881
S315080065B010300089A042DADC042001F0E3F900F08B
S315080065C097FC16E0052001F0DDF900F091FC10E0DB
S315080065D001F09EF90DE001F037F90AE001210C48B7
S315080065E0417706E001210A482030817101E000E088
S315080065F000BF00BF00BF00BF00210248417200BFB4
S3150800660029E70000780200204805002092010020B2
S3150800661000040020003801400EB5454800780028DF
S3150800662021D144490870012043490D233A2200919B
S31508006630019005210B20FDF7B1FF12203F493123B8
S315080066400C220091019016212120FDF7A7FF0020BA
S315080066503B49086001203649087002213948C17251
S315080066600020394908703948006800284ED0344857
S31508006670006832285BD336480078002820D1354890
S3150800668000780A2811DA334800782C49324A31232F
S315080066900092019102900C2216212120FEF734F86F
S315080066A02C480078401C2B4908702A4800780A288C
S315080066B028D100202749087001202549087021E0C3
S315080066C024480078322814DA224800780921081A62
S315080066D0C0B21A49204A31230092019102900C2235
S315080066E016212120FEF710F81A480078401C19498F
S315080066F00870184800780A2804D10020154908703F
S315080067001349087000200E49086010E00E4800780A
S3150800671000280CD11420094931230C22009101903C
S3150800672016212120FDF73AFF0120074908700EBD02
S31508006730CC00002014010020D6080000E406000062
S31508006740D000002078020020D9010020F0010020A6
S31508006750D7010020D8010020C6D500081CB58B48F3
S31508006760007800286FD18A49087001208749087087
S31508006770002088490870884908608849087088494F
S31508006780087088488078884908706C20FDF7B2FF41
S31508006790012086490D233A220091019005210B20FC
S315080067A0FDF7FCFE00240EE01020E121890000918F
S315080067B00190E0000146143105233C220A20FDF72A
S315080067C0EDFE601CC4B2102CEEDB7748007800287A
S315080067D02ADD01240EE00F20E121890000910190B5
S315080067E0E00001460C3105233C220A20FDF7D6FEBF
S315080067F0601CC4B26C4800788442ECDD6C480078B2
S31508006800002818D00D20E121890000910190601E12
S31508006810C0000C3081B205233C220A20FDF7BEFEDB
S3150800682001205F49087006E061480078002802D018
S3150800683001205B49087045205E490870601EC0004B
S315080068400C305D4908705A480078002847D05448EB
S315080068500078002806D101205149087000204B49CC
S3150800686008701CBD50480078002800D1F9E74A484E
S315080068700068212815D3494800783C2811DA4D4983
S315080068800978464A1278891A88B24B490978FDF779
S315080068901DFF42480078401C4049087000203E49C8
S315080068A008603E4800783C286DDB0D20E121890010
S315080068B005233C22009101903F4801780A20FDF704
S315080068C06DFE00203549087036484088401C364918
S315080068D00978884257D100202C49087053E030487F
S315080068E00078012805D10020284908702C4908702D
S315080068F0B7E72D480078102840DA2B4800780D288D
S315080069003CDB25480068FF21913188423BD321486A
S315080069100078002817D1244804780EE00F20E121DA
S31508006920890000910190E0000146143105233C22BC
S315080069300A20FDF733FE601CC4B2102CEEDB0120E2
S315080069401449087016E0184804780EE01020E12172
S31508006950890000910190E0000146143105233C228C
S315080069600A20FDF71BFE601CC4B2102CEEDB0020CB
S315080069700849087000200849086004E00020064914
S3150800698008600449087000BF6BE70000C9000020D2
S3150800699014010020D3010020D0000020D1010020DE
S315080069A0D201002088030020CE010020D60800006E
S315080069B0CD000020CF010020D00100201CB53248B0
S315080069C0007800282DD1314908706C20FDF792FE19
S315080069D001202F490D233A220091019005210B2011
S315080069E0FDF7DCFD11202B497B230C220091019039
S315080069F016212120FDF7D2FD1320B42105230C22F0
S31508006A00009101908D212120FDF7C8FD01201E4926
S31508006A100870002020490870204908600221204893
S31508006A20C1721F4910314A888988511A0A397D224C
S31508006A30D200514308464E21FAF784FF17490968E0
S31508006A40884220D8144800784E2812DC1320B42136
S31508006A5000910190104800788D22101A81B2052302
S31508006A600C222120FDF79AFD0B480078401C0A49A4
S31508006A700870094800784E2802DD0020064908708B
S31508006A800020064908601CBDCB0000201401002028
S31508006A90D60800004C110000D6010020D0000020C6
S31508006AA0780200201CB57D48007800281ED16C208D
S31508006AB0FDF720FE01207A490D233A220091019024
S31508006AC005210B20FDF76AFD0320764971231B2259
S31508006AD0009101901E211A20FDF760FD01206F49E3
S31508006AE00870002070490870704908606F4800688F
S31508006AF0502875D300206D4908606D48007803005A
S31508006B00FEF753FE0EB3C8C8A291806F5D4C3B2AB0
S31508006B101908C2C866480078624971231B22009189
S31508006B2001901E211A20FDF739FD61480078401CA6
S31508006B305F490870AFE05E4800785A4971231B2206
S31508006B40009101901E211A20FDF728FD584800786B
S31508006B50401C574908709EE05548007851497123F2
S31508006B601B22009101901E211A20FDF717FD50489F
S31508006B700078401C4E4908708DE04D480078494918
S31508006B8071231B22009101901E211A20FDF706FD94
S31508006B9047480078401C464908707CE0444800781D
S31508006BA0404971231B22009101901E211A20FDF7EE
S31508006BB0F5FC3F480078401C3D4908706BE03C48AE
S31508006BC00078384971231B22009101901E211A2052
S31508006BD0FDF7E4FC36480078401C354908705AE051
S31508006BE05AE0334800782F4971231B2200910190FF
S31508006BF01E211A20FDF7D2FC2D480078401C2C498E
S31508006C00087048E02A480078264971231B2200911B
S31508006C1001901E211A20FDF7C1FC25480078401C6A
S31508006C202349087037E0224800781E4971231B2241
S31508006C30009101901E211A20FDF7B0FC1C4800782F
S31508006C40401C1B49087026E019480078154971232D
S31508006C501B22009101901E211A20FDF79FFC144863
S31508006C600078401C1249087015E00F480078401C4F
S31508006C700D490870084600780A2804D100200870D3
S31508006C8003200B49087006E00020094908700949E5
S31508006C90087000E000BF00BF1CBD0000C80000204F
S31508006CA0D6080000C1230000CD010020D000002036
S31508006CB0CC010020140100200EB53A4800780028BF
S31508006CC021D1394908706C20FDF714FD0120374998
S31508006CD00D233A220091019005210B20FDF75EFC59
S31508006CE0112033497B230C22009101901621212083
S31508006CF0FDF754FC01202B49087001212D48C1726B
S31508006D0000202D4908602C480068322849D32B48B2
S31508006D100078002820D12A4800780A2811DA28485D
S31508006D2000782349274A7B230092019102900C227E
S31508006D3016212120FDF7E8FC21480078401C20494F
S31508006D4008701F4800780A2828D100201C490870B6
S31508006D5001201A49087021E0194800780A2814DA2F
S31508006D60174800780921081AC0B21149154A7B2329
S31508006D700092019102900C2216212120FDF7C4FCF5
S31508006D800F480078401C0E4908700D4800780A28FC
S31508006D9004D100200A4908700849087000200649ED
S31508006DA008600EBDCA00002014010020D6080000A5
S31508006DB04C11000078020020D0000020D4010020E9
S31508006DC0D50100207AC4000870B505460C4614485B
S31508006DD0844200DD0446002D02D0012D1ED10CE0B0
S31508006DE0602101208007FEF783F900210120800732
S31508006DF0FEF7DCF90B490C7010E00A480078A0424F
S31508006E0009D0602101208007FEF772F9214601208A
S31508006E108007FEF7CBF903490C7000BF00BF70BDB1
S31508006E20E7030000F8010020826904231A40002ABB
S31508006E300BD0002904D0C26910231A43C2610FE09F
S31508006E40C26910239A43C2610AE0002904D0C269C4
S31508006E5020231A43C26103E0C26920239A43C26110
S31508006E607047000010B5052416E0FF2101311F48C0
S31508006E70FAF795FDFF2101311C48FBF797FEFE2125
S31508006E801A48FBF779FD01461848C030C08F814281
S31508006E9002D100F0BBFC10BD2046611ECCB2002812
S31508006EA0E3D1052416E0FF2101311048FAF777FDF2
S31508006EB0FF2101310D48FBF797FEFE210B48FBF732
S31508006EC05BFD01460948C030C08F814202D100F0FF
S31508006ED09DFCE0E72046611ECCB20028E3D100F015
S31508006EE0BBF900F005F800BFD5E7000088020020CE
S31508006EF010B5FBF7EFFF1A491A48018108300089D7
S31508006F001C2815DA1748083001890E30FBF78AFC69
S31508006F1014490831088908E000228300114916310E
S31508006F20CA52830059184A80401C1E28F4D300E030
S31508006F3010BDFE210B480830FBF71EFD0146094827
S31508006F40C830C187FF210131C038FBF789FEFF2110
S31508006F50013104480830FBF78FFE00BFE8E7000060
S31508006F60FBAA00008002002070B504460D46E1B277
S31508006F700548FEF797FA00BF01210348FEF735FAE0
S31508006F800028F9D0204670BD0038014010B5002809
S31508006F9023D0124B0022001F196803E0814203D850
S31508006FA00A4649680029F9D1002A0AD01368841AC2
S31508006FB09C4204D1006818181060104602E0506020
S31508006FC000E01860002907D002680B1A934203D123
S31508006FD00B68D21802604968416010BD340200206F
S31508006FE070B5044600250121554881720020544990
S31508006FF03839C86253480088FA2804DD0020514908
S31508007000088051490870504800780300FEF7CDFB08
S3150800701008051624384451667295AA2C0DD101200C
S3150800702049490870474801880088401C454A10802D
S31508007030901D445400201146C8707FE0FB2C0AD1ED
S31508007040404801880088401C3E4A1080901D4454E0
S3150800705002203D49087071E0012C03D103203A490A
S31508007060087004E0032C02D1062037490870354819
S3150800707001880088401C334A1080901D44545DE006
S31508007080304801880088401C2E4A1080901D4454C0
S3150800709004202D49087051E02A4884700188008828
S315080070A0401C284A1080901D445405202649087023
S315080070B044E02448C078401CC0B22249C870897888
S315080070C0884202DB0620204908701E48018800888D
S315080070D0401C1C4A1080901D44542FE01948018812
S315080070E00088401C174A1080901D445407201649F2
S315080070F0087023E0134801880088401C114A108054
S31508007100901D4454801F0188801DFBF735FC00281C
S3150800711009D100210A4881720121417200200A49D9
S3150800712008700849088007480088FA2804DD002006
S31508007130044908800449087000E000BF00BF70BD1C
S3150800714078020020480500209201002070B502460A
S31508007150002013460C461D02FF26360235402543FD
S31508007160284670BD00BF00BF00BF00BF00BF00BFFC
S3150800717000BF00BF00BFFEE710B52748007800280B
S315080071800DD1264880887D21C900484324490860D6
S3150800719000202449086001201F4908703AE01E486B
S315080071A00078012809D11F48006800F07BFD0446D5
S315080071B00121204600F012FC2CE01748007802282E
S315080071C012D1194800681949884209D91548006832
S315080071D000F068FD04460121204600F0FFFB19E097
S315080071E003200D49087015E00B480078032811D1D3
S315080071F00D480068002809D00A48006800F052FDCA
S3150800720004460121204600F0E9FB03E00021084678
S3150800721000F0E4FB10BD00001601002088020020E3
S31508007220EC010020F4010020F001002010270000E6
S315080072300749084801810021083041805F21C900BB
S31508007240C180152181805F2101810021418170471C
S31508007250FBAA00008003002000201C4A1C490A8162
S31508007260282208314A8014228A8002220A81192299
S315080072704A81184A8A819200CA8000BF0FE000221C
S31508007280830013498E31CA52830059184A808300F5
S315080072900F491631CA52830059184A80401C1C28C7
S315080072A0EDDB00220A490831CA81FA220A82142231
S315080072B04A82FA228A8200228031CA80FA22891DED
S315080072C04A8014228A80FA22CA807047FBAA0000E4
S315080072D080020020EE020000F0B5C54A00248FB0F7
S315080072E091420ADA4B005B08934206D801254A0008
S315080072F06D05EA4205D1002803D0FEF701FB0FB061
S31508007300F0BD01252D05A94219DA034308D0002945
S3150800731010DA0120FEF710FBFEF7F7FA0FB0F0BD02
S315080073200220FEF709FBFEF7E1FA0122D2075140D7
S315080073300FB0F0BD3524E4433622FAF728FF0A15C4
S31508007340AC4B1219D4180A03120BAB49AB4B56189F
S315080073502E403146594011430192321512190B92AB
S315080073600022FAF7A0FC019A0446921C1003A44EC8
S31508007370000B0D467E44032860D2204673683268A7
S31508007380FAF7BAFD1CD10B98002815D0FAF716FFA4
S3150800739004460E469B4A9C4BFAF794FC0D46074654
S315080073A09A4A9B4B20463146FAF78CFC3A462B46BE
S315080073B0FAF7D4FB0FB0F0BD716830680FB0F0BDB6
S315080073C0944A954B20462946FAF77CFC0022934BB3
S315080073D0FAF76FFC06460F4622462B461046194614
S315080073E0FAF770FC32463B46FAF76CFC06460B98F1
S315080073F00F4600281DD0FAF7E1FE824A824B059116
S315080074000490FAF75FFC32463B46FAF752FC2246EE
S315080074102B46FAF748FC04460D467C4A7C4B0599F0
S315080074200498FAF74FFC22462B46FAF73CFC0FB0B5
S31508007430F0BD0B46324620462946C4E00123002209
S315080074409B072046FAF78AFB02460B462046294642
S31508007450FAF7A0FC06460F460B98FAF7AFFE324637
S315080074603B460591049010461946FAF72BFC0991FC
S315080074700C906B490198099B421800920C9A194680
S315080074801046FAF71FFC024607910A9065490198CB
S315080074900B1A6548019303217844079BFEF7D0F938
S315080074A0079B0A9AFAF70EFC0E905F480D91042185
S315080074B07844079B0A9AFEF7C3F9099B0C9AFAF7D0
S315080074C001FC019B009A1A4300920D9B0E9AFAF74B
S315080074D045FB009A01910C90002A4DDD0022D2430B
S315080074E020462946FAF753FE22462B46FAF7EAFBC8
S315080074F000910A900B9800282BD0424A424B0599D6
S315080075000498FAF7DFFB07910E90019B0C9A0099F5
S315080075100A98FAF723FB32463B46FAF7D3FB079B52
S315080075200E9AFAF71BFB009B0A9AFAF7C2FB224649
S315080075302B46FAF7B8FB04460D46344A344B0599F0
S315080075400498FAF7BFFB22462B46FAF7ACFB0FB0B6
S31508007550F0BD019B0C9A0A98FAF700FB32463B46A7
S31508007560FAF7B0FB009B0A9AFAF7A3FB22462B46CA
S31508007570FAF79FFB0FB0F0BD0B98002827D0214AD9
S31508007580214B05990498FAF79DFB07910090204630
S315080075902946019B0C9AFAF786FB32463B46FAF7D0
S315080075A091FB079B009AFAF77EFB22462B46FAF7D1
S315080075B07AFB04460D46154A154B05990498FAF7C1
S315080075C081FB22462B46FAF76EFB0FB0F0BD0B4641
S315080075D0204629460C9AFAF766FB32463B46FAF7E6
S315080075E071FB22462B46FAF764FB0FB0F0BD00008C
S315080075F00000F07F01FCFFFF645F09000000F03F18
S31508007600386C0000763C7935EF39EA3D0000E0FE3B
S31508007610422EE63F555555555555D53F0000E03F96
S3150800762086EBF9FF51B80600DC6A0000FDF776FC28
S31508007630E1204002FBF74AF9FDF76AFEFFF712FC64
S3150800764000F0BEF800213748C171FBF735FDFCF79D
S31508007650D1FAFCF7F9FDFDF7CBF8FCF7C3FBFCF70D
S31508007660F5FB3148006A000C000420302E490862F8
S315080076702E4A2F490B20FCF75DFC2E4A2C490C207C
S31508007680FCF758FC2C4A2D491120FCF753FC2C4AD0
S315080076902C491220FCF74EFC2348006A000C000413
S315080076A0801C21490862FCF71DF8FAF7B9FE01218A
S315080076B02548FAF7D1FFFF2101310920C006FBF75B
S315080076C006FF0021084600F089F929E01548C07927
S315080076D0002802D001281ED108E0FEF72DFEFAF791
S315080076E0E9FFFBF7BBFD00F069FA18E00021084640
S315080076F0FFF76AFB0B483838C0681449884207D92F
S3150800770000210848C171012202211148FDF77FFEB8
S31508007710FBF734F803E000210248C17100BF00BF3F
S31508007720D4E700007802002000300140F87C000809
S31508007730C1230000B9A000087AC400084C11000053
S31508007740C6D50008E406000000240140204E0000CB
S3150800775000380140F0B50B30C108C900144F0026A7
S31508007760144A0FE003688B420BD38B4205D95C1A87
S315080077704318456830C3083B00E04368136002C0FD
S3150800778004E0021D10680028ECD13046002803D119
S315080077903868002801D00020F0BD064A0648106067
S315080077A0064A121AD208D20044C001203860D7E728
S315080077B03802002034020020041700200019002097
S315080077C010B540210F48FAF7EAF840210D48FBF7B3
S315080077D029FA06210B48FEF79BFD0A498989884242
S315080077E00AD10848083800890749884208D0FFF7AF
S315080077F01FFDFDF795FF03E0FFF71AFDFDF790FF64
S3150800780010BD000088030020FBAA000010B5002464
S315080078100C484089052803DB0A484089282803DDE7
S315080078201921084841810124064800891D2803DDDD
S315080078300124022103480181012C01D1FFF758FBDD
S3150800784010BD00008802002070B5A0B000250026F3
S3150800785080216846FAF7A3F8AA2168460170FB2139
S31508007860417001218170A521C1701248007A8006F5
S31508007870010E6846017102790E490E31401DFAF76C
S3150800788075F868460079411D6846FBF775F80446A1
S31508007890211268460079401D6A46115468460079E7
S315080078A0801D145468460079C11D6846FDF784FD9D
S315080078B020B070BD8802002030B5A1B004468021F2
S315080078C001A8FAF76CF80025AA2168460171FB2180
S315080078D0417101218171A621C17102210172FF2026
S315080078E0000220400112684641728472072101A8ED
S315080078F0FBF742F80546FF200002284001126846B9
S31508007900C1720573092101A8FDF756FD21B030BDE6
S31508007910F0B5A1B000260027802101A8FAF73FF8A4
S315080079200025AA2168460171FB2141710121817157
S31508007930A121C1710B2101720FA5027A29460930CE
S31508007940FAF714F86846007A411D01A8FBF714F8FF
S31508007950044621126846007A401D01AA1154684659
S31508007960007A801D14546846007AC11D01A8FDF7E7
S3150800797023FD21B0F0BD00004E5F433243355F560C
S31508007980315F330030B5A1B00446802101A8FAF76B
S3150800799006F80025AA2168460171FB2141710221DA
S315080079A081710521C17102210172FF200002204068
S315080079B00112684641728472072101A8FAF7DCFFB2
S315080079C00546FF200002284001126846C172057369
S315080079D0092101A8FDF7F0FC21B030BDF0B585B04E
S315080079E005460C46002C0ED10020674908706749E9
S315080079F008606749086000210846FFF7E5F9002096
S31508007A0064490860BEE03220634908602846FAF7F0
S31508007A1044FA0646614801683046FAF7BBFA2CD2A2
S31508007A2059480078002828D15C48006858490860F9
S31508007A302846FAF732FA02902846FAF72EFA009004
S31508007A40564801680098FAF706F801900299FAF77D
S31508007A5047F853490390FAF706F807465149F9F7E4
S31508007A60A9FF0646FAF720FA48490860084600883A
S31508007A7081B20120FFF7A8F970E02846FAF70DFA57
S31508007A800646464801683046FAF784FA23D23E4845
S31508007A90007801281FD13E48016840480068FAF777
S31508007AA06FFA5BD801208007FDF728FB3749086085
S31508007AB0084600683C49884208D234480068401C99
S31508007AC0324A81B210600120FFF77EF93348006818
S31508007AD02F49086042E02846FAF7DFF906462F489C
S31508007AE001683046FAF74CFA0DD12C480068284947
S31508007AF0086001208007FDF701FB24490860012082
S31508007B00214908702AE02846FAF7C7F906462348A5
S31508007B1001683046FAF734FA20D21D4801681F4832
S31508007B200068FAF737FA19D801208007FDF7E6FA50
S31508007B30164908600120144908701448006832285C
S31508007B4008D912480068401E104A81B21060012008
S31508007B50FFF73AF9114800680D49086013480068AC
S31508007B6000280FD11248007801280BD102201049AD
S31508007B700870104841888088081A7D21C900484342
S31508007B800D49086005B0F0BD00020020FC01002088
S31508007B9004020020F4010020DC000020240200205A
S31508007BA000802C4400009643DE030000EC01002010
S31508007BB01601002088020020F001002010B5314887
S31508007BC0007800281CD101202F49087000202F4971
S31508007BD008702F4908702F4908702F4908702F49D7
S31508007BE008702F490870FBF7B7FE01210807FBF755
S31508007BF053FF01210846FBF7FFFDFBF70FFF3FE0A8
S31508007C002048007801281CD1002022490870224902
S31508007C100870224908702249087000210846FFF7B3
S31508007C20DDFE19480078012805D10020184908709A
S31508007C30FEF738FF24E0002014490870FEF78EFD91
S31508007C401EE01048007802281AD100200F49087053
S31508007C500F490870FFF790FA11480078012802D1F9
S31508007C60FFF72AF80CE00E480078022802D1FEF742
S31508007C70A5FE05E00A480078032801D1FEF7CCFCEA
S31508007C8010BD00001301002014010020C8000020C8
S31508007C90C9000020CA000020CB000020CC0000202C
S31508007CA016010020F8B5054600247D21C90028469E
S31508007CB0F9F732FE064600270020009000BF0BE0C9
S31508007CC0A1000C48405AB04205DCA1000948081832
S31508007CD0408800900127641C06480E380089A04297
S31508007CE0EEDC002F03D103480E38008A0090009876
S31508007CF0F8BD00009602002000006C00006C000031
S31508007D006C00006C00006C00006C00006C00006CDD
S31508007D1000006C00006C00006C00006C00006C0039
S31508007D20006C00006C00006C00006C00006C000029
S31508007D306C00006C00006C00006C00006C00006CAD
S31508007D4000006C00006C00006C00006C00006C0009
S31508007D50006C00006C00006C00006C00006C0000F9
S31508007D606C00006C00006C00006C00006C00006C7D
S31508007D7000006C00006C00006C00006C00006C00D9
S31508007D80006C00006C00006C00006C00006C0000C9
S31508007D906C00006C00006C00006C00006C00006C4D
S31508007DA000006C00006C00006C00006C00006C00A9
S31508007DB0006C00006C00006C00006C00006C000099
S31508007DC06C00006C00006C00006C00006C00006C1D
S31508007DD000006C00006C00006C00006C00006C0079
S31508007DE0006C00006C00006C00006C00006C000069
S31508007DF06C00006C00006C00006C00006C00006CED
S31508007E0000006C00006C00006C00006C00006C0048
S31508007E10006C00006C00006C00006C00006C000038
S31508007E206C00006C00006C00006C00006C00006CBC
S31508007E3000006C00006C00006C00006C00006C0018
S31508007E40006C00006C00006C00006C00006C000008
S31508007E506C00006C00006C00006C00006C00006C8C
S31508007E6000006C00006C00006C00006C00006C00E8
S31508007E70006C00006C00006C00006C00006C0000D8
S31508007E806C00006C00006C00006C00006C00006C5C
S31508007E9000006C00006C00006C00006C00006C00B8
S31508007EA0006C00006C00006C00006C00006C0000A8
S31508007EB06C00006C00006C00006C00006C00006C2C
S31508007EC000006C00006C00006C00006C00006C0088
S31508007ED0006C00006C00006C00006C00006C000078
S31508007EE06C00006C00006C00006C00006C00006CFC
S31508007EF000006C00006C00006C00006C00006C0058
S31508007F00006C00006C00006C00006C00006C000047
S31508007F106C00006C00006C00006C00006C00006CCB
S31508007F2000006C00006C00006C00006C00006C0027
S31508007F30006C00006C00006C00006C00006C000017
S31508007F406C00006C00006C00006C00006C00006C9B
S31508007F5000006C00006C00006C00006C00006C00F7
S31508007F60006C00006C00006C00006C00006C0000E7
S31508007F706C00006C00006C00006C00006C00006C6B
S31508007F8000006C00006C00006C00006C00006C00C7
S31508007F90006C00006C00006C00006C00006C0000B7
S31508007FA06C00006C00006C00006C00006C00006C3B
S31508007FB000006C00006C00006C00006C00006C0097
S31508007FC0006C00006C00006C00006C00006C000087
S31508007FD06C00006C00006C00006C00006C00006C0B
S31508007FE000006C00006C00006C00006C00006C0067
S31508007FF0006C00006C00006C00006C00006C000057
S315080080006C00006C00006C00006C00006C00006CDA
S3150800801000006C00006C00006C00006C00006C0036
S31508008020006C00006C00006C00006C00006C000026
S315080080306C00006C00006C00006C00006C00006CAA
S3150800804000006C00006C00006C00006C00006C0006
S31508008050006C00006C00006C00006C00006C0000F6
S315080080606C00006C00006C00006C00006C00006C7A
S3150800807000006C00006C00006C00006C00006C00D6
S31508008080006C00006C00006C00006C00006C0000C6
S315080080906C00006C00006C00006C00006C00006C4A
S315080080A000006C00006C00006C00006C00006C00A6
S315080080B0006C00006C00006C00006C00006C000096
S315080080C06C00006C00006C00006C00006C00006C1A
S315080080D000006C00006C00006C00006C00006C0076
S315080080E0006C00006C00006C00006C00006C000066
S315080080F06C00006C00006C00006C00006C00006CEA
S3150800810000006C00006C00006C00006C00006C0045
S31508008110006C00006C00006C00006C00006C000035
S315080081206C00006C00006C00006C00006C00006CB9
S3150800813000006C00006C00006C00006C00006C0015
S31508008140006C00006C00006C00006C00006C000005
S315080081506C00006C00006C00006C00006C00006C89
S3150800816000006C00006C00006C00006C00006C00E5
S31508008170006C00006C00006C00006C00006C0000D5
S315080081806C00006C00006C00006C00006C00006C59
S3150800819000006C00006C00006C00006C00006C00B5
S315080081A0006C00006C00006C00006C00006C0000A5
S315080081B06C00006C00006C00006C00006C00006C29
S315080081C000006C00006C00006C00006C00006C0085
S315080081D0006C00006C00006C00006C00006C000075
S315080081E06C00006C00006C00006C00006C00006CF9
S315080081F000006C00006C00006C00006C00006C0055
S31508008200006C00006C00006C00006C00006C000044
S315080082106C00006C00006C00006C00006C00006CC8
S3150800822000006C00006C00006C00006C00006C0024
S31508008230006C00006C00006C00006C00006C000014
S315080082406C00006C00006C00006C00006C00006C98
S3150800825000006C00006C00006C00006C00006C00F4
S31508008260006C00006C00006C00006C00006C0000E4
S315080082706C00006C00006C00006C00006C00006C68
S3150800828000006C00006C00006C00006C00006C00C4
S31508008290006C00006C00006C00006C00006C0000B4
S315080082A06C00006C00006C00006C00006C00006C38
S315080082B000006C00006C00006C00006C00006C0094
S315080082C0006C00006C00006C00006C00006C000084
S315080082D06C00006C00006C00006C00006C00006C08
S315080082E000006C00006C00006C00006C00006C0064
S315080082F0006C00006C00006C00006C00006C000054
S315080083006C00006C00006C00006C00006C00006CD7
S3150800831000006C00006C00006C00006C00006C0033
S31508008320006C00006C00006C00006C00006C000023
S315080083306C00006C00006C00006C00006C00006CA7
S3150800834000006C00006C00006C00006C00006C0003
S31508008350006C00006C00006C00006C00006C0000F3
S315080083606C00006C00006C00006C00006C00006C77
S3150800837000006C00006C00006C00006C00006C00D3
S31508008380006C00006C00006C00006C00006C0000C3
S315080083906C00006C00006C00006C00006C00006C47
S315080083A000006C00006C00006C00006C00006C00A3
S315080083B0006C00006C00006C00006C00006C000093
S315080083C06C00006C00006C00006C00006C00006C17
S315080083D000006C00006C00006C00006C00006C0073
S315080083E0006C00006C00006C00006C00006C000063
S315080083F06C00006C00006C00006C00006C00006CE7
S3150800840000006C00006C00006C00006C00006C0042
S31508008410006C00006C00006C00006C00006C000032
S315080084206C00006C00006C00006C00006C00006CB6
S3150800843000006C00006C00006C00006C00006C0012
S31508008440006C00006C00006C00006C00006C000002
S315080084506C00006C00006C00006C00006C00006C86
S3150800846000006C00006C00006C00006C00006C00E2
S31508008470006C00006C00006C00006C00006C0000D2
S315080084806C00006C00006C00006C00006C00006C56
S3150800849000006C00006C00006C00006C00006C00B2
S315080084A0006C00006C00006C00006C04007000009A
S315080084B06C00006C00007000006C04006C00006C1E
S315080084C000007000006C00006C00006C00006C007E
S315080084D0006C00006C00006C00006C00006C000072
S315080084E06C00006C00006C00006C00006C00006CF6
S315080084F000006C00006C00006C00006C040070004A
S31508008500006C00006C00006C00006C00006C000041
S315080085106C00006C00006C00006C00006C00006CC5
S3150800852000006C04006C00006C00006C00006C001D
S31508008530006C00006C00006C00006C00006C000011
S315080085406C00006C00006C00006C00007000006C91
S3150800855000006C04006C00006C00007000006C00E9
S31508008560006C00006C04007000006C00006C0000D9
S315080085706C00006C00006C00006C00006C00006C65
S3150800858000006C00006C00006C00006C00006C00C1
S31508008590006C00006C00006C00006C00006C0000B1
S315080085A07000006C00006C00006C00006C04007029
S315080085B000006C00006C00006C04006C0000700089
S315080085C0006C00006C00006C00006C00006C000081
S315080085D06C00006C00006C00006C00006C00006C05
S315080085E000006C00006C00006C00006C00006C0061
S315080085F0006C00007004006C204CB82858C40000B9
S315080086006C04007000006C00006C04007004006CC0
S3150800861000006C00006C00006C00006C00006C0030
S31508008620006C00006C00006C00006C00006C000020
S315080086306C00006C00006C00006C00006C00006CA4
S3150800864000006C00006C040470387CE44494FC2838
S3150800865054BC00006C00006C00006C00006C040048
S315080086607000006C00006C04006C00006C00006C6C
S3150800867000006C00006C00006C00006C00006C00D0
S31508008680006C00006C00006C00006C00006C0000C0
S315080086906C00006C00006C2C64CC4498FC3C80E8B0
S315080086A01C40A804047010208C04007000006C00A4
S315080086B0006C00006C00006C00006C00006C000090
S315080086C06C00006C00006C00006C00006C00006C14
S315080086D000006C00006C00006C00006C00006C0070
S315080086E0006C0400702860C83874DC18349C0404D4
S315080086F0742044AC3C88F04098FC2C64C804047090
S3150800870004007000006C00006C04006C00006C0033
S31508008710006C00006C00006C00006C00006C00002F
S315080087206C00006C00006C00006C00006C00006CB3
S3150800873018309C2048B4101C8C00006C101C8C3817
S3150800874080E43478DC3064CC3470D84098FC285403
S31508008750C000006C00006C00006C00006C00006C2F
S3150800876000006C00006C00006C00006C00006C00DF
S31508008770006C00006C00006C00006C00006C0000CF
S315080087806C1C40AC4090F410208C1428981C3CAC0F
S3150800879004047400006C00006C1C40A84494FC207F
S315080087A044AC00006C00006C00006C00006C00001B
S315080087B06C00006C00006C00006C00006C00006C23
S315080087C000006C00006C00006C00006C00006C007F
S315080087D0006C142C984498FC3474D80C148000004F
S315080087E06C00006C00006C00006C3064CC3884E8C7
S315080087F004007000006C00006C00007000006C0043
S31508008800006C00006C00006C00006C00006C00003E
S315080088106C00006C00006C00006C00006C00006CC2
S3150800882000006C0404744094F83470D80404741876
S31508008830349C2C60CC306CD41834A4408CF0204482
S31508008840B000006C00007004006C00006C00006C46
S3150800885000006C00006C00006C00006C00006C00EE
S31508008860006C00006C00006C00006C00006C0000DE
S315080088706C00006C0000703064D03878E03880E412
S315080088803064CC18309C0404741428984090F80876
S31508008890087800006C00006C00006C00006C00009A
S315080088A06C00006C00006C00006C00006C00006C32
S315080088B000006C00006C00006C00006C00006C008E
S315080088C0006C00006C00006C101C883880E40810EE
S315080088D07C0000700404741424943474DC2040ACC6
S315080088E000007000007000006C00006C00006C0056
S315080088F0006C00006C00006C00006C00006C00004E
S315080089006C00006C00006C00006C00006C00006CD1
S3150800891000006C00006C00006C00006C2454BC0461
S3150800892008743068CC2048B01028943064CC000015
S315080089306C00006C00006C00006C00006C00006CA1
S3150800894000006C00006C00006C00006C00006C00FD
S31508008950006C00006C00006C00006C00006C0000ED
S315080089606C00006C00006C00006C00006C080C7851
S3150800897004007000006C00006C0C1480000070008D
S31508008980006C00006C00006C00006C0400700000B5
S315080089906C00006C04007000006C00006C00006C39
S315080089A000006C00006C00006C00006C00006C009D
S315080089B0006C00006C00006C00006C00006C00008D
S315080089C06C00006C00006C00006C00006C00006C11
S315080089D000007000006C00006C00006C00006C0069
S315080089E0006C00007000006C00006C00006C000059
S315080089F06C00006C00006C00006C00006C00006CE1
S31508008A0000006C00006C00006C0000700400700030
S31508008A10006C00007000006C00007000006C000024
S31508008A206C04006C00006C00006C00006C00006CAC
S31508008A3000006C00006C04007000006C00006C0004
S31508008A40006C00006C00006C00006C00006C0000FC
S31508008A506C00006C00006C00006C00006C00006C80
S31508008A6000007000006C04007000006C1C38A40C38
S31508008A70188400006C00007000006C00006C040094
S31508008A806C00006C00006C00006C00006C00006C50
S31508008A9000006C00006C00006C00006C00006C00AC
S31508008AA0006C00006C00006C00006C000070040094
S31508008AB07000006C00006C00006C040070182C98A4
S31508008AC03C80E804006C00006C04006C0400700034
S31508008AD0006C00006C00006C00006C00006C00006C
S31508008AE06C00006C00006C00006C00006C00006CF0
S31508008AF000006C00006C00006C00006C080C781814
S31508008B0038A42044B004087404007000006C1024D3
S31508008B10904498FC14289800007000006C00006CC3
S31508008B2000006C04006C04007000006C00006C000F
S31508008B30006C00006C00006C00006C00006C00000B
S31508008B406C00006C00006C00006C00006C2454BCC7
S31508008B504498FC4498FC387CE41020900C1484104B
S31508008B60208C4090F4080C7800006C04006C00001F
S31508008B706C00006C00006C00006C00006C00006C5F
S31508008B8000006C00006C00006C00006C00006C00BB
S31508008B90006C00006C00006C00006C00006C0000AB
S31508008BA06C0408782858C43878E01C44AC3C84EC3B
S31508008BB010208C3C88EC2C60C4101C8804047014AB
S31508008BC0289400006C00006C00006C00006C00002B
S31508008BD06C00006C00006C00006C00006C00006CFF
S31508008BE000006C00006C00006C00006C00006C005B
S31508008BF0006C00006C1830A00400701C3CA840945F
S31508008C00F81424903C84E82C64CC3474DC3470D892
S31508008C100C148000006C00006C00006C00006C00F6
S31508008C20006C00006C00006C00006C00006C00001A
S31508008C306C00006C00006C00006C00006C00006C9E
S31508008C4000006C00006C1834A0101C8C1C38A43072
S31508008C5068D41024903878DC10208C4494FC20408A
S31508008C60AC00006C00006C00006C00006C0000702A
S31508008C7000006C00006C00006C00006C00006C00CA
S31508008C80006C00006C00006C00006C00006C0000BA
S31508008C906C285CC4387CE04494FC306CD41C38A442
S31508008CA0204CB42C5CC83070D4080C7C1C40AC0C2E
S31508008CB01C8800006C00006C00006C00006C000052
S31508008CC06C00006C00006C00006C00006C00006C0E
S31508008CD000006C00006C00006C00006C00006C006A
S31508008CE0006C3068CC4494FC3070D81C3CA8182C16
S31508008CF0981834A01834A03064C8346CD4101C8872
S31508008D0000006C00006C00006C00007004006C0031
S31508008D10006C00006C00006C00006C00006C000029
S31508008D206C00006C00006C00006C00006C00006CAD
S31508008D3000006C040070101C8C0810802048B410C9
S31508008D40249410208C04006C1424904090F404049D
S31508008D507000007000007000006C00006C00006C71
S31508008D6000006C00006C00006C00006C00006C00D9
S31508008D70006C00006C00006C00006C00006C0000C9
S31508008D806C00006C0408741C40AC387CE40C148439
S31508008D90101C8C0408780000702048B4306CD4008D
S31508008DA0007000006C00006C00006C00006C040091
S31508008DB06C00006C00006C00006C00006C00006C1D
S31508008DC000006C00006C00006C00006C00006C0079
S31508008DD0006C00006C1C40A8408CF42858C00000A9
S31508008DE06C1424942C60C8408CF44494FC1C38A45D
S31508008DF000006C00006C04006C00006C00006C0045
S31508008E00006C00006C00006C00006C00006C000038
S31508008E106C00006C00006C00006C00006C00006CBC
S31508008E2000006C00006C0404742448B4040C781C1C
S31508008E3038A41834A40C188804087800006C0000BC
S31508008E406C00006C04006C00006C04007000006C80
S31508008E5000006C00006C00006C00006C00006C00E8
S31508008E60006C00006C00006C00006C00006C0000D8
S31508008E706C00006C00006C00006C00006C00006C5C
S31508008E8000006C00006C00006C00007000006C04B0
S31508008E90007000007000006C00006C00006C0000A0
S31508008EA06C04006C00007000006C00006C00006C24
S31508008EB000006C00006C00006C00006C00006C0088
S31508008EC0006C00006C00006C00006C00006C000078
S31508008ED06C00006C00006C00007000006C00006CF8
S31508008EE000007000006C00006C00006C00006C0054
S31508008EF0006C00006C00006C00006C00006C000048
S31508008F006C00006C00006C00006C00006C00006CCB
S31508008F1000006C00006C00006C00006C00006C0027
S31508008F20006C04007000006C00006C00007000000B
S31508008F306C3068D00C188400006C00006C0000705F
S31508008F4000006C00006C00006C00006C00006C00F7
S31508008F50006C00006C00006C00006C00006C0400E3
S31508008F607004007000006C00006C00006C00006C5F
S31508008F7000006C1838A000006C00006C000070043B
S31508008F80006C2850BC2854BC00007000007000001B
S31508008F906C00007000006C00006C00006C00006C37
S31508008FA000006C00006C00006C00006C00006C0097
S31508008FB0006C00006C00006C00006C04007004007B
S31508008FC0700C14804494FC204CB404006C0C188873
S31508008FD00C148018349C2044B000006C0400700007
S31508008FE0007000006C00006C00006C00006C000053
S31508008FF06C00006C00006C00006C00006C00006CDB
S3150800900000006C00006C00006C00006C00006C0432
S3150800901008743880E44098FC285CC01C3CA8409042
S31508009020F44498FC2C60C81C3CA804007004006C2E
S3150800903000006C04006C04007000006C00006C00FA
S31508009040006C00006C00006C00006C00006C0000F6
S315080090506C00006C00006C00006C00006C08087462
S315080090603470DC3878E01C38A400006C0404741CE6
S315080090703CA82450B82040AC1830A000006C04006E
S315080090806C04007000006C00006C00006C00006C42
S3150800909000006C00006C00006C00006C00006C00A6
S315080090A0006C00006C00006C04007004047020481A
S315080090B0B01028901C3CA8387CE41024901C38A4D6
S315080090C03C84EC4094F8244CB8142C980808780092
S315080090D0006C00006C00006C00006C00006C000066
S315080090E06C00006C00006C00006C00006C00006CEA
S315080090F000006C00006C00006C00006C00006C0046
S31508009100006C2448B44498FC4498FC3878DC000089
S315080091106C0C1888306CD42858C4346CD43C90F441
S315080091200C1C8800006C00006C00007004007000C5
S31508009130006C00006C00006C00006C00006C000005
S315080091406C00006C00006C00006C0400700C188841
S315080091502C64CC4494FC4498FC3880E808087808C9
S31508009160107C3068D0387CE44498FC4498FC4088ED
S31508009170F02C60C800006C00006C00006C00006CED
S3150800918000006C00006C00006C00006C00006C00B5
S31508009190006C00006C00006C00006C00006C04049D
S315080091A074204CB43880E42860C82C60CC3470D85D
S315080091B04094F84094F82C5CC82C60C818309C1071
S315080091C0208C00006C00006C00006C000070000031
S315080091D06C00006C00006C00006C00006C00006CF9
S315080091E000006C00006C04007000006C0400700441
S315080091F0006C0404743478E01028942048B01020D9
S31508009200882048B408107C080C7C3478E01834A010
S3150800921000006C00006C00006C00006C00006C0024
S31508009220006C00006C00006C00006C00006C000014
S315080092306C00006C00007000006C04006C00006C90
S3150800924000006C2448B40C18841028942048B004F4
S3150800925000700400702044B03470D82C60C8081020
S315080092607C00006C04006C00007000006C00006C50
S3150800927000006C00006C00006C00006C00006C00C4
S31508009280006C04006C00007004006C00006C0000A8
S3150800929070142C98080C78040474346CD82048B0E0
S315080092A00000703470D8285CC0000070285CC40CBC
S315080092B0188800006C00006C00006C00006C000050
S315080092C06C00006C00006C00006C00006C00006C08
S315080092D000006C00006C00007000006C00006C0060
S315080092E0006C00006C00006C0000701C3CA8204854
S315080092F0B40400701834A02040AC1C34A43874DCC4
S3150800930014249000007000006C04007000006C00CB
S31508009310006C00006C00006C00006C00006C04001F
S315080093207000006C00006C00006C00007000006C9F
S3150800933000006C00006C00006C00006C04007008F3
S31508009340107C00006C00006C00006C04007010209B
S315080093508C0C188800006C00007000006C0000700F
S3150800936000006C00006C00006C00006C00006C04CF
S31508009370007000006C00006C00006C00006C0000BF
S315080093806C00006C00006C04006C00006C00006C43
S3150800939000006C00006C00006C00006C00006C049F
S315080093A0006C00006C00007000006C00006C00008F
S315080093B06C00006C04006C00006C00006C00006C13
S315080093C000006C00006C00006C00006C04006C006F
S315080093D0006C00006C00007000006C00006C00005F
S315080093E06C00007000006C00006C18309C0404705F
S315080093F000006C04007000006C00006C00006C003B
S31508009400006C00006C00006C00006C00006C000032
S315080094106C00006C04007000006C04007000006CA6
S3150800942000006C00006C00006C00006C00006C14FE
S31508009430289800006C04007000006C3064CC285436
S31508009440BC00006C00006C00006C00006C00006C36
S3150800945004006C00006C00006C00006C00006C00DE
S31508009460006C00006C00006C04007000006C0000CA
S315080094706C00006C00006C00006C00006C0400704E
S31508009480306CD408108000006C00006C2858C0248A
S3150800949050B800006C00006C04006C00006C0400FE
S315080094A07000006C00006C00006C00006C00006C22
S315080094B000006C00006C00006C00006C040070007A
S315080094C0006C00006C00006C00006C00006C000072
S315080094D06C2450BC04047400006C0000702458BC52
S315080094E0306CD410289400006C00007000006C00EA
S315080094F0006C00006C00006C00006C00006C000042
S315080095006C00006C00006C00006C00006C04006CC1
S3150800951000006C00006C00006C00006C0000700419
S3150800952000703068D4285CC4080C782044A844909D
S31508009530FC4498FC408CF004007004006C00006C3D
S3150800954000006C00006C04007000006C00006C00E9
S31508009550006C00006C00006C00006C00006C0000E1
S315080095607000007000006C00006C00006C04047051
S31508009570285CC44498FC4494FC3068D03878E03CB5
S3150800958084EC2448B4040874080C7C0404780000AD
S315080095906C00006C04007000006C00006C00006C2D
S315080095A000006C00006C00006C00006C00006C0091
S315080095B0006C00006C00006C0000701C3CA8388031
S315080095C0E44498FC4098FC2C64CC08087C040070A1
S315080095D02C60C8204CB83064D018309C00006C0051
S315080095E0006C00006C00006C00007000006C00004D
S315080095F06C00006C00006C00006C00006C00006CD5
S3150800960000006C00007000006C00006C0C1C8834B4
S3150800961070D83070D83470D80C14840404740814C4
S3150800962080387CE42448B44498FC2C60CC04006C54
S3150800963000006C00006C00006C00006C00006C0000
S31508009640006C00006C00006C04006C00006C0000EC
S315080096506C00006C00007004006C04007000006C64
S3150800966000007000006C3474DC10289010249038C8
S3150800967080E80C14841C38A4306CD42854C000002C
S315080096806C00006C00006C04006C00006C00006C40
S3150800969000006C00006C00006C00006C00006C00A0
S315080096A0006C00006C04006C00006C00006C00008C
S315080096B06C00006C204CB43874E000006C2044B494
S315080096C01024902454BC3478DC0808783068D0001C
S315080096D0006C00006C04006C00007000006C040054
S315080096E06C00006C00006C00006C00006C00006CE4
S315080096F004007000006C00006C00006C00006C0434
S3150800970008743068CC1C38A43068D000006C04009B
S31508009710700000702858C43470D8081080387CE46B
S3150800972000006C04007000007004006C00006C00FF
S31508009730006C00006C00006C00006C00006C0000FF
S315080097406C00006C00006C00006C00006C00006C83
S3150800975010208C3068D00808783070D80400700063
S31508009760006C18309C18309C040C78306CD43C88FB
S31508009770EC00006C00006C00006C00006C00006CD3
S3150800978000006C00006C00006C00006C00006C00AF
S31508009790006C00006C00006C00006C00006C00009F
S315080097A06C04007000006C101C882C5CC8000474E3
S315080097B0040070080C7C00006C04006C080C7834FB
S315080097C078DC00007004007000006C00006C00007B
S315080097D06C00006C00006C00006C00006C00006CF3
S315080097E000006C00006C00006C00006C00006C004F
S315080097F0006C00006C00006C00007000006C040037
S315080098007000006C00006C04006C00006C040070B2
S3150800981000006C00006C04007000006C00006C0016
S31508009820006C00006C00006C00006C00006C00000E
S315080098306C00006C00006C04007000006C00006C8A
S3150800984000006C00006C00006C04007004006C00E2
S31508009850006C00006C00006C00006C04006C0400D6
S315080098607000006C04006C00006C00006C00006C5A
S3150800987000006C00006C00006C00006C00006C04BA
S31508009880006C00006C00006C04006C00006C0000AA
S315080098906C00006C00007000006C00006C00006C2E
S315080098A000006C00006C04007000006C00006C0086
S315080098B0006C04006C00006C00006C00006C00007A
S315080098C06C00006C00006C00006C00006C00006C02
S315080098D000006C00006C00006C00006C00006C005E
S315080098E0006C00006C00006C00006C00006C00004E
S315080098F06C00006C00006C00006C00006C00006CD2
S3150800990000006C00006C00006C00006C00006C002D
S31508009910006C00006C00006C00006C00006C00001D
S315080099206C00006C00006C00006C00006C00006CA1
S3150800993000006C00006C00006C00006C00006C00FD
S31508009940006C00006C00006C00006C00006C0000ED
S315080099506C00006C00006C00006C00006C00006C71
S3150800996000006C00006C00006C00006C00006C00CD
S31508009970006C00006C00006C00006C00006C0000BD
S315080099806C00006C00006C00006C00006C00006C41
S3150800999000006C00006C00006C00006C00006C009D
S315080099A0006C00006C00006C00006C00006C00008D
S315080099B06C00006C00006C00006C00006C00006C11
S315080099C000006C00006C00006C00006C00006C006D
S315080099D0006C00006C00006C00006C00006C00005D
S315080099E06C00006C00006C00006C00006C00006CE1
S315080099F000006C00006C00006C00006C00006C003D
S31508009A00006C00006C00006C00006C00006C00002C
S31508009A106C00006C00006C00006C00006C00006CB0
S31508009A2000006C00006C00006C00006C00006C000C
S31508009A30006C00006C00006C00006C00006C0000FC
S31508009A406C00006C00006C00006C00006C00006C80
S31508009A5000006C00006C00006C00006C00006C00DC
S31508009A60006C00006C00006C00006C00006C0000CC
S31508009A706C00006C00006C00006C00006C00006C50
S31508009A8000006C00006C00006C00006C00006C00AC
S31508009A90006C00006C00006C00006C00006C00009C
S31508009AA06C00006C00006C00006C00006C00006C20
S31508009AB000006C00006C00006C00006C00006C007C
S31508009AC0006C00006C00006C00006C00006C00006C
S31508009AD06C00006C00006C00006C00006C00006CF0
S31508009AE000006C00006C00006C00006C00006C004C
S31508009AF0006C00006C00006C00006C00006C00003C
S31508009B006C00006C00006C00006C00006C00006CBF
S31508009B1000006C00006C00006C00006C00006C001B
S31508009B20006C00006C00006C00006C00006C00000B
S31508009B306C00006C00006C00006C00006C00006C8F
S31508009B4000006C00006C00006C00006C00006C00EB
S31508009B50006C00006C00006C00006C00006C0000DB
S31508009B606C00006C00006C00006C00006C00006C5F
S31508009B7000006C00006C00006C00006C00006C00BB
S31508009B80006C00006C00006C00006C00006C0000AB
S31508009B906C00006C00006C00006C00006C00006C2F
S31508009BA000006C00006C00006C00006C00006C008B
S31508009BB0006C00006C00006C00006C00006C00007B
S31508009BC06C00006C00006C00006C00006C00006CFF
S31508009BD000006C00006C00006C00006C00006C005B
S31508009BE0006C00006C00006C00006C00006C00004B
S31508009BF06C00006C00006C00006C00006C00006CCF
S31508009C0000006C00006C00006C00006C00006C002A
S31508009C10006C00006C00006C00006C00006C00001A
S31508009C206C00006C00006C00006C00006C00006C9E
S31508009C3000006C00006C00006C00006C00006C00FA
S31508009C40006C00006C00006C00006C00006C0000EA
S31508009C506C00006C00006C00006C00006C00006C6E
S31508009C6000006C00006C00006C00006C00006C00CA
S31508009C70006C00006C00006C00006C00006C0000BA
S31508009C806C00006C00006C00006C00006C00006C3E
S31508009C9000006C00006C00006C00006C00006C009A
S31508009CA0006C00006C00006C00006C00006C00008A
S31508009CB06C00006C00006C00006C00006C00006C0E
S31508009CC000006C00006C00006C00006C00006C006A
S31508009CD0006C00006C00006C00006C00006C00005A
S31508009CE06C00006C00006C00006C00006C00006CDE
S31508009CF000006C00006C00006C00006C00006C003A
S31508009D00006C00006C00006C00006C00006C000029
S31508009D106C00006C00006C00006C00006C00006CAD
S31508009D2000006C00006C00006C00006C00006C0009
S31508009D30006C00006C00006C00006C00006C0000F9
S31508009D406C00006C00006C00006C00006C00006C7D
S31508009D5000006C00006C00006C00006C00006C00D9
S31508009D60006C00006C00006C00006C00006C0000C9
S31508009D706C00006C00006C00006C00006C00006C4D
S31508009D8000006C00006C00006C00006C00006C00A9
S31508009D90006C00006C00006C00006C00006C000099
S31508009DA06C00006C00006C00006C00006C00006C1D
S31508009DB000006C00006C00006C00006C00006C0079
S31508009DC0006C00006C00006C00006C00006C000069
S31508009DD06C00006C00006C00006C00006C00006CED
S31508009DE000006C00006C00006C00006C00006C0049
S31508009DF0006C00006C00006C00006C00006C000039
S31508009E006C00006C00006C00006C00006C00006CBC
S31508009E1000006C00006C00006C00006C00006C0018
S31508009E20006C00006C00006C00006C00006C000008
S31508009E306C00006C00006C00006C00006C00006C8C
S31508009E4000006C00006C00006C00006C00006C00E8
S31508009E50006C00006C00006C00006C00006C0000D8
S31508009E606C00006C00006C00006C00006C00006C5C
S31508009E7000006C00006C00006C00006C00006C00B8
S31508009E80006C00006C00006C00006C00006C0000A8
S31508009E906C00006C00006C00006C00006C00006C2C
S31508009EA000006C00006C00006C00006C00006C0088
S31508009EB0006C00006C00006C00006C00006C000078
S31508009EC06C00006C00006C00006C00006C00006CFC
S31508009ED000006C00006C00006C00006C00006C0058
S31508009EE0006C00006C00006C00006C00006C000048
S31508009EF06C00006C00006C00006C00006C00006CCC
S31508009F0000006C00006C00006C00006C00006C0027
S31508009F10006C00006C00006C00006C00006C000017
S31508009F206C00006C00006C00006C00006C00006C9B
S31508009F3000006C00006C00006C00006C00006C00F7
S31508009F40006C00006C00006C00006C00006C0000E7
S31508009F506C00006C00006C00006C00006C00006C6B
S31508009F6000006C00006C00006C00006C00006C00C7
S31508009F70006C00006C00006C00006C00006C0000B7
S31508009F806C00006C00006C00006C00006C00006C3B
S31508009F9000006C00006C00006C00006C00006C0097
S31508009FA0006C00006C00006C00006C00006C000087
S31508009FB06C00006C00006C00006C00006C00006C0B
S31508009FC000006C00006C00006C00006C00006C0067
S31508009FD0006C00006C00006C00006C00006C000057
S31508009FE06C00006C00006C00006C00006C00006CDB
S31508009FF000006C00006C00006C00006C00006C0037
S3150800A000006C00006C00006C00006C00006C000026
S3150800A0106C00006C00006C00006C00006C00006CAA
S3150800A02000006C00006C00006C00006C00006C0006
S3150800A030006C00006C00006C00006C00006C0000F6
S3150800A0406C00006C00006C00006C00006C00006C7A
S3150800A05000006C00006C00006C00006C00006C00D6
S3150800A060006C00006C00006C00006C00006C0000C6
S3150800A0706C00006C00006C00006C00006C00006C4A
S3150800A08000006C00006C00006C00006C00006C00A6
S3150800A090006C00006C00006C00006C00006C000096
S3150800A0A06C00006C00006C00006C00006C00006C1A
S3150800A0B000006C00006C00006C00006C00006C0076
S3150800A0C0006C00006C00006C00006C00006C000066
S3150800A0D06C00006C00006C00006C00006C00006CEA
S3150800A0E000006C00006C00006C00006C00006C0046
S3150800A0F0006C00006C00006C00006C00006C000036
S3150800A1006C00006C00006C00006C00006C00006CB9
S3150800A11000006C00006C00006C00006C00006C0015
S3150800A120006C00006C00006C00006C00006C000005
S3150800A1306C00006C00006C00006C00006C00006C89
S3150800A14000006C00006C00006C00006C00006C00E5
S3150800A150006C00006C00006C00006C00006C0000D5
S3150800A1606C00006C00006C00006C00006C00006C59
S3150800A17000006C00006C00006C00006C00006C00B5
S3150800A180006C00006C00006C00006C00006C0000A5
S3150800A1906C00006C00006C00006C00006C00006C29
S3150800A1A000006C00006C00006C00006C00006C0085
S3150800A1B0006C00006C00006C00006C00006C000075
S3150800A1C06C00006C00006C00006C00006C00006CF9
S3150800A1D000006C00006C00006C00006C00006C0055
S3150800A1E0006C00006C00006C00006C00006C000045
S3150800A1F06C00006C00006C00006C00006C00006CC9
S3150800A20000006C00006C00006C00006C00006C0024
S3150800A210006C00006C00006C00006C00006C000014
S3150800A2206C00006C00006C00006C00006C00006C98
S3150800A23000006C00006C00006C00006C00006C00F4
S3150800A240006C00006C00006C00006C00006C0000E4
S3150800A2506C00006C00006C00006C00006C00006C68
S3150800A26000006C00006C00006C00006C00006C00C4
S3150800A270006C00006C00006C00006C00006C0000B4
S3150800A2806C00006C00006C00006C00006C00006C38
S3150800A29000006C00006C00006C00006C00006C0094
S3150800A2A0006C00006C00006C00006C00006C000084
S3150800A2B06C00006C00006C00006C00006C00006C08
S3150800A2C000006C00006C00006C00006C00006C0064
S3150800A2D0006C00006C00006C00006C00006C000054
S3150800A2E06C00006C00006C00006C00006C00006CD8
S3150800A2F000006C00006C00006C00006C00006C0034
S3150800A300006C00006C00006C00006C00006C000023
S3150800A3106C00006C00006C00006C00006C00006CA7
S3150800A32000006C00006C00006C00006C00006C0003
S3150800A330006C00006C00006C00006C00006C0000F3
S3150800A3406C00006C00006C00006C00006C00006C77
S3150800A35000006C00006C00006C00006C00006C00D3
S3150800A360006C00006C00006C00006C00006C0000C3
S3150800A3706C00006C00006C00006C00006C00006C47
S3150800A38000006C00006C00006C00006C00006C00A3
S3150800A390006C00006C00006C00006C00006C000093
S3150800A3A06C00006C00006C00006C00006C00006C17
S3150800A3B000006C00006C00006C00006C00006C0073
S3150800A3C0006C00006C00006C00006C00006C000063
S3150800A3D06C00006C00006C00006C00006C00006CE7
S3150800A3E000006C00006C00006C00006C00006C0043
S3150800A3F0006C00006C00006C00006C00006C000033
S3150800A4006C00006C00006C00006C00006C00006CB6
S3150800A41000006C00006C00006C00006C00006C0012
S3150800A420006C00006C00006C00006C00006C000002
S3150800A4306C00006C00006C00006C00006C00006C86
S3150800A44000006C00006C00006C00006C00006C00E2
S3150800A450006C00006C00006C00006C00006C0000D2
S3150800A4606C00006C00006C00006C00006C00006C56
S3150800A47000006C00006C00006C00006C00006C00B2
S3150800A480006C00006C00006C00006C00006C0000A2
S3150800A4906C00006C00006C00006C00006C00006C26
S3150800A4A000006C00006C00006C00006C00006C0082
S3150800A4B0006C00006C00006C00006C00006C000072
S3150800A4C06C00006C00006C00006C00006C00006CF6
S3150800A4D000006C00006C00006C00006C00006C0052
S3150800A4E0006C00006C00006C00006C00006C000042
S3150800A4F06C00006C00006C00006C00006C00006CC6
S3150800A50000006C00006C00006C00006C00006C0021
S3150800A510006C00006C00006C00006C00006C000011
S3150800A5206C00006C00006C00006C00006C00006C95
S3150800A53000006C00006C00006C00006C00006C00F1
S3150800A540006C00006C00006C00006C00006C0000E1
S3150800A5506C00006C00006C00006C00006C00006C65
S3150800A56000006C00006C00006C00006C00006C00C1
S3150800A570006C00006C00006C00006C00006C0000B1
S3150800A5806C00006C00006C00006C00006C00006C35
S3150800A59000006C00006C00006C00006C00006C0091
S3150800A5A0006C00006C00006C00006C00006C000081
S3150800A5B06C00006C00006C00006C00006C00006C05
S3150800A5C000006C00006C00006C00006C00006C0061
S3150800A5D0006C00006C00006C00006C00006C000051
S3150800A5E06C00006C00006C00006C00006C00006CD5
S3150800A5F000006C00006C00006C00006C00006C0031
S3150800A600006C00006C00006C00006C00006C000020
S3150800A6106C00006C00006C00006C00006C00006CA4
S3150800A62000006C00006C00006C00006C00006C0000
S3150800A630006C00006C00006C00006C00006C0000F0
S3150800A6406C00006C00006C00006C00006C00006C74
S3150800A65000006C00006C00006C00006C00006C00D0
S3150800A660006C00006C00006C00006C00006C0000C0
S3150800A6706C00006C00006C00006C00006C00006C44
S3150800A68000006C00006C00006C00006C00006C00A0
S3150800A690006C00006C00006C00006C00006C000090
S3150800A6A06C00006C00006C00006C00006C00006C14
S3150800A6B000006C00006C00006C00006C00006C0070
S3150800A6C0006C00006C00006C00006C00006C000060
S3150800A6D06C00006C00006C00006C00006C00006CE4
S3150800A6E000006C00006C00006C00006C00006C0040
S3150800A6F0006C00006C00006C00006C00006C000030
S3150800A7006C00006C00006C00006C00006C00006CB3
S3150800A71000006C00006C00006C00006C00006C000F
S3150800A720006C00006C00006C00006C00006C0000FF
S3150800A7306C00006C00006C00006C00006C00006C83
S3150800A74000006C00006C00006C00006C00006C00DF
S3150800A750006C00006C00006C00006C00006C0000CF
S3150800A7606C00006C00006C00006C00006C00006C53
S3150800A77000006C00006C00006C00006C00006C00AF
S3150800A780006C00006C00006C00006C00006C00009F
S3150800A7906C00006C00006C00006C00006C00006C23
S3150800A7A000006C00006C00006C00006C00006C007F
S3150800A7B0006C00006C00006C00006C00006C00006F
S3150800A7C06C00006C00006C00006C00006C00006CF3
S3150800A7D000006C00006C00006C00006C00006C004F
S3150800A7E0006C00006C00006C00006C00006C00003F
S3150800A7F06C00006C00006C00006C00006C00006CC3
S3150800A80000006C00006C00006C00006C00006C001E
S3150800A810006C00006C00006C00006C00006C00000E
S3150800A8206C00006C00006C00006C00006C00006C92
S3150800A83000006C00006C00006C00006C00006C00EE
S3150800A840006C00006C00006C00006C00006C0000DE
S3150800A8506C00006C00006C00006C00006C00006C62
S3150800A86000006C00006C00006C00006C00006C00BE
S3150800A870006C00006C00006C00006C00006C0000AE
S3150800A8806C00006C00006C00006C00006C00006C32
S3150800A89000006C00006C00006C00006C00006C008E
S3150800A8A0006C00006C00006C00006C00006C00007E
S3150800A8B06C00006C00006C00006C00006C00006C02
S3150800A8C000006C00006C00006C00006C00006C005E
S3150800A8D0006C00006C00006C00006C00006C00004E
S3150800A8E06C00006C00006C00006C00006C00006CD2
S3150800A8F000006C00006C00006C00006C00006C002E
S3150800A900006C00006C00006C00006C00006C00001D
S3150800A9106C00006C00006C00006C00006C00006CA1
S3150800A92000006C00006C00006C00006C00006C00FD
S3150800A930006C00006C00006C00006C00006C0000ED
S3150800A9406C00006C00006C00006C00006C00006C71
S3150800A95000006C00006C00006C00006C00006C00CD
S3150800A960006C00006C00006C00006C00006C0000BD
S3150800A9706C00006C00006C00006C00006C00006C41
S3150800A98000006C00006C00006C00006C00006C009D
S3150800A990006C00006C00006C00006C00006C00008D
S3150800A9A06C00006C00006C00006C00006C00006C11
S3150800A9B000006C00006C00006C00006C00006C006D
S3150800A9C0006C00006C00006C00006C00006C00005D
S3150800A9D06C00006C00006C00006C00006C00006CE1
S3150800A9E000006C00006C00006C00006C00006C003D
S3150800A9F0006C00006C00006C00006C00006C00002D
S3150800AA006C00006C00006C00006C00006C00006CB0
S3150800AA1000006C00006C00006C00006C00006C000C
S3150800AA20006C00006C00006C00006C00006C0000FC
S3150800AA306C00006C00006C00006C00006C00006C80
S3150800AA4000006C00006C00006C00006C00006C00DC
S3150800AA50006C00006C00006C00006C00006C0000CC
S3150800AA606C00006C00006C00006C00006C00006C50
S3150800AA7000006C00006C00006C00006C00006C00AC
S3150800AA80006C00006C00006C00006C00006C00009C
S3150800AA906C00006C00006C00006C00006C00006C20
S3150800AAA000006C00006C00006C00006C00006C007C
S3150800AAB0006C00006C00006C00006C00006C00006C
S3150800AAC06C00006C00006C00006C00006C00006CF0
S3150800AAD000006C00006C00006C00006C00006C004C
S3150800AAE0006C00006C00006C00006C00006C00003C
S3150800AAF06C00006C00006C00006C00006C00006CC0
S3150800AB0004007000006C00007000006C04006C000B
S3150800AB10006C00006C00006C04006C00006C000007
S3150800AB206C00006C00006C00006C00006C00006C8F
S3150800AB3000006C00006C00006C00006C00006C00EB
S3150800AB40006C00006C00006C00006C04006C0000D7
S3150800AB506C00006C00006C04006C04007000006C53
S3150800AB6000006C04006C00007000006C04007000AB
S3150800AB70006C00006C00006C00006C00006C0000AB
S3150800AB806C00006C00006C00006C00006C00006C2F
S3150800AB9000006C00006C00006C00006C00006C1873
S3150800ABA0309C2C64CC04047000006C00006C00001F
S3150800ABB06C00006C00007000006C00006C00006CFB
S3150800ABC000006C00006C00006C00006C00006C005B
S3150800ABD0006C00006C00006C00006C00006C00004B
S3150800ABE06C00006C00006C04006C04006C080C78A7
S3150800ABF03880E84498FC204CB404007000006C00CF
S3150800AC00006C00007000006C04007000006C00000E
S3150800AC106C00006C00006C00006C00006C00006C9E
S3150800AC2000006C00006C00006C00006C00006C00FA
S3150800AC30006C00006C00006C00006C08087C347422
S3150800AC40DC3068CC1024941428943068D42C5CC862
S3150800AC5004047400006C00006C00006C04006C00B6
S3150800AC60006C00006C00006C00006C00006C0000BA
S3150800AC706C00006C00006C00006C00006C00006C3E
S3150800AC8000006C00006C00006C203CA81C3CA80C62
S3150800AC9010800C1484306CD4387CE42C68D0409036
S3150800ACA0F43470D800006C00007000006C00006C72
S3150800ACB000006C00007000006C00006C00006C0066
S3150800ACC0006C00006C00006C00006C00006C00005A
S3150800ACD06C00006C00006C00006C2C64CC3878E0CA
S3150800ACE010209018309C0404700400700400704012
S3150800ACF08CF02854BC04007004007000007000003A
S3150800AD006C00006C00006C00006C00006C00006CAD
S3150800AD1000006C00006C00006C00006C00006C0009
S3150800AD20006C00006C00006C00006C2044B0449875
S3150800AD30FC101C8C0400700C1C8414249414289891
S3150800AD404090F4080C7800006C00006C00006C0061
S3150800AD50006C00006C00006C00006C00006C0000C9
S3150800AD606C00006C00006C00006C00006C00006C4D
S3150800AD7000006C00006C00006C00006C0C14804431
S3150800AD8094FC2044B03470D82858C0142C98285401
S3150800AD90C02858C000006C00006C00006C00006CF5
S3150800ADA000006C00006C00006C00006C00006C0079
S3150800ADB0006C00006C00006C00006C00006C000069
S3150800ADC06C00006C00006C00006C00007000006CE9
S3150800ADD02C5CC81C3CA40404700C148018309C38E5
S3150800ADE080E8080C7804006C00006C00006C000019
S3150800ADF06C00006C00006C00006C00006C00006CBD
S3150800AE0000006C00006C00006C00006C00006C0018
S3150800AE10006C00006C00006C00006C00006C000008
S3150800AE2070040C781428942040AC1428981C38A474
S3150800AE30101C8800006C00006C00006C00006C049C
S3150800AE40006C00006C00006C04006C00006C0000D4
S3150800AE506C00006C00006C00006C00006C00006C5C
S3150800AE6000006C00006C00006C00006C00006C00B8
S3150800AE70006C00006C04007004007000006C000098
S3150800AE806C00006C00006C00006C00006C00006C2C
S3150800AE9000007000006C00006C00006C00006C0084
S3150800AEA0006C00006C00006C00006C00006C000078
S3150800AEB06C00006C00006C00006C00006C00006CFC
S3150800AEC000006C00006C00006C00006C0000700054
S3150800AED0007000007000007000006C00006C00003C
S3150800AEE06C00006C00006C00006C00006C00006CCC
S3150800AEF000006C00006C00006C00006C00006C0028
S3150800AF00006C00006C00006C00006C00006C000017
S3150800AF106C00006C04006C00006C00006C00006C97
S3150800AF201C40A8080C7C00006C00006C00006C003B
S3150800AF30006C00006C00006C00006C00006C0000E7
S3150800AF406C00006C00006C00006C00006C00006C6B
S3150800AF5000006C00006C00006C00006C00006C00C7
S3150800AF60006C00006C00006C00006C00006C0400B3
S3150800AF70702044B02C64CC00006C00006C00006C9F
S3150800AF8004006C04007004007000006C00006C0083
S3150800AF90006C00006C00006C00006C00006C000087
S3150800AFA06C00006C00006C00006C00006C00006C0B
S3150800AFB00400703064CC408CF4306CD4080C7804EF
S3150800AFC004741C40A83068D400006C00006C0400AF
S3150800AFD06C00006C04007000006C00006C00006CD3
S3150800AFE000006C00006C00006C00006C00006C0037
S3150800AFF0006C00006C00006C00006C00006C000027
S3150800B0006C00006C0808781834A0408CF41C40AC1E
S3150800B0103474DC1C3CA82454C0204CB400006C10CA
S3150800B0201C8800006C00006C00006C0000700000BA
S3150800B0306C00006C00006C00006C00006C00006C7A
S3150800B04000006C00006C00006C00006C00006C00D6
S3150800B050006C00006C00006C0C1888080C78102432
S3150800B060944088F01C3CAC2450B84094F83068D41E
S3150800B0700C188400006C00006C00006C00006C006A
S3150800B080006C00006C00006C00006C00006C000096
S3150800B0906C00006C00006C00006C00006C00006C1A
S3150800B0A000006C0400700C18842044B03068D0147A
S3150800B0B02494285CC8204CB01C40A82044B02854CE
S3150800B0C0BC04007000006C00006C00006C0000708E
S3150800B0D000007000006C00006C00006C00006C0042
S3150800B0E0006C00006C00006C00006C00006C000036
S3150800B0F06C00006C0808744090F44494FC245CC40A
S3150800B1001428981C3CA4306CD41C38A42048B008D9
S3150800B110107C00006C00006C04007000006C0000DD
S3150800B1206C00006C00006C00006C00006C00006C89
S3150800B13000006C00006C00006C00006C00006C00E5
S3150800B140006C00006C0400700C10801020882048E9
S3150800B150B00C147C142894080C782448B82044B001
S3150800B16000006C04007000006C00006C00007000A9
S3150800B170006C00006C00006C00006C00006C0000A5
S3150800B1806C00006C00006C00006C00006C00006C29
S3150800B19000006C00006C00006C1834A42858C01C11
S3150800B1A03CA8080878081080142894387CE40C1405
S3150800B1B08400007000006C00006C04006C00006CD9
S3150800B1C000006C00006C00006C00006C00006C0055
S3150800B1D0006C00006C00006C00006C00006C000045
S3150800B1E06C00006C00006C0400702044B03878E0F5
S3150800B1F00C18882048B02C5CC82454BC2044AC00E9
S3150800B200006C00006C00006C00006C00006C000014
S3150800B2106C00006C00006C00006C00006C00006C98
S3150800B22000006C00006C00006C00006C00006C00F4
S3150800B230006C00006C00006C00006C00006C0000E4
S3150800B2406C04007000006C00006C00007000006C5C
S3150800B25000006C00006C00006C00006C00006C00C4
S3150800B260006C00006C00006C00006C00006C0000B4
S3150800B2706C00006C00006C00006C00006C00006C38
S3150800B28000006C00006C00006C00006C00006C0094
S3150800B290006C00007000006C00007000006C040474
S3150800B2A07400007000006C00006C04006C00006CF8
S3150800B2B000006C00006C00006C00006C00006C0064
S3150800B2C0006C00006C00006C00006C00006C000054
S3150800B2D06C00006C00006C00006C00006C04006CD4
S3150800B2E004006C00006C00006C04007000006C0C1C
S3150800B2F018883068D000007004006C00006C0000EC
S3150800B3006C00007000006C00006C00006C00006CA3
S3150800B31000006C00006C00006C00006C00006C0003
S3150800B320006C00006C00006C00006C00006C0000F3
S3150800B3306C00006C2454BC14309C00006C00007037
S3150800B34000006C3874DC04006C00006C04006C04AB
S3150800B350007000006C00006C00006C00006C0000BF
S3150800B3606C00006C00006C00006C00006C00006C47
S3150800B37000006C00006C00006C00006C00006C00A3
S3150800B380006C1424904094F83878E018349C3C8873
S3150800B390EC3070D82C64CC00006C04006C00007093
S3150800B3A000006C00006C00006C00006C00006C0073
S3150800B3B0006C00006C00006C00006C00006C000063
S3150800B3C06C00006C00006C00006C00006C00006CE7
S3150800B3D0142894347CE42C5CC000006C0C14802483
S3150800B3E050BC1C3CA42C5CC800006C00006C00001F
S3150800B3F06C00006C00006C00006C00006C00006CB7
S3150800B40000006C00006C00006C00006C00006C0012
S3150800B410006C00006C00006C00006C00006C0408F6
S3150800B420741428941428944090F82C5CC80C1C8832
S3150800B4302C60C83470D8285CC41834A00404700082
S3150800B440006C00006C00006C00006C00006C0000D2
S3150800B4506C00006C00006C00006C00006C00006C56
S3150800B46000006C00006C00006C00006C00006C04AE
S3150800B47008742044B04494FC4494FC2048B4040066
S3150800B4806C2854C02858BC4490F84498FC2C68D0C2
S3150800B49000006C00006C00006C00006C00006C0082
S3150800B4A0006C00006C00006C00006C00006C000072
S3150800B4B06C00006C00006C00006C00006C00006CF6
S3150800B4C00C1C8C306CD43878E03068D02454BC38E6
S3150800B4D080E44090F42854BC3068D01834A404089A
S3150800B4E07400006C00006C04007000006C00006CB6
S3150800B4F000006C00006C00006C00006C00006C0022
S3150800B500006C00006C00006C00006C00006C000011
S3150800B5106C0400701834A01C38A4285CC008107C81
S3150800B5201838A40808781C3CA8346CD404007000A9
S3150800B530006C00006C00007000006C00006C0000DD
S3150800B5406C00006C00006C00006C00006C00006C65
S3150800B55000006C00006C00006C00006C00006C00C1
S3150800B560006C0C1888182C9808107C2C64CC0000E9
S3150800B5706C1024903070D81028942858C400006C99
S3150800B58004006C00006C00006C00006C00006C008D
S3150800B590006C00006C00006C00006C00006C000081
S3150800B5A06C00006C00006C00006C00006C00006C05
S3150800B5B000006C080C7800006C0C18843474D800F1
S3150800B5C0006C2C5CC81C38A41024902C60C80000A1
S3150800B5D06C00006C00006C00007000006C00006CD1
S3150800B5E000006C00006C00006C00006C00006C0031
S3150800B5F0006C00006C00006C00006C00006C000021
S3150800B6006C00006C04007000007000006C0C18845C
S3150800B61004006C00006C0400700C1C8C1834A0002C
S3150800B620006C00006C00006C00006C00006C0000F0
S3150800B6306C04006C00006C00006C00006C00006C70
S3150800B64000006C00006C00006C00006C00006C00D0
S3150800B650006C00006C00006C00006C0000700400B8
S3150800B6607000006C04006C00006C04006C00006C38
S3150800B67000006C00006C00006C00006C00006C00A0
S3150800B680006C04006C00006C00006C00006C00008C
S3150800B6906C00006C00006C00006C00006C00006C14
S3150800B6A000006C00006C00006C00006C00006C0070
S3150800B6B0006C04006C00006C2C5CC8080C7C000054
S3150800B6C06C00006C00006C00006C00006C00006CE4
S3150800B6D000006C00006C00006C00006C00006C0040
S3150800B6E0006C00006C00006C00006C00006C000030
S3150800B6F06C00006C00006C00006C00006C10249458
S3150800B7002040AC00006C00006C3470D814249400FF
S3150800B710006C00006C00006C00006C04006C0000FB
S3150800B7206C00006C00006C00006C00006C00006C83
S3150800B73000006C00006C00006C00006C00006C00DF
S3150800B740006C00006C00006C00007000006C080CB7
S3150800B7507C1C40A800006C00006C3470D82858C0C7
S3150800B760080C7804006C00006C04006C00006C0087
S3150800B770006C00006C00006C00006C00006C00009F
S3150800B7806C00006C00006C00006C00006C00006C23
S3150800B79000006C00006C00006C00006C00006C1867
S3150800B7A0309C3C88EC1834A02C64CC4498FC3C882B
S3150800B7B0EC14289800007004007004006C00006CFB
S3150800B7C000006C00006C00006C00006C00006C004F
S3150800B7D0006C00006C00006C00006C00006C00003F
S3150800B7E06C00006C00006C00006C08107C2858C0C7
S3150800B7F04098FC4494FC2450B8142C983064CC141B
S3150800B8002C98080C780C188800006C00006C000056
S3150800B8106C00006C00006C00006C00006C00006C92
S3150800B82000006C00006C00006C00006C00006C00EE
S3150800B830006C00006C00006C00006C1C40A83C8882
S3150800B840EC3474DC2450B8080C780C107C3070D8B2
S3150800B8503474D83874DC14249400006C00006C002E
S3150800B860006C00006C04006C00006C00006C0000AA
S3150800B8706C00006C00006C00006C00006C00006C32
S3150800B88000006C00006C00006C00006C00006C008E
S3150800B890006C1428982858C410208C3474DC0C10BA
S3150800B8A07C3068D01C3CA810249000006C04007002
S3150800B8B000007004007004006C00006C00006C004E
S3150800B8C0006C00006C00006C00006C00006C00004E
S3150800B8D06C00006C00006C00006C00006C00006CD2
S3150800B8E0182C982C58C41834A40C18840810802CCA
S3150800B8F068D02040AC1C3CA810208C0400700000C6
S3150800B9006C00006C00006C00006C00006C00006CA1
S3150800B91000006C00006C00006C00006C00006C00FD
S3150800B920006C00006C00006C00006C00006C182CA9
S3150800B9309C285CC01024901834A000006C0C188455
S3150800B940203CAC2854BC306CD410208C000070000D
S3150800B950006C00006C00006C00006C00006C0000BD
S3150800B9606C00006C00006C00006C00006C00006C41
S3150800B97000006C00006C00006C00006C00006C009D
S3150800B980006C101C8818309C1830A000006C0C182D
S3150800B9908800006C00006C2450B8142C9800006CC9
S3150800B9A000006C00006C00006C00006C00006C006D
S3150800B9B0006C00006C00006C00006C00006C00005D
S3150800B9C06C00006C00006C00006C00006C00006CE1
S3150800B9D000006C00006C00006C00006C00006C003D
S3150800B9E0006C04006C04007000006C00006C000021
S3150800B9F06C04006C00006C00006C00006C00006CAD
S3150800BA0000006C00006C00006C00006C00006C000C
S3150800BA10006C00006C00006C00006C00006C0000FC
S3150800BA206C00006C00006C00006C00006C00006C80
S3150800BA3000006C00006C00006C00006C00006C00DC
S3150800BA40006C00006C00006C00006C00006C0000CC
S3150800BA506C00006C00006C00006C00006C00006C50
S3150800BA6000006C00006C00006C00006C00006C00AC
S3150800BA70006C00006C00006C00006C00006C00009C
S3150800BA806C00006C00006C00006C00006C00006C20
S3150800BA9000006C00006C00006C00006C00006C007C
S3150800BAA0006C00006C00006C00006C00006C00006C
S3150800BAB06C00006C00006C00006C00006C00006CF0
S3150800BAC000006C00006C00006C00006C00006C004C
S3150800BAD0006C00006C00006C00006C00006C00003C
S3150800BAE06C00006C00006C00006C00006C00006CC0
S3150800BAF000006C00006C00006C00006C00006C001C
S3150800BB00006C00006C00006C00006C00006C00000B
S3150800BB106C00006C00006C00006C00006C00006C8F
S3150800BB2000006C00006C00006C00006C00006C00EB
S3150800BB30006C00006C00006C00006C00006C0000DB
S3150800BB406C00006C00006C00006C00006C00006C5F
S3150800BB5000006C00006C00006C00006C00006C00BB
S3150800BB60006C00006C00006C00006C00006C0000AB
S3150800BB706C00006C00006C00006C00006C00006C2F
S3150800BB8000006C00006C00006C00006C00006C008B
S3150800BB90006C00006C00006C00006C00006C00007B
S3150800BBA06C00006C00006C00006C00006C00006CFF
S3150800BBB000006C00006C00006C00006C00006C005B
S3150800BBC0006C00006C00006C00006C00006C00004B
S3150800BBD06C00006C00006C00006C00006C00006CCF
S3150800BBE000006C00006C00006C00006C00006C002B
S3150800BBF0006C00006C00006C00006C00006C00001B
S3150800BC006C00006C00006C00006C00006C00006C9E
S3150800BC1000006C00006C00006C00006C00006C00FA
S3150800BC20006C00006C00006C00006C00006C0000EA
S3150800BC306C00006C00006C00006C00006C00006C6E
S3150800BC4000006C00006C00006C00006C00006C00CA
S3150800BC50006C00006C00006C00006C00006C0000BA
S3150800BC606C00006C00006C00006C00006C00006C3E
S3150800BC7000006C00006C00006C00006C00006C009A
S3150800BC80006C00006C00006C00006C00006C00008A
S3150800BC906C00006C00006C00006C00006C00006C0E
S3150800BCA000006C00006C00006C00006C00006C006A
S3150800BCB0006C00006C00006C00006C00006C00005A
S3150800BCC06C00006C00006C00006C00006C00006CDE
S3150800BCD000006C00006C00006C00006C00006C003A
S3150800BCE0006C00006C00006C00006C00006C00002A
S3150800BCF06C00006C00006C00006C00006C00006CAE
S3150800BD0000006C00006C00006C00006C00006C0009
S3150800BD10006C00006C00006C00006C00006C0000F9
S3150800BD206C00006C00006C00006C00006C00006C7D
S3150800BD3000006C00006C00006C00006C00006C00D9
S3150800BD40006C00006C00006C00006C00006C0000C9
S3150800BD506C00006C00006C00006C00006C00006C4D
S3150800BD6000006C00006C00006C00006C00006C00A9
S3150800BD70006C00006C00006C00006C00006C000099
S3150800BD806C00006C00006C00006C00006C00006C1D
S3150800BD9000006C00006C00006C00006C00006C0079
S3150800BDA0006C00006C00006C00006C00006C000069
S3150800BDB06C00006C00006C00006C00006C00006CED
S3150800BDC000006C00006C00006C00006C00006C0049
S3150800BDD0006C00006C00006C00006C00006C000039
S3150800BDE06C00006C00006C00006C00006C00006CBD
S3150800BDF000006C00006C00006C00006C00006C0019
S3150800BE00006C00006C00006C00006C00006C000008
S3150800BE106C00006C00006C00006C00006C00006C8C
S3150800BE2000006C00006C00006C00006C00006C00E8
S3150800BE30006C00006C00006C00006C00006C0000D8
S3150800BE406C00006C00006C00006C00006C00006C5C
S3150800BE5000006C00006C00006C00006C00006C00B8
S3150800BE60006C00006C00006C00006C00006C0000A8
S3150800BE706C00006C00006C00006C00006C00006C2C
S3150800BE8000006C00006C00006C00006C00006C0088
S3150800BE90006C00006C00006C00006C00006C000078
S3150800BEA06C00006C00006C00006C00006C00006CFC
S3150800BEB000006C00006C00006C00006C00006C0058
S3150800BEC0006C00006C00006C00006C00006C000048
S3150800BED06C00006C00006C00006C00006C00006CCC
S3150800BEE000006C00006C00006C00006C00006C0028
S3150800BEF0006C00006C00006C00006C00006C000018
S3150800BF006C00006C00006C00006C00006C00006C9B
S3150800BF1000006C00006C00006C00006C00006C00F7
S3150800BF20006C00006C00006C00006C00006C0000E7
S3150800BF306C00006C00006C00006C00006C00006C6B
S3150800BF4000006C00006C00006C00006C00006C00C7
S3150800BF50006C00006C00006C00006C00006C0000B7
S3150800BF606C00006C00006C00006C00006C00006C3B
S3150800BF7000006C00006C00006C00006C00006C0097
S3150800BF80006C00006C00006C00006C00006C000087
S3150800BF906C00006C00006C00006C00006C00006C0B
S3150800BFA000006C00006C00006C00006C00006C0067
S3150800BFB0006C00006C00006C00006C00006C000057
S3150800BFC06C00006C00006C00006C00006C00006CDB
S3150800BFD000006C00006C00006C00006C00006C0037
S3150800BFE0006C00006C00006C00006C00006C000027
S3150800BFF06C00006C00006C00006C00006C00006CAB
S3150800C00000006C00006C00006C00006C00006C0006
S3150800C010006C00006C00006C00006C00006C0000F6
S3150800C0206C00006C00006C00006C00006C00006C7A
S3150800C03000006C00006C00006C00006C00006C00D6
S3150800C040006C00006C00006C00006C00006C0000C6
S3150800C0506C00006C00006C00006C00006C00006C4A
S3150800C06000006C00006C00006C00006C00006C00A6
S3150800C070006C00006C00006C00006C00006C000096
S3150800C0806C00006C00006C00006C00006C00006C1A
S3150800C09000006C00006C00006C00006C00006C0076
S3150800C0A0006C00006C00006C00006C00006C000066
S3150800C0B06C00006C00006C00006C00006C00006CEA
S3150800C0C000006C00006C00006C00006C00006C0046
S3150800C0D0006C00006C00006C00006C00006C000036
S3150800C0E06C00006C00006C00006C00006C00006CBA
S3150800C0F000006C00006C00006C00006C00006C0016
S3150800C100006C00006C00006C00006C00006C000005
S3150800C1106C00006C00006C00006C00006C00006C89
S3150800C12000006C00006C00006C00006C00006C00E5
S3150800C130006C00006C00006C00006C00006C0000D5
S3150800C1406C00006C00006C00006C00006C00006C59
S3150800C15000006C00006C00006C00006C00006C00B5
S3150800C160006C00006C00006C00006C00006C0000A5
S3150800C1706C00006C00006C00006C00006C00006C29
S3150800C18000006C00006C00006C00006C00006C0085
S3150800C190006C00006C00006C00006C00006C000075
S3150800C1A06C00006C00006C00006C00006C00006CF9
S3150800C1B000006C00006C00006C00006C00006C0055
S3150800C1C0006C00006C00006C00006C00006C000045
S3150800C1D06C00006C00006C00006C00006C00006CC9
S3150800C1E000006C00006C00006C00006C00006C0025
S3150800C1F0006C00006C00006C00006C00006C000015
S3150800C2006C00006C00006C00006C00006C00006C98
S3150800C21000006C00006C00006C00006C00006C00F4
S3150800C220006C00006C00006C00006C00006C0000E4
S3150800C2306C00006C00006C00006C00006C00006C68
S3150800C24000006C00006C00006C00006C00006C00C4
S3150800C250006C00006C00006C00006C00006C0000B4
S3150800C2606C00006C00006C00006C00006C00006C38
S3150800C27000006C00006C00006C00006C00006C0094
S3150800C280006C00006C00006C00006C00006C000084
S3150800C2906C00006C00006C00006C00006C00006C08
S3150800C2A000006C00006C00006C00006C00006C0064
S3150800C2B0006C00006C00006C00006C00006C000054
S3150800C2C06C00006C00006C00006C00006C00006CD8
S3150800C2D000006C00006C00006C00006C00006C0034
S3150800C2E0006C00006C00006C00006C00006C000024
S3150800C2F06C00006C00006C00006C00006C00006CA8
S3150800C30000006C00006C00006C00006C00006C0003
S3150800C310006C00006C00006C00006C00006C0000F3
S3150800C3206C00006C00006C00006C00006C00006C77
S3150800C33000006C00006C00006C00006C00006C00D3
S3150800C340006C00006C00006C00006C00006C0000C3
S3150800C3506C00006C00006C00006C00006C00006C47
S3150800C36000006C00006C00006C00006C00006C00A3
S3150800C370006C00006C00006C00006C00006C000093
S3150800C3806C00006C00006C00006C00006C00006C17
S3150800C39000006C00006C00006C00006C00006C0073
S3150800C3A0006C00006C00006C00006C00006C000063
S3150800C3B06C00006C00006C00006C00006C00006CE7
S3150800C3C000006C00006C00006C00006C00006C0043
S3150800C3D0006C00006C00006C00006C00006C000033
S3150800C3E06C00006C00006C00006C00006C00006CB7
S3150800C3F000006C00006C00006C00006C00006C0013
S3150800C400006C00006C00006C00006C00006C000002
S3150800C4106C00006C00006C00006C00006C00006C86
S3150800C42000006C00006C00006C00006C00006C00E2
S3150800C430006C00006C00006C00006C00006C0000D2
S3150800C4406C00006C00006C00006C00006C00006C56
S3150800C45000006C00006C00006C00006C00006C00B2
S3150800C460006C00006C00006C00006C00006C0000A2
S3150800C4706C00006C00006C00006C80BCFCA8D8FC4A
S3150800C480B0DCFCB8E0FCBCE4FCC4E8FCCCECFCD4B6
S3150800C490F0FCD8F4FCD0F0FCCCECFCBCFCFCA0D442
S3150800C4A0FCA8D8FCB0DCFCB8E0FCBCE4FCC4E8FCA6
S3150800C4B0CCECFCD4F0FCD8F4FCD0F0FCC8ECFCC006
S3150800C4C0E8FCA0D4FCA8D8FCB0DCFCB4E0FCBCE4D6
S3150800C4D0FCC4E8FCCCECFCD4F0FCD8F4FCD0F0FCB2
S3150800C4E0C8ECFCC0E8FCA0D4FCA8D8FCB0DCFCB8BE
S3150800C4F0E0FCBCE4FCC4E8FCCCECFCD4F0FCD8F4CE
S3150800C500FCD0F0FCC8ECFCC0E8FCA0D4FCA8D8FC25
S3150800C510B0DCFCB8E0FCBCE4FCC4E8FCCCECFCD425
S3150800C520F0FCD8F4FCD0F0FCC8ECFCC0E8FCA0D4C5
S3150800C530FCA8D8FCB0DCFCB8E0FCBCE4FCC4E8FC15
S3150800C540CCECFCD4F0FCD8F4FCD0F0FCC8ECFCC075
S3150800C550E8FCA0D4FCA8D8FCB0DCFCB4E0FCBCE445
S3150800C560FCC4E8FCCCECFCD4F0FCD8F4FCD0F0FC21
S3150800C570C8ECFCC0E8FCA0D4FCA8D8FCB0DCFCB431
S3150800C580E0FCBCE4FCC4E8FCCCECFCD4F0FCD8F43D
S3150800C590FCD0F0FCC8ECFCC0E8FCA0D4FCA8D8FC95
S3150800C5A0B0DCFCB8E0FCBCE4FCC4E8FCCCECFCD495
S3150800C5B0F0FCD8F4FCD0F0FCC8ECFCC0E8FCA0D435
S3150800C5C0FCA8D8FCB0DCFCB8E0FCBCE4FCC4E8FC85
S3150800C5D0CCECFCD4F0FCD8F4FCD0F0FCC8ECFCC0E5
S3150800C5E0E8FCA0D4FCA8D8FCB0DCFCB4E0FCBCE4B5
S3150800C5F0FCC4E8FCCCECFCD4F0FCD8F4FCD0F0FC91
S3150800C600C8ECFCC0E8FCA0D4FCA8D8FCB0DCFCB89C
S3150800C610E0FCBCE4FCC4E8FCCCECFCD4F0FCD8F4AC
S3150800C620FCD0F0FCC8ECFCC0E8FCA0D4FCA8D8FC04
S3150800C630B0DCFCB8E0FCBCE4FCC4E8FCCCECFCD404
S3150800C640F0FCD8F4FCD0F0FCC8ECFCC0E8FCA0D4A4
S3150800C650FCA8D8FCB0DCFCB8E0FCBCE4FCC4E8FCF4
S3150800C660CCECFCD4F0FCD8F4FCD0F0FCC8ECFCC054
S3150800C670E8FCA0D4FCA8D8FCB0DCFCB4E0FCBCE424
S3150800C680FCC4E8FCCCECFCD4F0FCD8F4FCD0F0FC00
S3150800C690C8ECFCC0E8FCA0D4FCA8D8FCB0DCFCB410
S3150800C6A0E0FCBCE4FCC4E8FCCCECFCD4F0FCD8F41C
S3150800C6B0FCD0F0FCC8ECFCC0E8FCA0D4FCA8D8FC74
S3150800C6C0B0DCFCB8E0FCBCE4FCC4E8FCCCECFCD474
S3150800C6D0F0FCD8F4FCD0F0FCC8ECFCC0E8FCA0D414
S3150800C6E0FCA8D8FCB0DCFCB8E0FCBCE4FCC4E8FC64
S3150800C6F0CCECFCD4F0FCD8F4FCD0F0FCC8ECFCC0C4
S3150800C700E8FCA0D4FCA8D8FCB0DCFCB4E0FCBCE493
S3150800C710FCC4E8FCCCECFCD4F0FCD8F4FCD0F0FC6F
S3150800C720C8ECFCC0E8FCA0D4FCA8D8FCB0DCFCB87B
S3150800C730E0FCBCE4FCC4E8FCCCECFCD4F0FCD8F48B
S3150800C740FCD0F0FCC8ECFCC0E8FCA0D4FCA8D8FCE3
S3150800C750B0DCFCB8E0FCBCE4FCC4E8FCCCECFCD4E3
S3150800C760F0FCD8F4FCD0F0FCC8ECFCC0E8FCA0D483
S3150800C770FCA8D8FCB0DCFCB8E0FCBCE4FCC4E8FCD3
S3150800C780CCECFCD4F0FCD8F4FCD0F0FCC8ECFCC033
S3150800C790E8FCA0D4FCA8D8FCB0DCFCB4E0FCBCE403
S3150800C7A0FCC4E8FCCCECFCD4F0FCD8F4FCD0F0FCDF
S3150800C7B0C8ECFCC0E8FCA0D4FCA8D8FCB0DCFCB4EF
S3150800C7C0E0FCBCE4FCC4E8FCCCECFCD4F0FCD8F4FB
S3150800C7D0FCD0F0FCC8ECFCC0E8FCA0D4FCA8D8FC53
S3150800C7E0B0DCFCB8E0FCBCE4FCC4E8FCCCECFCD453
S3150800C7F0F0FCD8F4FCD0F0FCC8ECFCC0E8FCA0D4F3
S3150800C800FCA8D8FCB0DCFCB8E0FCBCE4FCC4E8FC42
S3150800C810CCECFCD4F0FCD8F4FCD0F0FCC8ECFCC0A2
S3150800C820E8FCA0D4FCA8D8FCB0DCFCB4E0FCBCE472
S3150800C830FCC4E8FCCCECFCD4F0FCD8F4FCD0F0FC4E
S3150800C840C8ECFCC0E8FCA0D4FCA8D8FCB0DCFCB85A
S3150800C850E0FCBCE4FCC4E8FCCCECFCD4F0FCD8F46A
S3150800C860FCD0F0FCC8ECFCC0E8FCA0D4FCA8D8FCC2
S3150800C870B0DCFCB8E0FCBCE4FCC4E8FCCCECFCD4C2
S3150800C880F0FCD8F4FCD0F0FCC8ECFCC0E8FCA0D462
S3150800C890FCA8D8FCB0DCFCB8E0FCBCE4FCC4E8FCB2
S3150800C8A0CCECFCD4F0FCD8F4FCD0F0FCC8ECFCC012
S3150800C8B0E8FCA0D4FCA8D8FCB0DCFCB4E0FCBCE4E2
S3150800C8C0FCC4E8FCCCECFCD4F0FCD8F4FCD0F0FCBE
S3150800C8D0C8ECFCC0E8FCA0D4FCA8D8FCB0DCFCB4CE
S3150800C8E0E0FCBCE4FCC4E8FCCCECFCD4F0FCD8F4DA
S3150800C8F0FCD0F0FCC8ECFCC0E8FCA0D4FCA8D8FC32
S3150800C900B0DCFCB8E0FCBCE4FCC4E8FCCCECFCD431
S3150800C910F0FCD8F4FCD0F0FCC8ECFCC0E8FCA0D4D1
S3150800C920FCA8D8FCB0DCFCB8E0FCBCE4FCC4E8FC21
S3150800C930CCECFCD4F0FCD8F4FCD0F0FCC8ECFCC081
S3150800C940E8FCA0D4FCA8D8FCB0DCFCB4E0FCBCE451
S3150800C950FCC4E8FCCCECFCD4F0FCD8F4FCD0F0FC2D
S3150800C960C8ECFCC0E8FCA0D4FCA8D8FCB0DCFCB839
S3150800C970E0FCBCE4FCC4E8FCCCECFCD4F0FCD8F449
S3150800C980FCD0F0FCC8ECFCC0E8FCA0D4FCA8D8FCA1
S3150800C990B0DCFCB8E0FCBCE4FCC4E8FCCCECFCD4A1
S3150800C9A0F0FCD8F4FCD0F0FCC8ECFCC0E8FCA0D441
S3150800C9B0FCA8D8FCB0DCFCB8E0FCBCE4FCC4E8FC91
S3150800C9C0CCECFCD4F0FCD8F4FCD0F0FCC8ECFCC0F1
S3150800C9D0E8FCA0D4FCA8D8FCB0DCFCB4E0FCBCE4C1
S3150800C9E0FCC4E8FCCCECFCD4F0FCD8F4FCD0F0FC9D
S3150800C9F0C8ECFCC0E8FCA0D4FCA8D8FCB0DCFCB4AD
S3150800CA00E0FCBCE4FCC4E8FCCCECFCD4F0FCD8F4B8
S3150800CA10FCD0F0FCC8ECFCC0E8FCA0D4FCA8D8FC10
S3150800CA20B0DCFCB8E0FCBCE4FCC4E8FCCCECFCD410
S3150800CA30F0FCD8F4FCD0F0FCC8ECFCC0E8FCE8A894
S3150800CA4060ECB070ECB87CF0C088F4C894F4D0A45C
S3150800CA50F8D8B0FCDCBCFCE4C4FCDCB8FCD4A8FC0C
S3150800CA60D098ECA858F0B068F0B874F4C084F4C84C
S3150800CA7090F8CCA0F8D4ACFCDCBCFCE4C4FCDCB478
S3150800CA80FCD4A4FCD094ACACA8B8B8B4C4C4C0D088
S3150800CA90D0CCDCDCD8E8E8E8F4F4F0FCFCFCFCFCE0
S3150800CAA0FCFCF8F8F4F4F4F0F0ECA8ACACB4B8B8C4
S3150800CAB0C0C4C4D0D0D0DCDCDCE8E8E8F4F4F4FC8C
S3150800CAC0FCFCFCFCFCF8F8F8F4F4F4F0F0F0A8AC84
S3150800CAD0ACB4B8B8C0C4C4D0D0D0DCDCDCE8E8E874
S3150800CAE0F4F4F4FCFCFCFCFCFCF8F8F8F4F4F4F0C0
S3150800CAF0F0F0A8ACACB4B8B8C4C4C4D0D0D0DCDCB0
S3150800CB00DCE8E8E8F4F4F4FCFCFCFCFCFCF8F8F8D7
S3150800CB10F4F4F4F0F0F0A8ACACB4B8B8C4C4C4D01B
S3150800CB20D0D0DCDCDCE8E8E8F4F4F4FCFCFCFCFC43
S3150800CB30FCF8F8F8F4F4F4F0F0F0A8ACACB4B8B833
S3150800CB40C4C4C4D0D0D0DCDCDCE8E8E8F4F4F4FCF7
S3150800CB50FCFCFCFCFCF8F8F8F4F4F4F0F0F0A8ACF3
S3150800CB60ACB4B8B8C4C4C4D0D0D0DCDCDCE8E8E8DF
S3150800CB70F4F4F4FCFCFCFCFCFCF8F8F8F4F4F4F02F
S3150800CB80F0F0A8ACACB4B8B8C4C4C4D0D0D0DCDC1F
S3150800CB90DCE8E8E8F4F4F4FCFCFCFCFCFCF8F8F847
S3150800CBA0F4F4F4F0F0F0A8ACACB4B8B8C4C4C4D08B
S3150800CBB0D0D0DCDCDCE8E8E8F4F4F4FCFCFCFCFCB3
S3150800CBC0FCF8F8F8F4F4F4F0F0F0A8ACACB4B8B8A3
S3150800CBD0C0C4C4D0D0D0DCDCDCE8E8E8F4F4F4FC6B
S3150800CBE0FCFCFCFCFCF8F8F8F4F4F4F0F0F0A8AC63
S3150800CBF0ACB4B8B8C0C4C4D0D0D0DCDCDCE8E8E853
S3150800CC00F4F4F4FCFCFCFCFCFCF8F8F8F4F4F4F09E
S3150800CC10F0F0A8ACACB4B8B8C4C4C4D0D0D0DCDC8E
S3150800CC20DCE8E8E8F4F4F4FCFCFCFCFCFCF8F8F8B6
S3150800CC30F4F4F4F0F0F0A8ACACB4B8B8C4C4C4D0FA
S3150800CC40D0D0DCDCDCE8E8E8F4F4F4FCFCFCFCFC22
S3150800CC50FCF8F8F8F4F4F4F0F0F0A8ACACB4B8B812
S3150800CC60C4C4C4D0D0D0DCDCDCE8E8E8F4F4F4FCD6
S3150800CC70FCFCFCFCFCF8F8F8F4F4F4F0F0F0A8ACD2
S3150800CC80ACB4B8B8C4C4C4D0D0D0DCDCDCE8E8E8BE
S3150800CC90F4F4F4FCFCFCFCFCFCF8F8F8F4F4F4F00E
S3150800CCA0F0F0A8ACACB4B8B8C4C4C4D0D0D0DCDCFE
S3150800CCB0DCE8E8E8F4F4F4FCFCFCFCFCFCF8F8F826
S3150800CCC0F4F4F4F0F0F0A8ACACB4B8B8C4C4C4D06A
S3150800CCD0D0D0DCDCDCE8E8E8F4F4F4FCFCFCFCFC92
S3150800CCE0FCF8F8F8F4F4F4F0F0F0A8ACACB4B8B882
S3150800CCF0C0C4C4D0D0D0DCDCDCE8E8E8F4F4F4FC4A
S3150800CD00FCFCFCFCFCF8F8F8F4F4F4F0F0F0A8AC41
S3150800CD10ACB4B8B8C0C4C4D0D0D0DCDCDCE8E8E831
S3150800CD20F4F4F4FCFCFCFCFCFCF8F8F8F4F4F4F07D
S3150800CD30F0F0A8ACACB4B8B8C4C4C4D0D0D0DCDC6D
S3150800CD40DCE8E8E8F4F4F4FCFCFCFCFCFCF8F8F895
S3150800CD50F4F4F4F0F0F0A8ACACB4B8B8C4C4C4D0D9
S3150800CD60D0D0DCDCDCE8E8E8F4F4F4FCFCFCFCFC01
S3150800CD70FCF8F8F8F4F4F4F0F0F0A8ACACB4B8B8F1
S3150800CD80C4C4C4D0D0D0DCDCDCE8E8E8F4F4F4FCB5
S3150800CD90FCFCFCFCFCF8F8F8F4F4F4F0F0F0A8ACB1
S3150800CDA0ACB4B8B8C4C4C4D0D0D0DCDCDCE8E8E89D
S3150800CDB0F4F4F4FCFCFCFCFCFCF8F8F8F4F4F4F0ED
S3150800CDC0F0F0A8ACACB4B8B8C4C4C4D0D0D0DCDCDD
S3150800CDD0DCE8E8E8F4F4F4FCFCFCFCFCFCF8F8F805
S3150800CDE0F4F4F4F0F0F0A8ACACB4B8B8C4C4C4D049
S3150800CDF0D0D0DCDCDCE8E8E8F4F4F4FCFCFCFCFC71
S3150800CE00FCF8F8F8F4F4F4F0F0F0A8ACACB4B8B860
S3150800CE10C0C4C4D0D0D0DCDCDCE8E8E8F4F4F4FC28
S3150800CE20FCFCFCFCFCF8F8F8F4F4F4F0F0F0A8AC20
S3150800CE30ACB4B8B8C0C4C4D0D0D0DCDCDCE8E8E810
S3150800CE40F4F4F4FCFCFCFCFCFCF8F8F8F4F4F4F05C
S3150800CE50F0F0A8ACACB4B8B8C4C4C4D0D0D0DCDC4C
S3150800CE60DCE8E8E8F4F4F4FCFCFCFCFCFCF8F8F874
S3150800CE70F4F4F4F0F0F0A8ACACB4B8B8C4C4C4D0B8
S3150800CE80D0D0DCDCDCE8E8E8F4F4F4FCFCFCFCFCE0
S3150800CE90FCF8F8F8F4F4F4F0F0F0A8ACACB4B8B8D0
S3150800CEA0C4C4C4D0D0D0DCDCDCE8E8E8F4F4F4FC94
S3150800CEB0FCFCFCFCFCF8F8F8F4F4F4F0F0F0A8AC90
S3150800CEC0ACB4B8B8C4C4C4D0D0D0DCDCDCE8E8E87C
S3150800CED0F4F4F4FCFCFCFCFCFCF8F8F8F4F4F4F0CC
S3150800CEE0F0F0A8ACACB4B8B8C4C4C4D0D0D0DCDCBC
S3150800CEF0DCE8E8E8F4F4F4FCFCFCFCFCFCF8F8F8E4
S3150800CF00F4F4F4F0F0F0A8ACACB4B8B8C4C4C4D027
S3150800CF10D0D0DCDCDCE8E8E8F4F4F4FCFCFCFCFC4F
S3150800CF20FCF8F8F8F4F4F4F0F0F0A8ACACB4B8B83F
S3150800CF30C0C4C4D0D0D0DCDCDCE8E8E8F4F4F4FC07
S3150800CF40FCFCFCFCFCF8F8F8F4F4F4F0F0F0A8ACFF
S3150800CF50ACB4B8B8C0C4C4D0D0D0DCDCDCE8E8E8EF
S3150800CF60F4F4F4FCFCFCFCFCFCF8F8F8F4F4F4F03B
S3150800CF70F0F0A8ACACB4B8B8C4C4C4D0D0D0DCDC2B
S3150800CF80DCE8E8E8F4F4F4FCFCFCFCFCFCF8F8F853
S3150800CF90F4F4F4F0F0F0A8ACACB4B8B8C4C4C4D097
S3150800CFA0D0D0DCDCDCE8E8E8F4F4F4FCFCFCFCFCBF
S3150800CFB0FCF8F8F8F4F4F4F0F0F0A8ACACB4B8B8AF
S3150800CFC0C4C4C4D0D0D0DCDCDCE8E8E8F4F4F4FC73
S3150800CFD0FCFCFCFCFCF8F8F8F4F4F4F0F0F0A8AC6F
S3150800CFE0ACB4B8B8C4C4C4D0D0D0DCDCDCE8E8E85B
S3150800CFF0F4F4F4FCFCFCFCFCFCF8F8F8F4F4F4F0AB
S3150800D000F0F0A8ACACB4B8B8C4C4C4D0D0D0DCDC9A
S3150800D010DCE8E8E8F4F4F4FCFCFCFCFCFCF8F8F8C2
S3150800D020F4F4F4F0F0F0A8ACACB4B8B8C4C4C4D006
S3150800D030D0D0DCDCDCE8E8E8F4F4F4FCFCFCFCFC2E
S3150800D040FCF8F8F8F4F4F4F0F0F0A8ACACB4B8B81E
S3150800D050C0C4C4D0D0D0DCDCDCE8E8E8F4F4F4FCE6
S3150800D060FCFCFCFCFCF8F8F8F4F4F4F0F0F0A8ACDE
S3150800D070ACB4B8B8C0C4C4D0D0D0DCDCDCE8E8E8CE
S3150800D080F4F4F4FCFCFCFCFCFCF8F8F8F4F4F4F01A
S3150800D090F0F0A8ACACB4B8B8C4C4C4D0D0D0DCDC0A
S3150800D0A0DCE8E8E8F4F4F4FCFCFCFCFCFCF8F8F832
S3150800D0B0F4F4F4F0F0F0A8ACACB4B8B8C4C4C4D076
S3150800D0C0D0D0DCDCDCE8E8E8F4F4F4FCFCFCFCFC9E
S3150800D0D0FCF8F8F8F4F4F4F0F0F0A8ACACB4B8B88E
S3150800D0E0C4C4C4D0D0D0DCDCDCE8E8E8F4F4F4FC52
S3150800D0F0FCFCFCFCFCF8F8F8F4F4F4F0F0F0A8AC4E
S3150800D100ACB4B8B8C4C4C4D0D0D0DCDCDCE8E8E839
S3150800D110F4F4F4FCFCFCFCFCFCF8F8F8F4F4F4F089
S3150800D120F0F0A8ACACB4B8B8C4C4C4D0D0D0DCDC79
S3150800D130DCE8E8E8F4F4F4FCFCFCFCFCFCF8F8F8A1
S3150800D140F4F4F4F0F0F0A8ACACB4B8B8C4C4C4D0E5
S3150800D150D0D0DCDCDCE8E8E8F4F4F4FCFCFCFCFC0D
S3150800D160FCF8F8F8F4F4F4F0F0F0A8ACACB4B8B8FD
S3150800D170C0C4C4D0D0D0DCDCDCE8E8E8F4F4F4FCC5
S3150800D180FCFCFCFCFCF8F8F8F4F4F4F0F0F0A8ACBD
S3150800D190ACB4B8B8C0C4C4D0D0D0DCDCDCE8E8E8AD
S3150800D1A0F4F4F4FCFCFCFCFCFCF8F8F8F4F4F4F0F9
S3150800D1B0F0F0A8ACACB4B8B8C4C4C4D0D0D0DCDCE9
S3150800D1C0DCE8E8E8F4F4F4FCFCFCFCFCFCF8F8F811
S3150800D1D0F4F4F4F0F0F0A8ACACB4B8B8C4C4C4D055
S3150800D1E0D0D0DCDCDCE8E8E8F4F4F4FCFCFCFCFC7D
S3150800D1F0FCF8F8F8F4F4F4F0F0F0A8ACACB4B8B86D
S3150800D200C4C4C4D0D0D0DCDCDCE8E8E8F4F4F4FC30
S3150800D210FCFCFCFCFCF8F8F8F4F4F4F0F0F0A8AC2C
S3150800D220ACB4B8B8C4C4C4D0D0D0DCDCDCE8E8E818
S3150800D230F4F4F4FCFCFCFCFCFCF8F8F8F4F4F4F068
S3150800D240F0F0A8ACACB4B8B8C4C4C4D0D0D0DCDC58
S3150800D250DCE8E8E8F4F4F4FCFCFCFCFCFCF8F8F880
S3150800D260F4F4F4F0F0F0A8ACACB4B8B8C4C4C4D0C4
S3150800D270D0D0DCDCDCE8E8E8F4F4F4FCFCFCFCFCEC
S3150800D280FCF8F8F8F4F4F4F0F0F0A8ACACB4B8B8DC
S3150800D290C0C4C4D0D0D0DCDCDCE8E8E8F4F4F4FCA4
S3150800D2A0FCFCFCFCFCF8F8F8F4F4F4F0F0F0A8AC9C
S3150800D2B0ACB4B8B8C0C4C4D0D0D0DCDCDCE8E8E88C
S3150800D2C0F4F4F4FCFCFCFCFCFCF8F8F8F4F4F4F0D8
S3150800D2D0F0F0A8ACACB4B8B8C4C4C4D0D0D0DCDCC8
S3150800D2E0DCE8E8E8F4F4F4FCFCFCFCFCFCF8F8F8F0
S3150800D2F0F4F4F4F0F0F0A8ACACB4B8B8C4C4C4D034
S3150800D300D0D0DCDCDCE8E8E8F4F4F4FCFCFCFCFC5B
S3150800D310FCF8F8F8F4F4F4F0F0F0A8ACACB4B8B84B
S3150800D320C4C4C4D0D0D0DCDCDCE8E8E8F4F4F4FC0F
S3150800D330FCFCFCFCFCF8F8F8F4F4F4F0F0F0A8AC0B
S3150800D340ACB4B8B8C4C4C4D0D0D0DCDCDCE8E8E8F7
S3150800D350F4F4F4FCFCFCFCFCFCF8F8F8F4F4F4F047
S3150800D360F0F0A8ACACB4B8B8C4C4C4D0D0D0DCDC37
S3150800D370DCE8E8E8F4F4F4FCFCFCFCFCFCF8F8F85F
S3150800D380F4F4F4F0F0F0A8ACACB4B8B8C4C4C4D0A3
S3150800D390D0D0DCDCDCE8E8E8F4F4F4FCFCFCFCFCCB
S3150800D3A0FCF8F8F8F4F4F4F0F0F0A8ACACB4B8B8BB
S3150800D3B0C0C4C4D0D0D0DCDCDCE8E8E8F4F4F4FC83
S3150800D3C0FCFCFCFCFCF8F8F8F4F4F4F0F0F0A8AC7B
S3150800D3D0ACB4B8B8C0C4C4D0D0D0DCDCDCE8E8E86B
S3150800D3E0F4F4F4FCFCFCFCFCFCF8F8F8F4F4F4F0B7
S3150800D3F0F0F0A8ACACB4B8B8C4C4C4D0D0D0DCDCA7
S3150800D400DCE8E8E8F4F4F4FCFCFCFCFCFCF8F8F8CE
S3150800D410F4F4F4F0F0F0A8ACACB4B8B8C4C4C4D012
S3150800D420D0D0DCDCDCE8E8E8F4F4F4FCFCFCFCFC3A
S3150800D430FCF8F8F8F4F4F4F0F0F0A8ACACB4B8B82A
S3150800D440C4C4C4D0D0D0DCDCDCE8E8E8F4F4F4FCEE
S3150800D450FCFCFCFCFCF8F8F8F4F4F4F0F0F0A8ACEA
S3150800D460ACB4B8B8C4C4C4D0D0D0DCDCDCE8E8E8D6
S3150800D470F4F4F4FCFCFCFCFCFCF8F8F8F4F4F4F026
S3150800D480F0F0A8ACACB4B8B8C4C4C4D0D0D0DCDC16
S3150800D490DCE8E8E8F4F4F4FCFCFCFCFCFCF8F8F83E
S3150800D4A0F4F4F4F0F0F0A8ACACB4B8B8C4C4C4D082
S3150800D4B0D0D0DCDCDCE8E8E8F4F4F4FCFCFCFCFCAA
S3150800D4C0FCF8F8F8F4F4F4F0F0F0A8ACACB4B8B89A
S3150800D4D0C0C4C4D0D0D0DCDCDCE8E8E8F4F4F4FC62
S3150800D4E0FCFCFCFCFCF8F8F8F4F4F4F0F0F0A8AC5A
S3150800D4F0ACB4B8B8C0C4C4D0D0D0DCDCDCE8E8E84A
S3150800D500F4F4F4FCFCFCFCFCFCF8F8F8F4F4F4F095
S3150800D510F0F0A8ACACB4B8B8C4C4C4D0D0D0DCDC85
S3150800D520DCE8E8E8F4F4F4FCFCFCFCFCFCF8F8F8AD
S3150800D530F4F4F4F0F0F0FC6C48FC6C48FC6C48FC25
S3150800D5406C48FC6C48FC6C48FC6C48FC6C48FC6CF1
S3150800D55048FC6C48FC6C48FC6C48FC6C48FC6C4805
S3150800D560FC6C48FC6C48FC6C48FC6C48FC6C48FC41
S3150800D5706C48FC6C48FC6C48FC6C48FC6C48FC54D9
S3150800D58000FC6C44FC6C48FC6C48FC6C48FC6C4821
S3150800D590FC6C48FC6C48FC6C48FC6C48FC6C44FC15
S3150800D5A05400000000000000FC6C44FC6C48FC6C55
S3150800D5B048FC6C48FC6C48FC6C48FC6C48FC6C44A9
S3150800D5C000000000000080FCFCA8D8FCB0DCFCB41D
S3150800D5D0E0FCC0E4FCC4E8FCCCECFCD4F0FCD8F4D9
S3150800D5E0FCD0F0FCCCECFCFCFCFCA0D4FCA8D8FCE1
S3150800D5F0B0DCFCB8E0FCBCE4FCC4E8FCCCECFCD435
S3150800D600F0FCD8F4FCD0F0FCC8ECFCC0E8FCA0D4D4
S3150800D610FCA8D8FCB0DCFCB4E0FCBCE4FCC4E8FC28
S3150800D620CCECFCD4F0FCD8F4FCD0F0FCC8ECFCC084
S3150800D630E8FCA0D4FCA8D8FCB0DCFCB8E0FCBCE450
S3150800D640FCC4E8FCCCECFCD4F0FCD8F4FCD0F0FC30
S3150800D650C8ECFCC0E8FCA0D4FCA8D8FCB0DCFCB83C
S3150800D660E0FCBCE4FCC4E8FCCCECFCD4F0FCD8F44C
S3150800D670FCD0F0FCC8ECFCC0E8FCA0D4FCA8D8FCA4
S3150800D680B0DCFCB8E0FCBCE4FCC4E8FCCCECFCD4A4
S3150800D690F0FCD8F4FCD0F0FCC8ECFCC0E8FCA0D444
S3150800D6A0FCA8D8FCB0DCFCB4E0FCBCE4FCC4E8FC98
S3150800D6B0CCECFCD4F0FCD8F4FCD0F0FCC8ECFCC0F4
S3150800D6C0E8FCA0D4FCA8D8FCB0DCFCB4E0FCBCE4C4
S3150800D6D0FCC4E8FCCCECFCD4F0FCD8F4FCD0F0FCA0
S3150800D6E0C8ECFCC0E8FCA0D4FCA8D8FCB0DCFCB8AC
S3150800D6F0E0FCBCE4FCC4E8FCCCECFCD4F0FCD8F4BC
S3150800D700FCD0F0FCC8ECFCC0E8FCA0D4FCA8D8FC13
S3150800D710B0DCFCB8E0FCBCE4FCC4E8FCCCECFCD413
S3150800D720F0FCD8F4FCD0F0FCC8ECFCC0E8FCA0D4B3
S3150800D730FCA8D8FCB0DCFCB4E0FCBCE4FCC4E8FC07
S3150800D740CCECFCD4F0FCD8F4FCD0F0FCC8ECFCC063
S3150800D750E8FCA0D4FCA8D8FCB0DCFCB8E0FCBCE42F
S3150800D760FCC4E8FCCCECFCD4F0FCD8F4FCD0F0FC0F
S3150800D770C8ECFCC0E8FCA0D4FCA8D8FCB0DCFCB81B
S3150800D780E0FCBCE4FCC4E8FCCCECFCD4F0FCD8F42B
S3150800D790FCD0F0FCC8ECFCC0E8FCA0D4FCA8D8FC83
S3150800D7A0B0DCFCB8E0FCBCE4FCC4E8FCCCECFCD483
S3150800D7B0F0FCD8F4FCD0F0FCC8ECFCC0E8FCA0D423
S3150800D7C0FCA8D8FCB0DCFCB4E0FCBCE4FCC4E8FC77
S3150800D7D0CCECFCD4F0FCD8F4FCD0F0FCC8ECFCC0D3
S3150800D7E0E8FCA0D4FCA8D8FCB0DCFCB4E0FCBCE4A3
S3150800D7F0FCC4E8FCCCECFCD4F0FCD8F4FCD0F0FC7F
S3150800D800C8ECFCC0E8FCA0D4FCA8D8FCB0DCFCB88A
S3150800D810E0FCBCE4FCC4E8FCCCECFCD4F0FCD8F49A
S3150800D820FCD0F0FCC8ECFCC0E8FCA0D4FCA8D8FCF2
S3150800D830B0DCFCB8E0FCBCE4FCC4E8FCCCECFCD4F2
S3150800D840F0FCD8F4FCD0F0FCC8ECFCC0E8FCA0D492
S3150800D850FCA8D8FCB0DCFCB4E0FCBCE4FCC4E8FCE6
S3150800D860CCECFCD4F0FCD8F4FCD0F0FCC8ECFCC042
S3150800D870E8FCA0D4FCA8D8FCB0DCFCB8E0FCBCE40E
S3150800D880FCC4E8FCCCECFCD4F0FCD8F4FCD0F0FCEE
S3150800D890C8ECFCC0E8FCA0D4FCA8D8FCB0DCFCB8FA
S3150800D8A0E0FCBCE4FCC4E8FCCCECFCD4F0FCD8F40A
S3150800D8B0FCD0F0FCC8ECFCC0E8FCA0D4FCA8D8FC62
S3150800D8C0B0DCFCB8E0FCBCE4FCC4E8FCCCECFCD462
S3150800D8D0F0FCD8F4FCD0F0FCC8ECFCC0E8FCA0D402
S3150800D8E0FCA8D8FCB0DCFCB4E0FCBCE4FCC4E8FC56
S3150800D8F0CCECFCD4F0FCD8F4FCD0F0FCC8ECFCC0B2
S3150800D900E8FCA0D4FCA8D8FCB0DCFCB4E0FCBCE481
S3150800D910FCC4E8FCCCECFCD4F0FCD8F4FCD0F0FC5D
S3150800D920C8ECFCC0E8FCA0D4FCA8D8FCB0DCFCB869
S3150800D930E0FCBCE4FCC4E8FCCCECFCD4F0FCD8F479
S3150800D940FCD0F0FCC8ECFCC0E8FCA0D4FCA8D8FCD1
S3150800D950B0DCFCB8E0FCBCE4FCC4E8FCCCECFCD4D1
S3150800D960F0FCD8F4FCD0F0FCC8ECFCC0E8FCA0D471
S3150800D970FCA8D8FCB0DCFCB4E0FCBCE4FCC4E8FCC5
S3150800D980CCECFCD4F0FCD8F4FCD0F0FCC8ECFCC021
S3150800D990E8FCA0D4FCA8D8FCB0DCFCB8E0FCBCE4ED
S3150800D9A0FCC4E8FCCCECFCD4F0FCD8F4FCD0F0FCCD
S3150800D9B0C8ECFCC0E8FCA0D4FCA8D8FCB0DCFCB8D9
S3150800D9C0E0FCBCE4FCC4E8FCCCECFCD4F0FCD8F4E9
S3150800D9D0FCD0F0FCC8ECFCC0E8FCA0D4FCA8D8FC41
S3150800D9E0B0DCFCB8E0FCBCE4FCC4E8FCCCECFCD441
S3150800D9F0F0FCD8F4FCD0F0FCC8ECFCC0E8FCA0D4E1
S3150800DA00FCA8D8FCB0DCFCB4E0FCBCE4FCC4E8FC34
S3150800DA10CCECFCD4F0FCD8F4FCD0F0FCC8ECFCC090
S3150800DA20E8FCA0D4FCA8D8FCB0DCFCB4E0FCBCE460
S3150800DA30FCC4E8FCCCECFCD4F0FCD8F4FCD0F0FC3C
S3150800DA40C8ECFCC0E8FCA0D4FCA8D8FCB0DCFCB848
S3150800DA50E0FCBCE4FCC4E8FCCCECFCD4F0FCD8F458
S3150800DA60FCD0F0FCC8ECFCC0E8FCA0D4FCA8D8FCB0
S3150800DA70B0DCFCB8E0FCBCE4FCC4E8FCCCECFCD4B0
S3150800DA80F0FCD8F4FCD0F0FCC8ECFCC0E8FCA0D450
S3150800DA90FCA8D8FCB0DCFCB4E0FCBCE4FCC4E8FCA4
S3150800DAA0CCECFCD4F0FCD8F4FCD0F0FCC8ECFCC000
S3150800DAB0E8FCA0D4FCA8D8FCB0DCFCB8E0FCBCE4CC
S3150800DAC0FCC4E8FCCCECFCD4F0FCD8F4FCD0F0FCAC
S3150800DAD0C8ECFCC0E8FCA0D4FCA8D8FCB0DCFCB8B8
S3150800DAE0E0FCBCE4FCC4E8FCCCECFCD4F0FCD8F4C8
S3150800DAF0FCD0F0FCC8ECFCC0E8FCA0D4FCA8D8FC20
S3150800DB00B0DCFCB8E0FCBCE4FCC4E8FCCCECFCD41F
S3150800DB10F0FCD8F4FCD0F0FCC8ECFCC0E8FCA0D4BF
S3150800DB20FCA8D8FCB0DCFCB4E0FCBCE4FCC4E8FC13
S3150800DB30CCECFCD4F0FCD8F4FCD0F0FCC8ECFCC06F
S3150800DB40E8FCA0D4FCA8D8FCB0DCFCB4E0FCBCE43F
S3150800DB50FCC4E8FCCCECFCD4F0FCD8F4FCD0F0FC1B
S3150800DB60C8ECFCC0E8FCA0D4FCA8D8FCB0DCFCB827
S3150800DB70E0FCBCE4FCC4E8FCCCECFCD4F0FCD8F437
S3150800DB80FCD0F0FCC8ECFCC0E8FCECA860ECB0707B
S3150800DB90ECB87CF0C088F4C894F4D0A4F8D8B0FCEB
S3150800DBA0DCBCFCE4C4FCDCB8FCD4A8FCD098ECA82B
S3150800DBB058F0B068F0B874F4C084F4C890F8CCA0F3
S3150800DBC0F8D4ACFCDCBCFCE4C4FCDCB4FCD4A4FC9B
S3150800DBD0D094ACACACB8B8B8C4C4C0D0D0D0DCDC37
S3150800DBE0D8E8E8E4F4F4F0FCFCFCFCFCFCF8F8F8F3
S3150800DBF0F4F4F4F0F0ECA8ACACB4B8B8C0C4C4D033
S3150800DC00D0D0DCDCDCE8E8E8F4F4F4FCFCFCFCFC52
S3150800DC10FCF8F8F8F4F4F4F0F0F0E43004E4300436
S3150800DC20E43004E43004E43004E43004E43004E48A
S3150800DC303004E43004E43004E43004E43004E4401E
S3150800DC4014E43004E43004E43004E43004E430043A
S3150800DC50E43004E43004E43004E43004E43004E856
S3150800DC604014D418187C4014E83004E43004E43036
S3150800DC7004E43004E43004E43004E43004E8300416
S3150800DC80E84014DC18187C18187C18187C6448E4DA
S3150800DC903C14E83408E83004E83004E83408E43C86
S3150800DCA014E8644818187C18187C00C1814001C023
S3150800DCB0804101C0804100C1814001C0804100C14E
S3150800DCC0814000C1814001C0804101C0804100C13E
S3150800DCD0814000C1814001C0804100C1814001C02E
S3150800DCE0804101C0804100C1814001C0804100C11E
S3150800DCF0814000C1814001C0804100C1814001C00E
S3150800DD00804101C0804100C1814000C1814001C0FD
S3150800DD10804101C0804100C1814001C0804100C1ED
S3150800DD20814000C1814001C0804101C0804100C1DD
S3150800DD30814000C1814001C0804100C1814001C0CD
S3150800DD40804101C0804100C1814000C1814001C0BD
S3150800DD50804101C0804100C1814001C0804100C1AD
S3150800DD60814000C1814001C0804100C1814001C09D
S3150800DD70804101C0804100C1814001C0804100C18D
S3150800DD80814000C1814001C0804101C0804100C17D
S3150800DD90814000C1814001C0804100C1814001C06D
S3150800DDA0804101C0804100C1814000C0C101C30358
S3150800DDB002C2C60607C705C5C404CC0C0DCD0FCFD5
S3150800DDC0CE0E0ACACB0BC90908C8D81819D91BDB45
S3150800DDD0DA1A1EDEDF1FDD1D1CDC14D4D515D71795
S3150800DDE016D6D21213D311D1D010F03031F133F345
S3150800DDF0F23236F6F737F53534F43CFCFD3DFF3F95
S3150800DE003EFEFA3A3BFB39F9F83828E8E929EB2BC4
S3150800DE102AEAEE2E2FEF2DEDEC2CE42425E527E754
S3150800DE20E62622E2E323E12120E0A06061A163A3C4
S3150800DE30A26266A6A767A56564A46CACAD6DAF6F54
S3150800DE406EAEAA6A6BAB69A9A86878B8B979BB7BC4
S3150800DE507ABABE7E7FBF7DBDBC7CB47475B577B714
S3150800DE60B67672B2B373B17170B050909151935344
S3150800DE70529296565797559594549C5C5D9D5F9F14
S3150800DE809E5E5A9A9B5B99595898884849894B8B44
S3150800DE908A4A4E8E8F4F8D4D4C8C448485458747D4
S3150800DEA0468682424383418180400000000000008C
S3150800DEB07A36CB3E48504C3FBC059A3F764FCE3F0C
S3150800DEC0787A01409EEF1B40107A3640F90F514090
S3150800DED040A46B40121483408C4A9040D26F9D40F8
S3150800DEE04182AA400681B740F46CC4405249D140E9
S3150800DEF06519DE4048E1EA40B5A6F7404C370241CD
S3150800DF001B9E0841D5090F41B37B154188F41B4177
S3150800DF105474224116FB2841CE882F41151D3641DF
S3150800DF2017B73C416D56434144FA494134A2504122
S3150800DF303C4E5741F4FD5D418AB06441CF666B4162
S3150800DF408A1F72418CDB78419A997F41432D834120
S3150800DF50F38E8641DEF18941D0558D4193BA9041C1
S3150800DF605C209441F78697412FEE9A4139569E4197
S3150800DF70ABBEA1418727A54104FA97999999D93F3C
S3150800DF80AF788E1DC571CC3F9FC678D0099AC33F1E
S3150800DF90935555555555E53F599322942449D23FF3
S3150800DFA0DE03CB966446C73F44523EDF12F1C23FBA
S3150800DFB00000000000000000D8DF0008C8000020AC
S3150800DFC0780100006A22000844E0000840020020A8
S3150800DFD0C01A00002A590008C1033D88135B0101D5
S3150800DFE0082C0203040425060708097CA24A042112
S3150800DFF07915011229255940013910296666663FA7
S3150800E000295C4F3FBE9F3A3F2BF6273F5A2A173FB8
S3150800E010840C083F58E3F43E2C66DC3EEA5BC63EB9
S3150800E020EC85B23E001042448CE45CA0F4448CE0DB
S3150800E0303C84DC3480DC0312803F43C84105149AD3
S3090800E040998940006C
S705080018C515
